:020000040800F2
:10000000488400206902000821520008D9440008F1
:100010001D52000881190008257200080000000028
:100020000000000000000000000000000164000863
:100030000D200008000000009154000869640008C9
:10004000830200088302000883020008830200087C
:10005000830200088302000883020008830200086C
:1000600083020008112000081D20000883020008F8
:10007000F11E0008011F0008830200088302000827
:10008000830200088302000883020008830200083C
:100090008302000883020008830200082920000868
:1000A000830200088302000883020008830200081C
:1000B000830200088302000883020008830200080C
:1000C00083020008830200088302000883020008FC
:1000D00083020008830200088302000883020008EC
:1000E00083020008830200088302000883020008DC
:1000F00083020008830200088302000883020008CC
:1001000083020008830200088302000883020008BB
:1001100083020008830200088302000883020008AB
:1001200083020008111F0008211F0008311F00086A
:10013000830200088302000883020008830200088B
:10014000830200088302000883020008830200087B
:1001500083020008411F0008830200080D72000896
:10016000830200088302000883020008830200085B
:1001700083020008830200088302000800000000D8
:10018000830200088302000800F002F800F05CF827
:100190000AA090E8000C82448344AAF10107DA45E2
:1001A00001D100F051F8AFF2090EBAE80F0013F0D8
:1001B000010F18BFFB1A43F001031847F0CB0000F2
:1001C00010CC00000A444FF0000C10F8013B13F073
:1001D000070408BF10F8014B1D1108BF10F8015BA0
:1001E000641E05D010F8016B641E01F8016BF9D193
:1001F00013F0080F1EBF10F8014BAD1C0C1B09D1EA
:100200006D1E58BF01F801CBFAD505E014F8016B5B
:1002100001F8016B6D1EF9D59142D6D370470000ED
:100220000023002400250026103A28BF78C1FBD8FF
:10023000520728BF30C148BF0B6070471FB50CF094
:100240001CFB1FBD10B510BD00F062F91146FFF791
:10025000F5FF07F0B1F800F080F903B4FFF7F2FF03
:1002600003BC00F083F900000948804709480047B3
:10027000FEE7FEE7FEE7FEE7FEE7FEE7FEE7FEE756
:10028000FEE7FEE704480549054A064B70470000B3
:100290002165000889010008487E0020488400206C
:1002A000488000204880002053EA020C00F069805A
:1002B0002DE9F04B4FF00006002B1FBFB3FA83F57A
:1002C00003FA05F424FA05F65E4012BF1643B2FAAB
:1002D00082F502FA05F4C5F120051EBF22FA05FCDD
:1002E00044EA0C04203556EA044C4FEA144418BF83
:1002F000641C4FF000084FF00009904271EB030CB2
:1003000039D3002919BFB1FA81F701FA07F6B0FA1B
:1003100080F700FA07F6C7F120071EBF20FA07FC96
:1003200046EA0C062037B6FBF4FCA7EB0507103FA6
:1003300007F01F0BCBF120062CFA06F60CFA0BFB8C
:1003400044BFB3460026202FA4BF5E464FF0000BEB
:100350005BEA060C08BF4FF0010B19EB0B0948EBE9
:100360000608ABFB027C06FB02CC0BFB03CCC01BDC
:1003700071EB0C01C1E70B46024641464846BDE819
:10038000F08B13B5084318BF4FF0FF300146AFF3B1
:100390000080BDE81C407047032A40F2308010F016
:1003A000030C00F0158011F8013BBCF1020F624410
:1003B00098BF11F801CB00F8013B38BF11F8013BA1
:1003C000A2F1040298BF00F801CB38BF00F8013B4E
:1003D00011F0030300F02580083AC0F0088051F8BE
:1003E000043B083A51F804CBA0E80810F5E7121DC9
:1003F0005CBF51F8043B40F8043BAFF30080D207E8
:1004000024BF11F8013B11F801CB48BF11F8012BB3
:1004100024BF00F8013B00F801CB48BF00F8012BD6
:10042000704710B5203AC0F00B80B1E81850A0E832
:100430001850B1E81850A0E81850203ABFF4F5AFB2
:100440005FEA027C24BFB1E81850A0E8185044BF0E
:1004500018C918C0BDE810405FEA827C24BF51F87B
:10046000043B40F8043B08BF7047D20728BF31F86F
:10047000023B48BF11F8012B28BF20F8023B48BFC0
:1004800000F8012B704702F0FF0343EA032242EA1F
:10049000024200F002B84FF0000200B51346944645
:1004A0009646203922BFA0E80C50A0E80C50B1F1CC
:1004B0002001BFF4F7AF090728BFA0E80C5048BFE0
:1004C0000CC05DF804EB890028BF40F8042B08BF7E
:1004D000704748BF20F8022B11F0804F18BF00F87A
:1004E000012B704770477047704710B500F008F84F
:1004F000006810BD10B5044600F002F8046010BD9D
:10050000004870474001002000487047400100202B
:100510007546FFF7F9FFAE4605006946534620F0E1
:100520000700854618B020B5FFF7ACFEBDE82040B7
:100530004FF000064FF000074FF000084FF0000B9F
:10054000AC46ACE8C009ACE8C009ACE8C009ACE80E
:10055000C00921F007018D46704710B50446AFF37E
:1005600000802046BDE81040FFF777BE0149182003
:10057000ABBEFEE72600020070470000B0B52DEDCF
:10058000028B044600284FF0FF0061D00D46002981
:100590005ED095ED000A95ED011A95ED022A95EDD4
:1005A000033A20EE010A22EE033A21EE011A22EE6E
:1005B000022A31EE021A30EE030A31EE011AB7EECA
:1005C000008A30EE000A78EE410A09F055FFB0EEDD
:1005D000401A95ED000A95ED012A95ED023A95ED48
:1005E000034A20EE030A24EE022A30EE420A30EEDD
:1005F000000AB0EEC02AB4EE482AF1EE10FA84EDFB
:10060000011A02DA09F036FC01E006F07BFE84ED07
:10061000020A95ED000A95ED011A95ED032A95ED74
:10062000023A20EE020A21EE031A30EE010A23EE0E
:10063000031A22EE022A32EE011A31EE011A30EECE
:10064000000A78EE410A09F017FF002084ED000A45
:1006500040B2BDEC028BB0BD70B52DED028B002811
:100660004FD0B7EE001A81EE000A0D4604464FF057
:100670007E51002D80ED040A4FF00000C4E9001007
:10068000A060E06000F09F80D5E900600CF054F8B5
:1006900041EC180B30460CF04FF841EC110BB0EE6A
:1006A000480AF0EE680A09F0E7FD51EC100B0BF078
:1006B00001FA95ED000AB5EE400AF1EE10FA22D1EA
:1006C00095ED010AB5EE400AF1EE10FA1BD195ED59
:1006D000020AB5EE400AF1EE10FA14D140F2C560FC
:1006E000C3F64D7044F62D214AF2564244F2AD73E2
:1006F000C3F60D41CBF63932C3F619730FC400208F
:1007000061E0FF205FE09FED321A00EE100AB4EEC8
:10071000410AF1EE10FA1EDCB5EE400AF1EE10FAD5
:1007200019DB9FED2C2AB4EE420AF1EE10FA25DC1B
:10073000B4EE410AF1EE10FA20DB9FED271AB4EE79
:10074000410AF1EE10FA2CDCB4EE420AF1EE10FA96
:1007500027DB002037E045F66E10C3F67F7045F2C8
:100760000C3148F6AB0249F28553C3F6B011CBF613
:10077000BB32C3F697530FC4002024E040F2C5609B
:10078000C3F64D7044F62D214AF2564244F2AD7341
:10079000C3F60D41CBF63932C3F619730FC40020EE
:1007A00011E040F2C560C3F64D7044F62D214AF2C7
:1007B000564244F2AD73C3F60D41CBF63932C3F65F
:1007C00019730FC4002040B2BDEC028B70BD00BF96
:1007D000DB0FC9BFDB0F49C00000B4C2B0B52DEDBF
:1007E000108B8EB0044600284FF0FF0018BF002980
:1007F00004D140B20EB0BDEC108BB0BD002AF8D0D1
:1008000040F204054EF69E70C2F20005C3F6275072
:100810002860C3B193ED00EA93ED01FAD3ED028AAB
:10082000B5EE40EAF1EE10FA11D1B5EE40FAF1EE74
:1008300010FA0CD1F5EE408AF1EE10FA07D12046FD
:1008400000F094FAD5E7204600F090FAD1E792ED57
:10085000000A92ED011A94ED014A94ED025A92EDCC
:10086000022A94ED036A94ED003A24EE407A61EE98
:10087000050A37EE607A62EE060A37EE607A60EEBD
:10088000030A62EE051A71EEA00A61EE061A70EE16
:10089000E10A61EE031A62EE042A22EE032A21EE37
:1008A000041A91ED00DA71EEE21A20EE066A31EEDA
:1008B000021A20EE050A36EE216AD1ED019AD1ED39
:1008C00002AA31EE400AB6EE001AB5EE40DA27EE83
:1008D000015A60EE810A26EE017AF1EE10FA20EE5E
:1008E000016A0AD1F5EE409AF1EE10FA05D1F5EE63
:1008F00040AAF1EE10FA00F0EC812DEE0D0A29EE7F
:10090000A91A30EE010A2AEEAA1A30EE010A8DED7C
:100910000D6A8DED0C7ACDED0B0A8DED0A5A04F0BF
:1009200049F82DEE001A8DED071A29EE801A2AEEED
:10093000800A8DED081A8DED090A2EEE0E0A2FEEB3
:100940000F1A30EE010A28EEA81A30EE010A04F060
:1009500031F894ED001A6EEE00DA6FEE00AA94ED15
:10096000034A31EE01EA68EE808A94ED012A94EDA3
:10097000023A2AEE8E6A61EE01EA8DED026A28EEF5
:100980008E0A2DEEAE5A26EE046A62EE02BA35EEFB
:10099000465A20EE036A36EE055A2DEEAB6A32EE69
:1009A00002FA36EE055A2AEE8F6A23EE066A36EE12
:1009B000055A28EE8F6A26EE046A63EE03FA36EED5
:1009C000055A2DEEAF6A24EE048A35EE465A2DEE16
:1009D000886A2DEE8E9A35EE465A29EE046A2AEE82
:1009E000AE7A37EE066A22EE000A2DEE8FAA36EEB8
:1009F000400A23EE0A6A36EE000A2AEEAB6A30EEAF
:100A0000460A2AEEAF6A73EE039A36EE000A28EE23
:100A1000A96A24EE066A36EE000A2AEE886A30EEEB
:100A2000460A25EE055A20EE000A35EE000A21EEB0
:100A300002BA21EE035A21EE041A8DED051A22EEB8
:100A4000031A8DED031A23EE041A8DED041A34EE09
:100A5000041A8DED015A22EE04CA6EEE03CA8DED22
:100A6000061A29EE84DA03F0A5FF94ED013A94ED1D
:100A7000022A9DED021A29EE024A21EE031A31EEF6
:100A8000444A94ED031A28EEAE5A35EE044A2AEE93
:100A9000015A35EE044A28EEAB5AF7EE001A34EE4E
:100AA000454A2AEEA95A81EE800A25EE015A35EE12
:100AB000044A28EEAF5A34EE454A28EE885A75EEBD
:100AC000042A3CEE0C4A9DED075A34EE6C4A34EE93
:100AD000454A3BEE0B5A9DED086A35EE0D5A35EE50
:100AE000465A2FEE056A29EE847AF6EE007A76EE03
:100AF000470A37EEEF6A36EE486A9DED018A20EE2E
:100B0000066A3CEE487A27EE227A36EE076A36EE1F
:100B10006D7A22EE226A66EE073A70EEE33ADDED78
:100B2000050ADDED034A60EE015A74EEE00ADDEDE0
:100B3000044A60EE200A7BEE244A64EEA24A70EE7C
:100B4000A40A63EE224A70EEEA0A74EEE56A66EEE3
:100B5000A06A77EEEB7A76EEA33A78EE0C6A77EE3F
:100B6000EF7A60EE266A67EEA27A76EEA76A76EEF4
:100B7000E86A60EE027ADDED068A27EEA68A38EE94
:100B800023CA68EE843A2EEE058A78EE233A3BEECD
:100B9000AB8A71EEC81A3FEEAF8A71EEC81A9DEDAE
:100BA000098A21EE22AA71EEC81AB1EE008A23EE5C
:100BB000089A21EE899A73EEC93A94ED009A2AEECA
:100BC00007BA73EE8B3A29EE22BA77EE8B7A67EE8C
:100BD000A07A72EEA22A77EEA33A63EE227A75EE3D
:100BE000E75A65EEA65A35EEA3DA68EE853A6EEE60
:100BF000045A73EEE53A62EE085A65EEA11A73EEF6
:100C0000E11AF8EE003A60EE233A62EE235A75EEEE
:100C1000CB5A65EE875A20EE033A71EEA51A73EEB1
:100C20000A5A20EE090A22EE222A65EEA05A30EE78
:100C3000422A75EEA11A22EE262A23EE811A32EEFE
:100C4000218A2FEE042A29EE854A31EE241A34EE49
:100C5000022A21EE071A36EE400A32EE011A20EE81
:100C6000200A30EE010A23EE261A31EE009A2CEE0D
:100C70000C0A2DEE0D1A30EE010A28EE081A31EE9C
:100C8000000A29EE091A31EE000A03F093FE95EDF1
:100C9000004A9DED0A5A20EE0C1ADDED0B0A20EEFB
:100CA0000D2A24EE011A9DED0C7A9DED0D6A20EEC1
:100CB000083A20EE090A35EE415A24EE021A70EE87
:100CC000C10A24EE031A24EE000A37EE417A36EE0A
:100CD000406A94ED043A94ED000A94ED011A25EE71
:100CE000035A94ED022A30EE050A20EE835A94ED61
:100CF000034A35EE011A27EE035A35EE022A26EE94
:100D0000033A84ED000A84ED011A20EE000A21EE78
:100D1000011A33EE043A30EE010A22EE021A30EEE6
:100D2000010A23EE031A30EE010A84ED022A84ED53
:100D3000033A03F03FFE94ED001A94ED012A94ED7E
:100D4000023A94ED034A20EE011A20EE022A20EE28
:100D5000033A20EE040A002084ED001A84ED012AF3
:100D600084ED023A84ED030A43E50000B0B52DEDB1
:100D7000108B044600284FF0FF0018BF002900F038
:100D80006981002A00F0668140F2040542F60230D3
:100D9000C2F20005C3F60750286092ED000A92EDFA
:100DA000011A94ED014A94ED025A92ED022A94ED53
:100DB000036A94ED003A24EE407A61EE050A37EEBC
:100DC000607A62EE060A37EE607A60EE030A62EE3F
:100DD000051A71EEA00A61EE061A70EEE10A61EEE4
:100DE000031A62EE042A22EE032A21EE041A91ED80
:100DF00000CA71EEE21A20EE066A31EE021A20EE07
:100E0000050A36EE216A91ED01DA91ED02EA31EE42
:100E1000400AB6EE001AB5EE40CA27EE01BA20EE3F
:100E200081AA26EE019AF1EE10FA20EE018A0AD18B
:100E3000B5EE40DAF1EE10FA05D1B5EE40EAF1EE8A
:100E400010FA00F0BC802CEE0C0A2DEE0D1A30EEDC
:100E5000010A2EEE0E1A30EE010A03F0ABFD94EDFE
:100E6000003A94ED025AF1EE001A2CEE001A94EDBD
:100E7000014A75EE050A63EE212A65EE053A62EE37
:100E8000A34A61EE205A74EEA54A64EE045A2DEE90
:100E9000002A94ED036A34EE047A62EEA52A72EE1B
:100EA000A42A62EE074A32EEE4CA76EE062A64EE1F
:100EB000214A66EE066A64EEA67A21EE22DA77EE21
:100EC000CD7A23EE03DA2DEE21DA2EEE000A24EE9F
:100ED0000DEA33EE033A7EEE277A22EE03EA77EE4E
:100EE000CE7AB2EE00EA24EE0E4A77EEE47A24EEF1
:100EF00025FA7FEE277A24EE234A34EE274A60EE65
:100F0000244A34EE84FA2DEE054A21EE033A33EEFC
:100F1000043A25EE0E4A25EE215A65EE264A33EEB6
:100F2000243A62EE222A33EE623A33EE453A65EE17
:100F3000842A32EE833A24EE234A34EE033A20EE3A
:100F4000050A30EE03DA21EE070A25EEA11A21EE9A
:100F5000061A31EE400A23EEA11A26EE011A30EEEF
:100F6000010A22EE201A30EE41EA2CEE0C0A2FEE96
:100F70000F1A30EE010A2DEE0D1A31EE000A2EEE98
:100F80000E1A31EE000A03F015FD95ED004A20EE31
:100F90000C1A20EE0F2A24EE011A20EE0D3A20EE54
:100FA0000E0A3BEE41BA24EE021A3AEE41AA24EEB2
:100FB000031A24EE000A39EE419A38EE408A94ED85
:100FC000043A94ED000A94ED011A2BEE035A94EDC5
:100FD000022A30EE050A2AEE035A94ED034A35EE52
:100FE000011A29EE035A35EE022A28EE033A84ED5F
:100FF000000A84ED011A20EE000A21EE011A33EEF8
:10100000043A30EE010A22EE021A30EE010A23EE13
:10101000031A30EE010A84ED022A84ED033A03F04C
:10102000C9FC94ED001A94ED012A94ED023A94ED76
:10103000034A20EE011A20EE022A20EE033A20EEA7
:10104000040A002084ED001A84ED012A84ED023A9E
:1010500084ED030A40B2BDEC108BB0BDB1EE601A56
:10106000B4EE600AF1EE10FAB4EE401AC8BFB0EE6A
:10107000600AF1EE10FAC8BFB0EE410A70470000F6
:1010800000214FF07E524DF20A734CF28F2CC3F6C2
:101090002343C3F6F54CC0E90011C0E90221016108
:1010A0004FF07A5142618361C0F81CC00162704701
:1010B00090ED056A90ED035A66EE011AD0ED042A10
:1010C000D0ED063A31EE855A75EE224A63EE813A4A
:1010D00090ED024A74EEA33A63EE813A34EE234A6D
:1010E000D0ED083A71EEA21A74EE232AC4EE223A29
:1010F000C1EEA22AF6EE004A90ED013A60EE244AD3
:1011000064EE814A90ED002A23EE017A64EE814A72
:1011100034EE877A32EE072A90ED077A20EE010A44
:1011200030EE030A27EE011A30EEC23A36EE011A0B
:1011300023EE236A32EE062A80ED002A23EE222ACD
:1011400030EE020A80ED010A24EE230A34EE400A52
:1011500080ED020A25EE230A35EE400A80ED030AEF
:1011600024EE220A31EEC00A80ED040A25EE220A9E
:1011700031EE400A80ED050A7047000080B541F26B
:10118000B440C2F200000068042106F0C3FA80BD3A
:1011900080B540F23832C2F200020020122113233F
:1011A00000F086F9002080BD80B5012001214FF0BC
:1011B000FF3206F0EFFA80BD9FED010A704700BFD5
:1011C0000000C84380B541F2B440C2F2000000689C
:1011D000082106F09FFA80BD80B540F23830C2F297
:1011E0000000C21D01200221062300F061F9002049
:1011F00080BD000080B5022001214FF0FF3206F0D3
:10120000C9FA80BDF0B581B000284FF0FE0700F0AC
:1012100097800C46002900F0938040F6B006C2F299
:1012200000060546307808B1FD2789E006F010FB7E
:1012300041F2B441C2F20001002808607BD00020D6
:101240007E21B622EC6200F085F901201421B6223D
:1012500000F080F91E2000F0E7FA00201E2100F0C7
:1012600049F90020002100F045F91E2865D1012030
:101270000021012400F03EF90F2860D1022000F087
:101280008DF9032000F08AF941F26142C0F60002B4
:1012900000200121002700F09DFA41F27D11C0F6E7
:1012A0000001022000F0C0F941F2C511C0F60001B2
:1012B000032000F0B9F900204021AA2200F04AF9E9
:1012C00000204121012200F045F90020532108228D
:1012D00000F040F900205821042200F03BF90020E2
:1012E0007D21042200F036F9322000F09DFA012021
:1012F0000F21012200F02EF901201021032200F01D
:1013000029F901201621002200F024F901201821DA
:10131000012200F01FF901201521802200F01AF9A6
:101320000A2000F081FA0220347000F04FF9032007
:1013300000F04CF904E0FE2702E0FC2700E0FC2767
:1013400078B201B0F0BD0000002841D040F2383141
:10135000C2F20001B1F901209FED1F3A00EE102A00
:10136000B8EEC00A80EE030AB1F90330B1F905C046
:1013700001EE103A02EE10CAB8EEC11AB8EEC22A57
:1013800081EE031A82EE032A4FF60003CFF6FF73B5
:1013900080ED040A4A7C897CD20042EA5112002185
:1013A000B1EB922F80ED051A80ED062A18BF1A4383
:1013B00000EE102AB8EEC00AB4EE001A20EE010AC0
:1013C000B3EE071A30EE010A80ED0A0A48B2704700
:1013D000FE2148B2704700BF00A0AA45C0B340F24A
:1013E0003831C2F20001B1F90720B1F90930B1F981
:1013F0000B1000EE102A01EE103A9FED172A03EEB3
:10140000101AB8EEC00AB8EEC11AB8EEC33A80EEB0
:10141000020A81EE021A83EE022A9FED103AC16A97
:1014200091ED014A91ED025A20EE030A21EE031AD2
:1014300022EE032A91ED003A31EE441A30EE430ACF
:1014400032EE452A80ED070A80ED081A80ED092A60
:101450006FF00100704700BF6F12034235FA8E3CF7
:1014600010B5002000F0CAF841F2B444C2F2000402
:1014700038B90020012100F0FDF82068012106F0B4
:1014800049F9012000F0BAF8002818BF10BD01206A
:10149000012100F0EFF82068022106F03BF910BDB1
:1014A00080B50C2001214FF0FF3206F073F980BDAA
:1014B000002A08BF704770B51C4615460E46012825
:1014C00002D8002100F0D6F840F24B3146F08000FF
:1014D000C2F20001087000200122002300F08AF906
:1014E000002029462246012300F05AF9BDE8704049
:1014F0007047000070B5044601200D4600F094F9D5
:10150000012C03D82046002100F0B4F845F08000FB
:1015100040F24B35C2F200052E4606F8010B0020C2
:1015200029460122002300F065F900202946022205
:10153000002300F035F92CB1012C08D140F24B36D4
:10154000C2F200062046012100F094F83078C0B2C3
:1015500070BD000010B5044601F07F0040F24B3131
:10156000C2F20001087001204A7000F05DF9012C00
:1015700003D82046002100F07DF840F24B31C2F242
:10158000000100200222002300F034F9012C88BF62
:1015900010BD2046012100F06DF810BD0238C0B228
:1015A000022882BFFF2040B2704780B541F20A7125
:1015B000C000C0F2090121FA00F040B201F0C4F904
:1015C0000020BDE8804040B2704700000238C0B241
:1015D000022882BFFF2040B2704780B541F20A71F5
:1015E000C000C0F2090121FA00F040B201F0B0F9E8
:1015F0000020BDE8804040B270470000052884BF4D
:101600000020704780B54CF6D831C0F6000101EBE0
:10161000C002526831F83010104600F0C7FF0138A0
:10162000B0FA80F0400980BDB9B1052882BFFF2023
:1016300040B270474CF6D832C0F6000232F830C0E3
:10164000002000232CFA00F2D20709D10E2B03F15F
:10165000010300F10100F5D908E0FE2040B2704717
:1016600040F2A012C2F2000242F82010002040B264
:1016700070470000052882BFFF2040B2704780B548
:101680000A464CF6D831C0F6000101EBC0035B6896
:1016900031F83010184600F08FFF0020BDE8804080
:1016A00040B27047082882BFFF2040B270474CF616
:1016B0000841C0F60001B7EE001A51F83010B4EE40
:1016C000410AF1EE10FAC8BFB0EE410A0A689FED78
:1016D000181AD16AB5EE400A0131F1EE10FAB8BF1E
:1016E000B0EE410A01EE101AB8EE411A20EE010ADE
:1016F000BCEEC00A011F022910EE101A02D802F136
:10170000340010E0072801D0012802D102F138008E
:1017100009E040F2051323FA00F0C0070CBF02F104
:10172000400002F13C000160002040B2704700BF61
:1017300000000000082882BFFF2040B2704780B53B
:101740004CF60841C0F6000101EBC00251F8300030
:10175000918802F051FB0020BDE8804040B2704704
:10176000082882BFFF2040B2704780B54CF6084180
:10177000C0F6000101EBC00251F83000918802F080
:10178000CDFB0020BDE8804040B2704740F2606170
:10179000C2F20001002818BF00210846704700006F
:1017A00070B510B1FF2040B270BD1E4614460D4604
:1017B000FFF7ECFF0028F5D02946224616B101F0CC
:1017C0004FFD02E0142301F091FC002818BF012016
:1017D00040B270BD002A0FBFFE2040F20023C2F2CB
:1017E000000303EB40101CBF40F82120002040B252
:1017F0007047000070B510B1FF2040B270BD1E46AA
:1018000014460D46FFF7C2FF0028F5D029462246B0
:1018100016B102F013F802E0142301F0BBFD00281A
:1018200018BF012040B270BD70B5044605F02CFE13
:101830000546FF2605F00AFE411C05290BD80120AC
:10184000884010F0310F0BD110F0060F0AD020465F
:1018500000F0A6FD11E06FF00041884218BF00269D
:1018600070B270BD4FF47A70B0FBF5F1B4FBF1F0DB
:10187000A14288BF012005F0BFFD002670B270BDF7
:1018800070B5044600F00CF805460E4600F008F866
:10189000401BB141001B71F10000F7D3002070BD67
:1018A0002DE9F04105F0F0FD044608F02BF84FF467
:1018B0007A784EF21806B8FBF4F4CEF200063768D8
:1018C00004FB00F508F01EF860433168854208BF4C
:1018D000394656F8042C01FB08F10132B1FBF2F154
:1018E00000FB08F0401A00F57A700021BDE8F08195
:1018F00040F6200240F2D871C2F200020128C2F282
:10190000000118BF0022002818BF11460846704782
:1019100080B582B001680A68D20614D5002201920F
:101920000A68019249680191019905F00DFB40F2A6
:10193000202100EBC000C2F2000101EB8000006A30
:10194000002818BF804702B080BD00003AB10128CE
:101950004FF0FF0398BF082904D958B27047FE23FF
:1019600058B2704740F2202300EBC000C2F20003DF
:1019700003EB8000002340F8212058B2704700009C
:10198000FEE7000000284FF0FF0318BF002901D137
:1019900058B2704790ED013A9FED774A90ED022AD8
:1019A00033EE044A9FED755A9FED756A34EE044A92
:1019B00090ED031AC4EE050A32EE064A9FED716AF5
:1019C000DFED711A84EE067A31EE214A9FED6F6ADF
:1019D00090ED040A34EE044ADFED6D1A84EE066AD7
:1019E00030EE214A34EE044A84EE055ABFEE004A36
:1019F00070EE841AC1ED021AF0EEE11A81ED037A5D
:101A0000B0EEC77A76EE040A9FED626AC1ED040A71
:101A1000F4EE461A35EE045AF1EE10FAB4EE467AB8
:101A2000B0EEE07A81ED055ADCBF00228A60F1EE6B
:101A300010FAB4EE467AB0EEC55ADCBF0022CA6096
:101A4000F1EE10FAB4EE465ADCBF00220A61F1EE64
:101A500010FADCBF00224A6191ED026AB7EE005A2B
:101A6000B0EEC67AB4EE457AF1EE10FA0ADBB5EEC6
:101A7000406AB0EE446AF1EE10FAC8BFB0EE456AB3
:101A800081ED026A91ED036AB0EEC67AB4EE457A52
:101A9000F1EE10FA0ADBB5EE406AB0EE446AF1EE00
:101AA00010FAC8BFB0EE456A81ED036A91ED046A91
:101AB000B0EEC67AB4EE457AF1EE10FA0ADBB5EE76
:101AC000406AB0EE446AF1EE10FAC8BFB0EE456A63
:101AD00081ED046A91ED056AB0EEC67AB4EE457AFE
:101AE000F1EE10FA08DBB5EE406AF1EE10FAC8BF6D
:101AF000B0EE454A81ED054A90F800C0BCF1000FF8
:101B00000DD0837D012B02D1002048800CE0BCF178
:101B1000000F04D0807D022804D0032802D10120C8
:101B2000C87001E001208870B5EE403AF1EE10FA7D
:101B30004FF00000B5EE402A4FF0000208BF012030
:101B4000F1EE10FA08BF01221040B5EE401A002253
:101B5000F1EE10FA08BF01221040B5EE400A002253
:101B60000023F1EE10FA08BF01221040487081F8FE
:101B700000C058B2704700BF000051C30060AD44C0
:101B8000000032C30020AC44000052C30040AD440A
:101B900000005DC3CDCC4C3DB5EE401AF1EE10FA1D
:101BA00030EE600AD8BF7047B6EE002A21EE022A56
:101BB000B4EE420AF1EE10FAC4BF30EE410A7047AB
:101BC000B1EE422AB4EE420AF1EE10FAB8BF30EE9E
:101BD000010A704740F21400C2F200007047000092
:101BE000B0B5E8B140F6B104C2F20004207810B1FB
:101BF000FD2568B2B0BD05F02BFE41F2B841C2F23E
:101C00000001086060B141F6A162C0F60002002048
:101C100003210025FFF79AFE0120207068B2B0BDB5
:101C2000FE2568B2B0BD00002DE9F04F82B090F8FB
:101C300002C0C27841F2AC334FEADC04C2F20003C6
:101C400062F34A1490F8019005795C80C278467975
:101C5000AD0045EA921206F0010542EA85229A801B
:101C6000457987796E0867F3CA16DE808579C7796A
:101C70004FEA151E67F30A1EA3F808E0077A90F8EA
:101C80000780457A7F0047EAD81705F0030547EA41
:101C9000452BA3F80AB0457A877A4FEA950867F38F
:101CA0008A18A3F80C80C77A857AFF0047EA551591
:101CB000DD8190F80CA0477B009567F30A2AA3F812
:101CC00010A0477B857BFF0865F34A175F82019769
:101CD000C77B6CF30A2990F80EC0057CBF0047EA69
:101CE0009C1705F0010547EA852CA3F814C0057C74
:101CF000477C680800EE104A01EE102A02EE106AD6
:101D0000AEF22D1203EE109A67F3CA10C72AB8EE8E
:101D1000C33AB8EEC00AB8EEC11AB8EEC22AA3F8A8
:101D20000090D88281ED012A81ED021A81ED033AFB
:101D300081ED040A01D201220DE0AEF5FA72B2F58E
:101D40007A7F01D2032206E0AEF2DC520023C82AD9
:101D500038BF01235A00ABF22D13DDE900679BB2B7
:101D6000C72B0A7501D201220FE0ABF5FA7292B2CD
:101D7000B2F57A7F01D2032207E0ABF2DC5292B2D5
:101D80000023C82A38BF01235A00A8F22D13C72BFD
:101D90004A7501D201220DE0A8F5FA72B2F57A7FF8
:101DA00001D2032206E0A8F2DC520023C82A38BF81
:101DB00001235A00A6F22D13C72B8A7501D20222E5
:101DC0000CE0A6F5FA72B2F57A7F01D2032205E0A3
:101DD000A6F2DC530022C82B38BF0122AAF22D1331
:101DE000C72BCA7501D202220CE0AAF5FA72B2F52D
:101DF0007A7F01D2032205E0AAF2DC530022C82B2D
:101E000038BF0122A7F22D13C72B0A7601D2022276
:101E10000CE0A7F5FA72B2F57A7F01D2032205E051
:101E2000A7F2DC530022C82B38BF0122ACF22D13DD
:101E30009BB2C72B4A7601D201220FE0ACF5FA72B1
:101E400092B2B2F57A7F01D2032207E0ACF2DC5203
:101E500092B20023C82A38BF01235A00A0F22D13E2
:101E6000C72B8A7601D202220CE0A0F5FA72B2F5F5
:101E70007A7F01D2032205E0A0F2DC530022C82BB6
:101E800038BF0122B0F59670CA7618BF0120B9F5A7
:101E90007A7218BF01221040087002B0BDE8F08FBE
:101EA00080B541F2B840C2F2000000684FF48011E2
:101EB00005F030FC80BD000010B504460020FFF79F
:101EC00017FD2146192202F0B5FA002818BF4FF07D
:101ED000FF3010BD80B502464FF48010012105F09F
:101EE00059FCA0F58010B0FA80F0400980BD0000D8
:101EF00080B540F2E840C2F2000000F0F1F880BD89
:101F000080B540F2C830C2F2000000F0E9F880BDB0
:101F100080B540F24850C2F2000000F0E1F880BD08
:101F200080B540F22840C2F2000000F0D9F880BD30
:101F300080B540F28840C2F2000000F0D1F880BDC8
:101F400080B540F2A850C2F2000000F0C9F880BD90
:101F5000D0F800C06FF00F024AF6AB2352FA8CF2B1
:101F6000CAF6AA230146A2FB0330000905A31B5CA5
:101F700040F2FF302CEA00005F2A88BF0430C1E93C
:101F80001603704700061016000610168269816A53
:101F9000B2F5005F06D06AB9022912D0012914D027
:101FA000D1B90EE0032917D8DFE801F0020B020FC8
:101FB0000120704703293CBF012070471CBF00204F
:101FC0007047C06AC0F300607047C06AA0F1C0707B
:101FD000B0FA80F0400970470020704780B5D0F813
:101FE00000C0D0F808E0DCF80000BEF1400F20F49B
:101FF0008020CCF800000846CCF8043004BF10461E
:102000000A46CCF80800CCF80C2080BD70470000D0
:1020100080B5082000F0EEF980BD000080B51020EA
:1020200000F0E8F980BD000080B5202000F0E2F962
:1020300080BD000072B600BFFEE7000070B5866D7F
:10204000044600F0BFFA94F83510022925D1054660
:102050002068216C026822F016020260426922F0B8
:102060008002426109B9A16C19B1016821F008012F
:102070000160016821F00101016000BF2068006873
:10208000C0070ED000F09EFA401B0628F6D3202091
:102090006065032084F835000CE080206065012035
:1020A00008E0E06D3F2101FA00F0B060012084F803
:1020B00035000020002184F8341070BD90F83510F0
:1020C000022909D1052180F835100068016821F046
:1020D00001010160002070478021416501207047A7
:1020E000F0B581B004460020009040F20000C2F23A
:1020F00000000268D4E9166048F2B5133768082179
:10210000C1F64E3381403942A2FB03250CD0226830
:1021100013685B0708D5136823F004031360B160EC
:10212000616D41F00101616501218140394208D0B2
:1021300022685269120604D5B160616D41F0020156
:10214000616504218140394208D0226812689207F3
:1021500004D5B160616D41F00401616510218140D9
:10216000394215D020680268120711D5B1600268A3
:102170000168520306D4C90506D4016821F008019C
:10218000016001E0080342D4216C09B12046884770
:10219000E16D202000FA01F23A4244D02068036841
:1021A000DB0640D5B26094F835300268052B1ED1AD
:1021B00022F016020260426922F080024261226C23
:1021C0000AB9A26C1AB1026822F0080202603F202C
:1021D0008840B060012084F83500216D002000297E
:1021E00084F8340040D02046884701B0F0BD016833
:1021F000520310D4C90512D4016821F01001016006
:10220000012084F83500002084F8340007E0A16C38
:102210000029BBD1BCE7080301D4616C00E0E16B8D
:1022200009B120468847606DF0B1606DC00717D0D6
:10223000052084F835002068A90A026822F001020E
:10224000026000BF009A01328A42009202D80268FE
:10225000D207F7D1012084F83500002084F834003B
:10226000E16C09B12046884701B0F0BD2DE9F0418D
:10227000044600F0A7F9C4B10546022084F83500F1
:102280000020216884F83400086820F0010008600C
:1022900026683068C0070BD000F094F9401B052871
:1022A000F6D903212022032042E00120BDE8F0817D
:1022B000306848F23F01CFF21001251D00EA010C01
:1022C0002ECDD4E9050E41EA0C01114319432943EF
:1022D000D4E90778084340EA0E01606A39430428CC
:1022E00041EA080103D1D4E90B23114319433160BA
:1022F0007169042821F0070141EA00050CD1D4E9F5
:102300000A1045EA010538B12046FFF73FFE18B133
:102310000121402201200BE020467561FFF718FEE5
:10232000E16D3F2202FA01F18160002201210020CB
:10233000626584F83510BDE8F0810000B0B5044650
:1023400090F83400012828D0012084F83400A56DCD
:1023500094F8350001281DD1022084F835000020B2
:1023600060652046FFF73AFEE26D3F23206803FADE
:1023700002F2216CAA60026842F01602026019B1F2
:10238000016841F008010160016841F0010101604C
:102390000020B0BD002084F834000220B0BD000051
:1023A000B0B5044600F00EF9054640F23410C2F212
:1023B00000000078611C18BF044400BF00F002F95F
:1023C000401BA042FAD3B0BD70B540F2A01604463F
:1023D0000025C2F2000603E00135102D08BF70BDD4
:1023E00024FA05F0C007F7D056F82500002818BFDA
:1023F0008047F1E780B543F61441C4F201010A6851
:10240000024208BF80BD0860FFF7DEFF80BD00000C
:102410002DE9F04F83B000F13E4202F1FF724FEA26
:10242000B22241F600470192C4F2020708224FF09F
:10243000010E00254FF0000A4FF00008B84208BF17
:10244000072200920AE000BF08F101080AF1040A1D
:10245000B8F1100F05F1020500F0A4800C680EFA27
:1024600008FB14EA0B09EFD04C6804F0030CACF144
:10247000010EBEF1010F11D80322876802FA05F69A
:10248000CA68B743AA403A4382604268C4F300175F
:1024900022EA0B0207FA08F73A434260BCF1030F45
:1024A0001CD0C26803238E6803FA05F7BA4306FA04
:1024B00005F73A43BCF1020FC2600FD16FF003027F
:1024C00002EA580202440AF01C060F23176A03FAB4
:1024D00006F40B69A743B3403B431362026803232E
:1024E0004F68AB409A4307F00303AB401A4317F41D
:1024F000403F4FF0010E0260A6D0002243F6440395
:102500000292C4F202031A6843F6004442F4804285
:102510001A601A68C4F2010402F480420292029A1C
:1025200028F003024FF6084B2244CFF6FF7B52F807
:102530000B300AF00C070F26BE4023EA060C019B65
:10254000009E072B38BF1E4606FA07F747EA0C0322
:1025500042F80B30A2684B6842EA090743F60C4C7C
:10256000DE0258BF22EA0907A760C4F2010CDCF8BA
:1025700000209E0242EA090758BF22EA0907CCF868
:10258000007062689E0342EA090758BF22EA090701
:1025900067602268DB0342EA090358BF22EA0903A5
:1025A000236051E703B0BDE8F08F000000690840E8
:1025B00018BF012070470000002A08BF090481618C
:1025C0007047000047F26C60C2F20000006870477C
:1025D000F0B581B0B0B3044690F83D0028B90020B2
:1025E00084F83C00204600F0BFF8242084F83D0029
:1025F0002068016821F001010160016841F4004197
:102600000160016821F40041016000F06FFA48F2B6
:102610008041C0F21E0140F60012656888424FF00A
:102620000001C0F23D0248F2A16C4FF0000338BF38
:1026300001219042C0F2010C38BF0123654538BF2B
:102640000B4613B1012001B0F0BD4DF68361C4F219
:102650001B31A0FB011221684FEA924E4B684FF4E8
:10266000967623F03F0343EA92434B6044F6D353FC
:102670000F6A0EFB06F6C1F26203A6FB033627F0D3
:102680003F03B709654538BF970C7A1C1A430A62A5
:10269000CA6948F2A0674CF6FF73C0F20107BD4259
:1026A00022EA030C0AD801386A00B0FBF2F00130CC
:1026B0006FF31F30042898BF04202BE0A368A0F11B
:1026C000010E9BB119206843BEFBF0F004220130DB
:1026D00062F31F30000512D09BB119206843BEFB86
:1026E000F0F00422013062F31F3011E005EB4500E9
:1026F000BEFBF0F001306FF31F300005ECD101207C
:1027000008E005EB4500BEFBF0F001306FF31F3031
:1027100040F4004040EA0C00C8610868D4E907238F
:1027200020F0C000104318430860886848F2FF3268
:1027300004F10C0790438CCF18431043A6698860BE
:10274000C86820F0FF0038433043C860086840F094
:102750000100086000202021206484F83D102063DF
:1027600084F83E0001B0F0BD2DE9F04F87B004467B
:1027700045F600470068C4F200070026B8420696F6
:10278000CDE904660396029602D007B0BDE8F08F4B
:1027900043F630050196C4F2020528680DF10808D9
:1027A00040F00400286028684FF0120900F004008F
:1027B00001900198019628684FF0030A40F001004B
:1027C000286028684FF0040B00F001000190019888
:1027D0004FF40070029007F5D6304146CDE90396DC
:1027E000CDF814A0CDF818B0FFF712FE4FF48070AA
:1027F000CDE9020904A880E8400C07F5D230414633
:10280000FFF706FE019628694FF0C06140F4000012
:102810002861286940F2C83500F400000190019851
:1028200046F24000C2F20005C4F202004FF480629A
:1028300085E843002846C5E90362C5E90566C5E9A0
:1028400007666E62FFF712FD002818BFFFF7F2FB64
:10285000A563AC6307B0BDE8F08F000040F2341010
:1028600047F26C61C2F20000C2F2000100780A680F
:10287000104408607047000080B543F60040C4F281
:102880000200016841F400710160016841F4806157
:102890000160016841F480710160032000F06CF870
:1028A0000F2000F005F800F02BF8002080BD00009C
:1028B000B0B540F23412C2F2000240F200011278C8
:1028C000C2F200014FF47A730968B3FBF2F20446D6
:1028D000B1FBF2F1084601F05DF80F2C4FF0010555
:1028E0000CD858B94FF0FF3021460022002500F0E7
:1028F00033F840F23810C2F2000004602846B0BD40
:1029000080B582B0002043F640010190C4F202017C
:102910004A6842F480424A604A6802F48042019266
:10292000019A00900868002240F080500860086812
:102930000F2100F08050009000986FF0010000F02F
:102940000BF802B080BD000080B504F085FC80BDAE
:1029500080B504F095FC80BD70B514460D46064662
:1029600004F09EFC2946224602F05CFC01463046FB
:1029700004F09EFC70BD000080B504F0B3FC80BD87
:102980002DE9F041002800F08B8043F60808C4F2DE
:1029900002080446D8F8F8030D4600F00700884204
:1029A00007D288F8F853D8F8F80300F00700A842D7
:1029B00076D12068810717D5410705D5D8F80010D2
:1029C00041F4E051C8F80010010705D5D8F800100F
:1029D00041F46041C8F80010D8F80010A26821F056
:1029E000F0011143C8F80010C0073FD1D8F8F80330
:1029F00000F00700A84207D988F8F853D8F8F80380
:102A000000F00700A8424BD12068410707D5D8F84D
:102A10000010E26821F4E0511143C8F800100007EB
:102A200008D5D8F80000216920F4604040EAC100D0
:102A3000C8F8000000F07EF8D8F800104CF6C0325C
:102A4000C1F30311C0F60002515C40F2000220FA0B
:102A500001F140F23810C2F200000068C2F2000238
:102A60001160FFF725FF0020BDE8F0816068811E3E
:102A7000022907D258F8081C89015CBF0120BDE873
:102A8000F08110E0012807D158F8081C89035CBFC9
:102A90000120BDE8F08106E058F8081C890702D43F
:102AA0000120BDE8F081D8F8001021F003010843AF
:102AB000C8F80000FFF786FD064641F2883700BFE0
:102AC000D8F80000616800F00C00B0EB810F8DD0E9
:102AD000FFF778FD801BB842F2D90320BDE8F081F2
:102AE00040F20000C2F200000068704780B5FFF7B6
:102AF000F7FF43F60801C4F2020109684CF6D03230
:102B0000C1F38221C0F60002515CC84080BD0000C4
:102B100080B5FFF7E5FF43F60801C4F2020109683A
:102B20004CF6D032C1F34231C0F60002515CC840CD
:102B300080BD000010B543F60404C4F202046068CE
:102B400000F00C0008280AD0042819BF42F2004007
:102B5000C0F2F40041F60030C0F2B70010BD2068AA
:102B600021682368490241F60031C0F2B70100F044
:102B70003F02C3F388105CBF42F20041C0F2F4018F
:102B8000A1FB00010023FDF78FFB21680222C1F3A6
:102B9000014102EB4101B0FBF1F010BD2DE9F04124
:102BA00082B0002800F0A2800446007843F60006B8
:102BB000C007C4F2020643D0B06800F00C0004283D
:102BC00005D1306880033BD56068C8BB8EE0B06833
:102BD00000F00C00082802D170684002F1D465684A
:102BE000B5F5A02F0AD0B5F5803F0BD0306820F4A2
:102BF00080303060306820F4802006E0306840F497
:102C000080203060306840F480303060FFF7DAFCBC
:102C1000002D054611D000BF3068800310D4FFF7A7
:102C2000D1FC401B6428F7D922E100BFFFF7CAFCA2
:102C3000401B64284FF0030055D830688003F5D45A
:102C4000207880071AD5B06810F00C0F09D0B06852
:102C500000F00C00082840F08A807068400200F103
:102C600086803068800702D5E06801283ED1306850
:102C7000216920F0F80040EAC100306020780007A8
:102C800038D4207840074CD4A5695DB3B06800F013
:102C90000C00082840F09E80012D27D07068E16963
:102CA00000F480028A4221D1216A00F03F028A4268
:102CB0001CD147F6C071626A0140B1EB821F15D189
:102CC000A26A0023CFF6FF7303EBC23200F4403157
:102CD0006FF30F02914209D1E16A00F07060B0EB2E
:102CE000016F03D1002002B0BDE8F081012002B0E5
:102CF000BDE8F0816069002840F20000C4F247207E
:102D000057D00121C0F8801EFFF75CFC054600BFCC
:102D1000706F8007B5D4FFF755FC401B0228F7D928
:102D2000A6E0306C10F080580AD100200190306C81
:102D300040F080503064306C00F080500190019879
:102D400047F20007C4F200073868C00524D4386889
:102D500040F480703860FFF735FC05463868C005E0
:102D60001AD4FFF72FFC401B0228F7D980E0E06857
:102D7000002851D00020C4F2472001210160FFF754
:102D800021FC0546306880073FF571AFFFF71AFC5C
:102D9000401B0228F6D96BE0A568052D50D0012D07
:102DA00052D0306F20F001003067306F20F0040007
:102DB0004DE00021C0F8801EFFF704FC054600BF6F
:102DC000706F80077FF55DAFFFF7FCFB401B0228AB
:102DD000F6D94DE00027C4F2472700203866FFF7F8
:102DE000F1FB022D05460BD13068800158D5FFF765
:102DF000E9FB401B02284FF00300F5D973E700BF41
:102E0000306880017FF56EAFFFF7DCFB401B0228C6
:102E10004FF00300F4D966E70020C4F247200021F8
:102E20000160FFF7CFFB0546306880077FF526AFCE
:102E3000FFF7C8FB401B02284FF00300F4D952E70C
:102E4000306F40F004003067306F40F001003067B1
:102E5000FFF7B8FB002D054641F2883714D000BFBC
:102E6000306F800713D4FFF7ADFB401BB842F7D992
:102E7000032002B0BDE8F081FFF7A4FB401BB8427D
:102E80004FF003003FF62FAF306F8007F4D4B8F156
:102E9000000F7FF4F9AE306C20F080503064F3E620
:102EA00004F11C052FCD08430021CFF6FF7140EA45
:102EB000821001EBC3316FF30F0140EA0560084354
:102EC000706001203866FFF77DFB044630688001A2
:102ED0003FF508AFFFF776FB001B02284FF0030019
:102EE000F4D900E780B503F003F9022808BF80BDDC
:102EF00040F20021C2F2000101EB4010806900287D
:102F000018BF804780BD000070B538B10446406AE4
:102F100030B10020206104F1140007E0012070BDF1
:102F20006068B0F5827F03D004F11C0000210160CD
:102F30000026A66294F8510020B9204684F850601B
:102F400000F03CF8022084F8510094E80F0001F4EE
:102F50008271056802F4044225F0400505601144C1
:102F600003F400622369114403F00202636911440F
:102F700003F00102A369E569114403F400721144EE
:102F800005F03802256A114405F08002A56A114354
:102F900005F4005211430160626A042101EA134101
:102FA00002F0100211444160C16921F40061C16165
:102FB0000120666584F85100304670BD2DE9F04F60
:102FC00087B0044643F200070068C4F201070026F8
:102FD000B8420696CDE904660396029602D007B081
:102FE000BDE8F08F43F630000196C4F2020041695B
:102FF00002AD41F48051416141694FF0020901F491
:10300000805101910199019601684FF0010A41F048
:103010000201016001684FF0030B01F00201019110
:103020000199019601684FF0050841F00101016026
:103030000068294600F001000190019818200290D4
:1030400007F55440CDF80C90CDF810A0CDF814B091
:10305000CDF81880FFF7DCF9802002A981E8010E85
:10306000CDF8188046F2404807F550402946C4F292
:103070000208FFF7CDF940F22845C2F200054FF0F3
:10308000C0674FF480692846C5E90087C5E9026634
:10309000C5E90496C5E90666C5E90866FFF7E6F8DE
:1030A000002818BFFEF7C6FFE564AC6340F2884510
:1030B00008F11800C2F200054021C5E9000705F13A
:1030C0000800002280E806022846C5E90522C5E975
:1030D00007226A62FFF7CAF8002818BFFEF7AAFFA6
:1030E000A564AC6307B0BDE8F08F00002DE9F041A6
:1030F00082B0044690F85100012815D10E460029EF
:103100004FF0010060D01746002A5DD060681D4670
:10311000B0F5827F02D1A068002858D0FFF752FA9C
:1031200094F85010012903D1022002B0BDE8F081CB
:103130008046012084F85000042084F851000020CB
:103140006065A663A787E7872063A086E086A168FD
:103150002064B1F5004F606408D12068016821F057
:1031600040010160016821F480410160206801682C
:10317000490603D4016841F040010160E168E08F35
:1031800091B3002855D06E1C0BE000BFC068A16B46
:1031900021F8020BA163E08F0138E087E08F00285F
:1031A00047D020688168C907F0D1FFF70BFA002EDD
:1031B000F4D0A0EB0800A842F0D3012084F851001D
:1031C000002084F85000032002B0BDE8F081042004
:1031D00084F851002046314632463B46009500F0C7
:1031E0009FF902B0BDE8F08118B36E1C0BE000BF80
:1031F000007BA16B0870A06B0130A063E08F0138E9
:10320000E087E08FA8B120688168C907F0D1FFF797
:10321000D9F9002EF5D0A0EB0800A842F1D3012087
:1032200084F85100002084F85000032002B0BDE86B
:10323000F08120462946424602F0CCFE00281CBF01
:1032400020206065012084F85100002084F850009F
:10325000606D002818BF012002B0BDE8F0810000B9
:1032600010B5044690F8510001281CBF022010BD83
:1032700013460A4600294FF0010018BF002B00D169
:1032800010BDA06858B96168B1F5827F07D10420EC
:1032900084F851002046114600F03EFA10BD94F823
:1032A0005010012904BF022010BD012184F85010E4
:1032B000042184F851100021B0F5004F6165A2632C
:1032C000A387E387C4E91011A186E18608D12068AD
:1032D000036823F040030360036823F48043036022
:1032E000E06C45F67D6E45F6A163C0F6000EC0F6B3
:1032F0000003C0E90F3E45F65963C0F60003D4F859
:1033000000C0C0E91331E38F0CF10C01FFF716F890
:1033100040B1606D40F010006065002084F85000FE
:10332000012010BD21680868400603D4086840F0F9
:1033300040000860002084F850004A6842F02002F3
:103340004A604A6842F001024A6010BD80B502F04E
:10335000CFFE022808BF80BD40F20021C2F200016A
:1033600001EB40104068002818BF804780BD000076
:1033700080B502F0BDFE022808BF80BD40F20021EA
:10338000C2F2000101EB40100069002818BF80471D
:1033900080BD00002DE9F04182B01D4616460F4663
:1033A0000446FFF70FF994F8511001290DD180461A
:1033B000002F4FF0010018BF002E02D102B0BDE86F
:1033C000F08194F85000012803D1022002B0BDE83A
:1033D000F081012084F85000032084F8510000207F
:1033E00060652763A686E686A063A087E087A1685C
:1033F000C4E91000B1F5004F08D12068016821F040
:1034000040010160016841F4804101602068016869
:10341000490603D4016841F0400101606168731EF0
:10342000E268B1FA81F1B3FA83F349095B09B2F5B5
:10343000006F41EA030124D139B1216B0988C160D1
:10344000B81C2063E08E0138E086E08E002846D06C
:103450006E1C09E0216B31F8022BC2602163E08E03
:103460000138E086E08ED0B3206881688907F1D406
:10347000FFF7A8F8002EF5D0A0EB0800A842F1D382
:1034800023E039B139780173206B01302063E08E7D
:103490000138E086E08E10B36E1C0AE0216B0978DB
:1034A0000173206B01302063E08E0138E086E08EEE
:1034B000A8B1206881688907F0D4FFF783F8002E4F
:1034C000F5D0A0EB0800A842F1D3012084F8510008
:1034D000002084F85000032002B0BDE8F0812046AF
:1034E0002946424602F0BEFD00281CBF2020606530
:1034F000A06838B9002001902068C16801918068F7
:1035000001900198012084F85100002084F85000B7
:10351000606D002818BF012002B0BDE8F0810000F6
:103520002DE9F04381B01E4615460F460446FFF7CD
:1035300049F894F851108146012909D06068B0F526
:10354000827F14D104294FF0020007D1A16829B964
:10355000002F4FF0010018BF002D02D101B0BDE8CF
:10356000F083002EFAD094F85000012803D10220F5
:1035700001B0BDE8F083012084F8500094F85100B8
:10358000002104281CBF052084F851006165A56353
:10359000E687A6872763E6862068A686216461649D
:1035A0000168490603D4016841F040010160616887
:1035B000731EE268B1FA81F1B3FA83F3DDF820807B
:1035C00049095B09B2F5006F41EA030139D139B10C
:1035D000216B0988C160B81C2063E08E0138E08649
:1035E000012608F1010500BFE08E10B9E08F002828
:1035F0006CD02068816889070CD5E18E012E09D135
:1036000041B1216B002631F8022BC2602163E18EAB
:103610000139E1868168C9070AD0E18F41B1C068EC
:10362000A16B012621F8020BA163E08F0138E0872E
:10363000FEF7C8FF002DD7D0A0EB09004045D3D33B
:103640003AE039B139780173206B01302063E08EA4
:103650000138E086012608F1010500BFE08E08B9B7
:10366000E08F98B32068816889070DD5E18E012E1F
:103670000AD149B1216B002609780173206B013012
:103680002063E08E0138E08620688168C9070BD08E
:10369000E18F49B1C068A16B01260870A06B0130B1
:1036A000A063E08F0138E087FEF78CFF002DD5D0B6
:1036B000A0EB09004045D1D3012084F8510000203F
:1036C00084F85000032001B0BDE8F0832046414655
:1036D0004A4602F0C7FC40B120206065002084F813
:1036E0005000012001B0BDE8F083A06838B9002087
:1036F00000902068C16800918068009000980120C7
:1037000084F85100002084F85000606D002818BF34
:10371000012001B0BDE8F08370B5044690F8510077
:10372000012806D100294FF0010018BF002A0CD152
:1037300070BD6568B5F5827F0ED104284FF0020098
:10374000F6D1A568002DEDD0F2E7002B08BF70BDC3
:1037500094F85000012801D1022070BD012084F8A6
:10376000500094F85100002604281CBF052084F85E
:10377000510066652163A386E386A263A387E3877E
:10378000C4E9106694F8510045F67D6145F69563ED
:10379000C0F60001C0F60003042808BF0B4645F63A
:1037A000A16045F67971C0F60000C0F6000108BFBF
:1037B0000146E06C2568C0E90F1345F65961C0F673
:1037C0000001C0E91316E38F05F10C01FEF7B6FD09
:1037D00038B1606D40F010006065012084F85060E1
:1037E00070BD2268216BA06C536843F001035360E5
:1037F000C0E90F66C0E91366E38E0C32FEF79EFD4A
:1038000040B1606D40F010006065002084F8500009
:10381000012070BD21680868400603D4086840F0A4
:1038200040000860002084F850004A6842F02002FE
:103830004A604A6842F002024A6070BD10B5044610
:1038400090F8510001280AD100294FF0010018BF5B
:10385000002A00D110BD94F85000012801D10220A7
:1038600010BD012084F850000320002384F851008B
:1038700063652163A286E286A363C4E91033A3874C
:10388000E387A068B0F5004F08D12068026822F0F5
:1038900040020260026842F480420260A06C45F679
:1038A000896C45F60972C0F6000CC0F60002C0E94A
:1038B0000F2C45F65962C0F60002D4F800E0C0E9CA
:1038C0001323E38E0EF10C02FEF738FD40B1606D5C
:1038D00040F010006065002084F85000012010BD09
:1038E00021680868400603D4086840F0400008607A
:1038F000002084F850004A6842F020024A604A687A
:1039000042F002024A6010BD80B502F0F1FB0228CD
:1039100008BF80BD40F200214001C2F200010858FA
:10392000002818BF804780BD80B502F0E1FB022867
:1039300008BF80BD40F20021C2F2000101EB40103F
:10394000C068002818BF804780BD000080B502F025
:10395000CFFB022808BF80BD40F20021C2F2000167
:1039600001EB40108068002818BF804780BD000030
:1039700080B502F0BDFB022808BF80BD40F20021E7
:10398000C2F2000101EB40104069002818BF8047D7
:1039900080BD000080B502F04FFD80BDB0B590F84D
:1039A0003C20012A04BF0220B0BD01F108053CCD36
:1039B000D1E900CE23F47C5322F470521A432EF442
:1039C000F0431A432CF4E0431A4324F4C0431A434F
:1039D0002A43C96922F480420368114359640021D3
:1039E00080F83C100846B0BD10B590F83C20012A84
:1039F0004FF0020252D0012380F83C3080F83D2085
:103A00000268D2F804E0D2F808C00C682EF0700307
:103A1000234341F2FF74C4F20004A24253600DDC60
:103A200040F2FF73C4F200039A4215DCB2F1804FFA
:103A300029D040F20043C4F2000322E040F2FF33F9
:103A4000C4F201039A4212DC41F60003C4F20003FF
:103A50009A4218D0002312E040F60003C4F200039B
:103A60009A4210D040F60043C4F2000309E044F249
:103A70000003C4F201039A4205D040F20043C4F2AD
:103A800001039A4204D149682CF0800319439160E4
:103A90000121002280F83D1080F83C20104610BD26
:103AA000002804BF0120704710B5044690F83D007F
:103AB00028B9002084F83C00204600F01FF80220BE
:103AC00084F83D002068211D02F034FD012084F8B7
:103AD000460084F83E0084F83F0084F8400084F8F3
:103AE000410084F8420084F8430084F8440084F8DC
:103AF000450084F83D00002010BD000081B0006842
:103B000044F20041C4F20101884201D001B0704783
:103B10000020009043F64400C4F20200016841F422
:103B200000310160006800F400300090009801B09E
:103B30007047000080B586B000684FF6FF71C4F290
:103B4000000188424FF000010591CDE90311CDE954
:103B5000011129DC40F60001C4F2000188424AD07C
:103B600040F60041C4F20001884240F082804FF0EC
:103B7000000C43F63000CDF800C0C4F20200026829
:103B8000002342F0800202600068022200F0800000
:103B9000009000984FF4E050019040F60040C4F2CD
:103BA000020000F580505CE044F20041C4F20101E3
:103BB00088423BD00021C4F20101884259D14FF024
:103BC000000C43F63000CDF800C0C4F202000268D9
:103BD00042F0100202600068012200F01000009024
:103BE00000984FF4D440019040F60040C4F2020027
:103BF00000F5806034E04FF0000C43F63000CDF863
:103C000000C0C4F202000268002342F00802026011
:103C10000068022200F00800009000984FF48040F5
:103C2000019040F60040C4F202001AE0002000902B
:103C300043F63000C4F202000168032241F0200183
:103C4000016000684FF0020C00F020000090009826
:103C50004020019040F60040C4F2020000F50060F0
:103C600002230221CDE9021C01A9CDE90432FEF7AD
:103C7000CFFB06B080BD0000B0B5044690F83C0014
:103C8000012804BF0220B0BD0D464FEAB201012059
:103C9000032984F83C0037D8DFE801F0020A122239
:103CA0002068294602F0EEFC206850F8181F0EE04C
:103CB0002068294602F018FD206850F8181F16E009
:103CC0002068294602F046FD206850F81C1F41F08C
:103CD00008010160016821F00401016029690FE019
:103CE0002068294602F06AFD206850F81C1F41F444
:103CF00000610160016821F48061016029690902A5
:103D00000268114301600020002184F83C10B0BD1E
:103D1000002804BF0120704710B5044690F83D000C
:103D200028B9002084F83C00204600F01FF802204B
:103D300084F83D002068211D02F0FCFB012084F87E
:103D4000460084F83E0084F83F0084F8400084F880
:103D5000410084F8420084F8430084F8440084F869
:103D6000450084F83D00002010BD000083B00068CD
:103D700040F60001C4F2000188421BD040F6004129
:103D8000C4F20001884226D00021C4F20101884219
:103D900030D10020029043F64000C4F20200416896
:103DA00041F001014160406800F00100029002987A
:103DB00003B070470020019043F64000C4F20200B7
:103DC000016841F004010160006800F00400019006
:103DD000019803B070470020009043F64000C4F201
:103DE0000200016841F008010160006800F008006D
:103DF0000090009803B0704710B5044641B10829FF
:103E000009D0042914BF04F1410004F13F0004E08B
:103E100004F13E0001E004F14000007801281CBFDD
:103E2000012010BD022041B1082909D0042914BF86
:103E300084F8410084F83F0004E084F83E0001E08B
:103E400084F840002068012202F00AFC206841F258
:103E5000FF71C4F2000188420FDC40F2FF71C4F22E
:103E60000001884217DCB0F1804F49D040F2004198
:103E7000C4F20001884243D049E040F2FF32C4F26C
:103E80000102904214DC41F60003C4F200039842A0
:103E900036D0002314E040F60001C4F2000188424D
:103EA0002ED040F60041C4F20001884228D02EE016
:103EB00044F20003C4F20103984221D040F20043CF
:103EC000C4F20103984222D1436C884243F4004378
:103ED0004364C2DD904207DC41F60001C4F20001F8
:103EE00088420DD0002107E044F20001C4F2010134
:103EF000884205D040F20041C4F20101884206D157
:103F0000816801F00701062904BF002010BD016887
:103F100041F001010160002010BD0000B0B5044671
:103F2000006800220D4602F09BFB206840F2004230
:103F300040F48061C4F2010291420DD1016A41F264
:103F40001112114208D1016A40F24442114203D1D8
:103F5000416C21F400414164016A41F211121142A5
:103F600008D1016A40F24442114203D1016821F0B4
:103F7000010101600120082D09D0042D0BD0002D76
:103F800014BF84F8410084F83E000020B0BD84F8DE
:103F900040000020B0BD84F83F000020B0BD00000C
:103FA0007047000080B502F0CFFF032808BF80BD36
:103FB00040F2202100EBC000C2F2000101EB8000C2
:103FC0000069002818BF804780BD0000B0B582B0EE
:103FD000036804461868D9685A6900F02F05202D37
:103FE00001F0200505D125B1204602F0BDFF02B049
:103FF000B0BD5FEA007C1EBF02F0010E01F49072BA
:1040000012EB0E024AD1226B0840C1063DD5012AAF
:104010003BD10020019018680190586801900198E8
:104020005869400642D4A08DE18DE28D002A1CBF64
:10403000401A5FEA004101D102B0B0BD216851E8E9
:10404000031F226821F4907142E80313002BF5D17D
:10405000216851E8051F226821F0010142E805139B
:10406000002BF5D1202184F842100021216300BFEC
:10407000216851E8031F226821F0100142E8031370
:10408000002BF5D10221616354E0010654D44006AF
:10409000D2D5204602F03EFF02B0B0BDC20718BF25
:1040A00011F480725DD1420761D467E0E06B016872
:1040B00049688AB2002A44D0A38D9A4241D2E18550
:1040C000C069B0F5807F30D0206850E8030F2168C8
:1040D00020F4807041E80302002AF5D1206850E8FE
:1040E000050F216820F0010041E80502002AF5D102
:1040F000206850E8050F216820F0400041E80502E3
:10410000002AF5D1202084F842000020206300BF5F
:10411000206850E8030F216820F0100041E80302F6
:10412000002AF5D1E06BFDF789FF02206063A08DC6
:10413000E18D401A81B20FE0204603F03DF802B055
:10414000B0BDA18D91427FF477AFC069B0F5807F9B
:104150007FF472AF022060632046FFF721FF02B0B8
:10416000B0BD626C42F001026264420706D5BEF146
:10417000000F03D0626C42F002026264820706D52F
:10418000BEF1000F03D0626C42F004026264BCF125
:10419000000F06D55EEA050203D0626C42F0080209
:1041A0006264626C002A3FF447AF0840800602D583
:1041B000204602F0D9FE20684069616C00F04000A2
:1041C00001F00801401827D0204602F07BFE20684D
:1041D000406940061BD500BF206850E8050F2168E4
:1041E00020F0400041E80502002AF5D1E06B70B1F3
:1041F00046F6C551C0F600010165FDF75FFF0028D6
:104200003FF41AAFE06B016D884702B0B0BD2046A5
:10421000FFF7C8FE02B0B0BD2046FFF7C3FE002086
:10422000606402B0B0BD0000002804BF01207047E8
:1042300010B5044690F8410028B9002084F84000E9
:10424000204600F021F8242084F841002068C1684D
:1042500021F40051C160204602F0EAFE20680169A5
:1042600021F490410161416921F02A014161C16855
:1042700041F40051C16000202021606484F84110A5
:1042800084F84210606310BD2DE9F04387B0044606
:10429000006841F20041C4F2010100268842CDE9E4
:1042A0000566CDE90366029651D044F60001C4F2DA
:1042B0000001884240F0BB80002643F630000196A2
:1042C000C4F20200016941F480210161016901F435
:1042D0008021019101990196016841F0040101607A
:1042E000006802A900F00400019001984FF44060BA
:1042F00002900220CDE903060320059007200690D6
:1043000040F60000C4F20200FEF782F840F2E845F1
:1043100046F22800C2F20005C4F202004FF000612C
:104320004FF4806285E843002846C5E90362C5E989
:104330000566C5E907666E62FDF798FF002818BF9D
:10434000FDF778FEE563AC6307B0BDE8F08343F6A4
:1043500030000196C4F20200416946F2280841F09B
:10436000200141614169C4F2020801F0200101917C
:1043700001990196016841F040010160006802A9BD
:1043800000F04000019001984FF484400290022018
:10439000CDE90306032005900820069040F60000B2
:1043A000C4F2020000F58050FEF732F840F24855A2
:1043B00008F58060C2F200054FF020674FF4806975
:1043C000C5E900072846C5E90266C5E90496C5E9BE
:1043D0000666C5E90866FDF749FF002818BFFDF726
:1043E00029FEE563AC6340F2A85508F58F60C2F280
:1043F00000054021C5E9000705F10800002280E81A
:1044000006022846C5E90522C5E907226A62FDF7CA
:104410002DFF002818BFFDF70DFE472005210022C3
:10442000A563AC63FEF798FA4720FEF791FA07B050
:10443000BDE8F08380B590F84230202B1CBF0220ED
:1044400080BD00294FF0010318BF002A01D1184692
:1044500080BD0023036302F059FE0346184680BD69
:1044600080B502F071FD032808BF80BD40F2202115
:1044700000EBC000C2F2000101EB8000C068002820
:1044800018BF804780BD000080B502F05DFD0328A5
:1044900008BF80BD40F2202100EBC000C2F2000145
:1044A00001EB80008068002818BF804780BD0000B5
:1044B00080B502F049FD032808BF80BD40F22021ED
:1044C00000EBC000C2F2000101EB80004068002850
:1044D00018BF804780BD0000FEE70000F0B581B046
:1044E0002DED028B0C46054600F0CAF8FDF7D8F911
:1044F00008F04DF99FED238A00EE100A80EE080ABD
:1045000010EE100A08F010FA40F2F012C2F20002A7
:10451000C2E90001FDF7C4F940F2E816C2F2000654
:10452000D6E90023801A994108F031F900EE100A0B
:1045300080EE080A40F2E017C2F2000787ED000A99
:10454000FDF7AEF940F29022C2F2000292ED000AAD
:1045500041F2DC32C2F20002C6E9000140F2B426A8
:10456000D2ED000A97ED001AC2F200063046FCF7C1
:104570009FFD30682860716800202160BDEC028BCF
:1045800001B0F0BD00247449F0B581B02DED028B6F
:1045900084B0B0EE408A01F067FE6420FDF744F974
:1045A00040F29420C2F20000F2EE040AB0EE480A93
:1045B00000F078FA41F2E030C2F20000F1EE040AB5
:1045C000B0EE480A00F06EFA40F2B420C2F20000E9
:1045D000FCF756FD40F6B806C2F2000630886328A4
:1045E0001AD841F2B04440F6C80540F6B407C2F20A
:1045F0000004C2F20005C2F2000700BF20462946AF
:1046000001F066FE286801F0EFFD31883860481C33
:1046100081B264293080F1D39FED178A41F2304591
:104620000020C2F2000501AC30800390CDE901000A
:10463000A86921460022002302F090FF30889DEDFA
:10464000030A01303080142038EE008A02F0D4FED4
:1046500030886428ECD39FED090A40F2B83188EE27
:10466000000AC2F20001002081ED000A04B0BDEC96
:10467000028B01B0F0BD00BF000000000000C84286
:1046800010B52DED0E8B40F6C80441F2B040C2F2D9
:104690000004C2F200002146B0EE438AB0EE629AF6
:1046A000B0EE42AAB0EE61BAB0EE41CAB0EE60DA46
:1046B000B0EE40EA01F00CFE206801F095FD40F6F6
:1046C000B401C2F2000109689FED291A411A00EEF7
:1046D000101AB8EEC00A80EE010A40F20861C2F278
:1046E0000001086041F2DC30C2F2000080ED000AF7
:1046F00041F2E030C2F2000000F096F941F20040D1
:10470000C2F2000080ED000AB0EE4E0AF0EE4D0A53
:10471000B0EE4C1AF0EE4B1AB0EE4A2AF0EE492AEF
:10472000B0EE483A03F07CFE40F2682440F2942058
:10473000C2F20004C2F2000084ED000A00F074F935
:1047400040F2B830C2F2000090ED001A9FED092A45
:1047500084ED000A30EE410A40F2902120EE020A78
:10476000C2F20001002081ED000ABDEC0E8B10BDED
:1047700000007A440AE81C4110B541F20044C4F23A
:104780000204204602210022FDF716FF01F052FB31
:10479000204601210022FDF70FFF0220FDF770F8EF
:1047A000204602210122FDF707FF0220FDF768F8ED
:1047B000204602210022FDF7FFFE204601210122B2
:1047C000FDF7FAFE10BD000010B541F20044C4F23E
:1047D0000204204602210022FDF7EEFE01F02AFB32
:1047E000204601210122FDF7E7FE0420FDF748F8ED
:1047F000204602210122FDF7DFFE0420FDF740F8EC
:10480000204602210022FDF7D7FE20460121012289
:10481000FDF7D2FE10BD0000F0B581B041F20045B9
:104820000446C4F2020501F0F3FA0026002700BF97
:10483000284602210022FDF7BFFE0220FDF720F8E6
:10484000284602210122FDF7B7FE28460121FDF787
:10485000ADFE002818BF012040EA46060120FDF702
:104860000FF8072F07F10107E2D314B1FFF784FF18
:1048700001E0FFF7A9FFF0B201B0F0BD70B541F261
:1048800000450446C4F2020501F0D4FA284602218C
:1048900000220026FDF790FEE0B2C2092846012161
:1048A000FDF78AFE02206400FCF7EAFF2846022199
:1048B0000122FDF781FE0220FCF7E2FF28460221DB
:1048C0000022FDF779FE0220FCF7DAFF072E06F141
:1048D0000106E1D370BD000010B501F0ABFA41F262
:1048E0000044C4F20204204601210122FDF764FEC7
:1048F000204602210122FDF75FFE0420FCF7C0FFE5
:10490000204601210022FDF757FE0420FCF7B8FFE6
:10491000204602210022FDF74FFE10BD10B501F028
:1049200089FA41F20044C4F2020420460221012225
:10493000FDF742FE204601210022FDF73DFE042046
:10494000FCF79EFF204601210122FDF735FE0420E1
:10495000FCF796FF10BD0000B0B541F20044C4F270
:10496000020401F055FA204601210122FDF724FE40
:104970000120FCF785FF204602210122FDF71CFEE5
:104980000120FCF77DFF002520460121FDF70EFEEA
:1049900038B1642D05F10105F6D3FFF7BFFF012003
:1049A000B0BD2046022100220024FDF705FE20466E
:1049B000B0BD000045F6DF1110EE100AC5F63771E4
:1049C000B6EE001AA1EB600020EE011A00EE100A0C
:1049D00021EE002A22EE002AB7EE083A33EE422AF0
:1049E00022EE000A21EE001A20EE011A33EE411ADF
:1049F00020EE010A7047000041F26F2C49F6A63202
:104A00004CF28F23C3F6832CC3F64432C3F6F5432E
:104A10000021C0E900C2C0E90231C0E90411C0E9C7
:104A2000061101627047000010B52DED088B88B3A8
:104A3000B0EE408A90ED010A90ED069A90ED021AD0
:104A400090ED07AA29EE000A38EE400A2AEE011A74
:104A500030EE41BA04461BEE100A02F0F5FB0028C6
:104A600008BFB0EE4B8A94ED030A94ED041A94ED5E
:104A7000052A20EE080A29EE011A30EE010A2AEE74
:104A8000021A30EE010A84ED068A84ED079ABDEC25
:104A9000088B10BD9FED020ABDEC088B10BD00BF56
:104AA00000000000002808BF704710B5F5EE400A6E
:104AB0000446C0ED000A0020F1EE10FAA061E061AA
:104AC0002EDD80EE200A9FED1E1A81EE000A06F010
:104AD00023FD9FED1C1AB7EE002A20EE011A31EEDD
:104AE000023A20EE000ABFEE005A30EE033A30EEF2
:104AF000055A32EE411A80EE034A35EE055A30EE81
:104B0000010A85EE035A80EE030A34EE041A84ED9E
:104B1000034A84ED041A84ED054A84ED015A07E046
:104B20004FF07E519FED050AC4E90310606160609B
:104B300084ED020ABDE81040704700BF000000008D
:104B4000DB0F4940F304B53F10B52DED048B10B3D6
:104B5000B0EE408A90ED030A90ED041A90ED052A1C
:104B600030EE010A30EE020A88EE009A044619EE91
:104B7000100A02F059FB00282046B0EE480A08BF90
:104B8000B0EE489A84ED069A84ED079AFFF74CFF41
:104B9000BDEC048B10BD9FED020ABDEC048B10BD73
:104BA0000000000080B582B0002043F63001019083
:104BB000C4F202010A6842F400120A600A6802F4B0
:104BC00000120192019A00900868002240F48000CF
:104BD00008600868052100F48000009000980C200F
:104BE000FDF7BAFE0C20FDF7B3FE0D2005210022D3
:104BF000FDF7B2FE0D20FDF7ABFE392005210022A6
:104C0000FDF7AAFE3920FDF7A3FE3A200521002278
:104C1000FDF7A2FE3A20FDF79BFE3B200521002276
:104C2000FDF79AFE3B20FDF793FE4520052100226B
:104C3000FDF792FE4520FDF78BFE02B080BD00001F
:104C400080B546F22D404CF62852C0F60000C0F662
:104C50000002002102F000FE40F27C31C2F20001AD
:104C6000086046F60D004CF6E042C0F60000C0F6C3
:104C70000002002102F0F0FD80BD00002DE9F04FA0
:104C800087B0002743F630000697CDE90477CDE9D9
:104C900002770197C4F20200016841F6000441F076
:104CA000400101600168C4F2020401F04001019179
:104CB000019901970168A4F5806541F00201016046
:104CC0000168002201F00201019101990197016838
:104CD0004FF0030A41F001010160016801F0010198
:104CE000019101990197016841F004010160016897
:104CF00001F00401019101990197016841F020013F
:104D00000160016801F0200101910199019701689A
:104D100041F080010160016801F080010191019979
:104D20000197016841F008010160016801F0080184
:104D3000019101990197016841F01001016000683B
:104D4000032100F01000019001982846FDF734FC83
:104D50002046402100224FF0400BFDF72DFCA4F52A
:104D6000C0594846102101220126FDF725FCA4F573
:104D7000A058404601210122FDF71EFC112003A985
:104D8000C1C102AF28463946CDF808A0FDF740FB67
:104D900020463946CDE902B6CDE90466FDF738FB79
:104DA000082002904FF4041520463946CDE90356F9
:104DB000FDF72EFB1020CDE9020648463946CDE925
:104DC0000466FDF725FB302002A961C1A4F58050DF
:104DD0003946FDF71DFB40463946CDE90266CDE96F
:104DE0000466FDF715FB092005210022FDF7B4FD3F
:104DF0000920FDF7ADFD0A2005210022FDF7ACFDDD
:104E00000A20FDF7A5FD172005210022FDF7A4FDCE
:104E10001720FDF79DFD07B0BDE8F08F80B540F28B
:104E20000C6045F60041C2F20000C4F2000141F6F8
:104E3000802200234FF4804CC0F2060280E80E006E
:104E4000C0E9033CC0E90533C0E90733FDF7C0FB07
:104E5000002818BFFDF7EEF880BD0000B0B540F2A5
:104E6000606043F20001C2F20000C4F201014FF49D
:104E70008272002380E80E0000F10C014FF0020C5A
:104E80004FF0010E4FF40074182581E808500A21F4
:104E9000C0E90645C0E90833C0E90A31FEF734F835
:104EA000002818BFFDF7C6F8B0BD000080B588B077
:104EB00040F2007044F200420021C2F20000C4F24D
:104EC00001024FF6FF730791CDE90511CDE90311FA
:104ED000CDE90111C0E90021C0E90213016181613E
:104EE000FEF7DEFD002818BFFDF7A4F840F20070C1
:104EF000C2F20000FEF70CFF002818BFFDF79AF879
:104F0000602001900020CDE90200059040F2007081
:104F1000C2F2000001A90022FEF7AEFE002818BF71
:104F2000FDF788F840F20070C2F20000FEF702FEC2
:104F300008B080BD10B592B040F2B86000210024E6
:104F4000C2F20000C4F2010140F69F731194CDE952
:104F50000F44CDE90D44CDE90B44CDE90944CDE939
:104F60000744CDE90544CDE90344CDE90144A72236
:104F700080E81600C0E90334C0E90544FEF7C8FE26
:104F8000002818BFFDF756F840F2B860C2F20000E2
:104F900010A9CDE91044FEF727FD002818BFFDF742
:104FA00049F8602009900020CDE90A00CDE90C0005
:104FB000CDE90E0040F2B860C2F2000009A900225B
:104FC000FEF75AFE002818BFFDF734F840F2B8602B
:104FD000C2F2000009A90422FEF74EFE002818BF05
:104FE000FDF728F840F2B860C2F2000009A90822D3
:104FF000FEF742FE002818BFFDF71CF840F2B8602B
:10500000C2F2000009A90C22FEF736FE002818BFE4
:10501000FDF710F800200590CDE90300CDE901006F
:105020004FF40051089040F2B8600691C2F20000BF
:1050300001A9FEF7B3FC002818BFFCF7FBFF40F204
:10504000B860C2F20000FEF775FD12B010BD00009E
:1050500010B58AB040F2487040F600010024C2F258
:105060000000C4F200014FF6FF730994CDE9074434
:10507000CDE90544CDE90344CDE90144A72280E808
:105080001600C0E903348461FEF742FE002818BF11
:10509000FCF7D0FF40F24870C2F2000008A9CDE949
:1050A0000844FEF7A1FC002818BFFCF7C3FF6020EE
:1050B00001900020CDE90200059040F24870C2F254
:1050C000000001A90822FEF7D7FD002818BFFCF751
:1050D000B1FF40F24870C2F20000FEF72BFD0AB0AB
:1050E00010BD000010B58AB040F2907040F600414B
:1050F0000024C2F20000C4F200014FF6FF720994CE
:10510000CDE90744CDE90544CDE90344CDE90144A7
:10511000C0E90014C0E9024204618461FEF7F8FDB1
:10512000002818BFFCF786FF40F29070C2F2000022
:1051300008A9CDE90844FEF757FC002818BFFCF782
:1051400079FF602001900020CDE90200059040F237
:105150009070C2F2000001A90022FEF78DFD002828
:1051600018BFFCF767FF40F29070C2F2000001A97F
:105170000422FEF781FD002818BFFCF75BFF40F218
:105180009070C2F2000001A90822FEF775FD002808
:1051900018BFFCF74FFF40F29070C2F20000FEF71C
:1051A000C9FC0AB010BD000080B540F2D87044F6CA
:1051B0000001C2F20000C4F2000148F2A062002324
:1051C0004FF00C0CC0F2010280E80E00C0E903337E
:1051D000C0E905C3C361FFF727F8002818BFFCF733
:1051E00029FF80BD80B540F6200041F20041C2F2A7
:1051F0000000C4F2010100234FF00C0C4FF4E13227
:1052000080E80E00C0E90333C0E905C3C361FFF7BE
:105210000BF8002818BFFCF70DFF80BDFEE700006B
:10522000FEE7000000F0070080F00703042B28BF12
:1052300004234FF0FF3C03380CFA03F338BF00207F
:10524000994381400CFA00F022EA000008437047BD
:10525000B0B52DED0C8B044610EE100AB0EE618A4D
:10526000B0EE419AB0EE60AAB0EE40BA01F0E4FFB1
:10527000002800F0A2801AEE100A01F0DDFF0028DD
:1052800000F09B8019EE100A01F0D6FF002800F014
:10529000948018EE100A01F0CFFF002800F08D80F6
:1052A0006068B0EE4B0A90ED071AF0EE4A0AFCF780
:1052B00073FC6068B0EE40BA90ED001A04F128006B
:1052C00020EE01CA21EE0A0AFFF7AEFB207888B172
:1052D000012811D194ED081A94ED022A30EE411AFA
:1052E000B4EE428AF1EE10FAC8BFB0EE482A81EE61
:1052F000029A01E09FED339A19EE100A84ED07BA85
:1053000084ED080A01F098FF65689FED2E0A0028D9
:1053100008BFB0EE409A95ED010A95ED032A95ED90
:10532000021A2CEE00DA29EE02AA94ED030A9FED90
:10533000269A2CEE082A32EE00CAB4EE491A3DEE47
:105340004ABAF1EE10FA2CEE018A1ADD1CEE100AB0
:1053500001F072FFA8B13BEE080A95ED051AB0EE18
:10536000C00AB4EE410AF1EE10FA0ADC95ED040A27
:10537000B0EECC1AB4EE401AF1EE10FAD8BF84EDBC
:1053800003CA84ED058A3BEE088A18EE100A84ED04
:1053900004DA84ED06AA01F04FFF70B1D5ED050ADD
:1053A000F4EE490AF1EE10FA05DDB0EE480AFBF71B
:1053B00055FEB0EE408A84ED098A94ED090ABDECF1
:1053C0000C8BB0BD00000000BD37863570B52DEDEB
:1053D000048B90B3044650681646B0EE408A0D46E2
:1053E00001F02AFF58B3B06801F026FF48B3F06817
:1053F00001F022FF38B3306901F01EFF28B3706955
:1054000001F01AFF18B3B7EE000A80EE089A666042
:1054100019EE100A01F010FFD8B1D6ED060A04F11A
:105420002800B0EE480A84ED029AFFF73BFB2046C5
:10543000257000F013F800200CE0FF200AE0FF20A8
:1054400008E0FF2006E0FF2004E0FF2002E0FF204C
:1054500000E0FF2040B2BDEC048B70BD10B558B128
:1054600000249FED070AC460C0E907444462283065
:10547000FFF76AFB60B210BDFF2460B210BD00BF31
:10548000000000000000000000000000000000001C
:10549000EFF30980BFF36F8F154B1A681EF0100FE2
:1054A00008BF20ED108A20E9F04F10602DE90900B7
:1054B0004FF0500080F31188BFF34F8FBFF36F8F11
:1054C00003F034FC4FF0000080F31188BDE80900C0
:1054D00019680868B0E8F04F1EF0100F08BFB0EC74
:1054E000108A80F30988BFF36F8F704700BF00BF39
:1054F000C0090020B0B52DED028B00F59B659FED36
:10550000118AD5ED010A95ED050AD0ED021A04467F
:105510007030B0EE481AFFF79BFE85ED080AD5ED16
:10552000000A95ED060AD4ED021A04F58070B0EE7B
:10553000481AFFF78DFE002085ED090ABDEC028BAD
:10554000B0BD00BF0000000070B52DED028B00F56E
:1055500099669FED1D8AD6ED000A96ED0D0AD0EDF5
:10556000021A044600F12805B830B0EE481AFFF7D9
:105570006FFE96ED021A86ED130A96ED0B0AD4ED36
:10558000021A04F5A470F1EE410AB0EE481AFFF7D2
:105590005FFE96ED011A86ED140A96ED0C0AD4ED25
:1055A000021AF1EE410A2846B0EE481AFFF750FE03
:1055B00086ED120A96ED130A04F57270FFF734FABD
:1055C0000020BDEC028B70BD000000000000000058
:1055D0002DE9F0472DED028B002800F0BB8004463A
:1055E0000D46FCF75DF907F0D2F89FED878A00EED3
:1055F000100A80EE080A10EE100A07F051F9C4E90B
:105600000001FCF74DF9D4E90423801A994107F011
:10561000BEF800EE100A80EE080A84ED020AFCF7DC
:105620003FF994F82020C4E90401022A00F0948094
:10563000012A60D0002A40F0DA80686807F07CF820
:105640009FED6D0B58EC109B4A46434606F07AFDE1
:105650009FED6B0B56EC107B3A46334606F05CFA36
:1056600006F028FA00EE100A0420FCF71BF8686820
:1056700007F062F84A46434606F064FD3A46334670
:1056800006F04AFA06F016FA00EE100A01204FF072
:10569000010AFCF707F8686807F04EF84A464346E7
:1056A00006F050FD3A46334606F036FA06F002FAA6
:1056B00000EE100A0220FBF7F5FF686807F03CF8DF
:1056C0004A46434606F03EFD3A46334606F024FA83
:1056D00006F0F0F900EE100A0320FBF7E3FF204686
:1056E000294600F0F3FA002871D0D4E9000184F8CB
:1056F00020A0C4E906019FED458A0420B0EE480AC7
:10570000FBF7D0FF0120B0EE480AFBF7CBFF0220E9
:10571000B0EE480A0225FBF7C5FF0320B0EE480AA9
:10572000FBF7C0FFD4E90002A6694FF47A73A0FB2F
:105730000317881B86B2B6F5FA6F40F28036C2F2C4
:105740000006308053D902FB037084F82050C4E96E
:1057500006104CE0FF204AE0204600F01BFB2046EC
:10576000294600F075FA40F2FC16C2F200063078C5
:105770004CF6CD410130CCF6CC41A0FB0112D10852
:1057800001EB8101A0EB4100307040B994ED020AB9
:10579000B2EE041A20EE010A204600F029FA307811
:1057A000800702D12046FFF7A5FE2046FFF7CCFE7A
:1057B000204600F08DF9E87878B10020C4F82C0577
:1057C000C4F83005C4F83405C4F838050AE004F21A
:1057D0000C5000F035FAFF2009E0A878002818BF27
:1057E00000F008FB04F20C5000F0E2F9002040B297
:1057F000BDEC028BBDE8F087E17A14AE47E1CA3F09
:105800009A9999999999D13F00247449CDCC8C3EAD
:10581000002900F014812DE9F04F81B02DED068BA9
:1058200082B0054600F5966A416200F58D60B0EEE3
:10583000408A0C46FFF7E0F805F28C40FFF7DCF8F1
:105840002088B3EE0E9A00906088B4F8049001901E
:10585000B4F806B005F51A70B0EE480AF0EE490A41
:10586000FFF720F905F52270B0EE480AF0EE490A7C
:10587000FFF718F905F52A70B0EE480AF0EE490A6C
:10588000FFF710F9B3EE04AA05F53270B0EE480A3E
:10589000F0EE4A0AFFF706F905F53A70B0EE480A4D
:1058A000F0EE4A0AFFF7FEF805F54270B0EE480A3E
:1058B000F0EE4A0AFFF7F6F805F54A70B0EE480A2E
:1058C000F0EE4A0AFFF7EEF8B2EE04AA05F55270C0
:1058D000B0EE480AF0EE4A0AFFF7E4F805F55A7010
:1058E000B0EE480AF0EE4A0AFFF7DCF805F5627000
:1058F000B0EE480AF0EE4A0AFFF7D4F805F56A70F0
:10590000F2EE0E0AB0EE480AFFF7CCF805F5727019
:10591000F1EE040AB0EE480AFFF7C4F805F57A770D
:10592000002600BFB819B0EE480AF0EE490AFFF7AA
:10593000B9F82036802EF5D100EE109AB8EE408AE4
:1059400005F5C87004F14C020121B0EE480A05F1DA
:10595000280804F10C07FFF739FD05F580700121D7
:10596000B0EE480A3A46FFF731FD05F1700004F148
:105970002C020121B0EE480AFFF728FD00EE10BA14
:10598000B8EE408A05F5A47004F1AC020121B0EE36
:10599000480AFFF71BFD05F1B80004F16C02012174
:1059A000B0EE480AFFF712FD04F18C0240460121D7
:1059B000B0EE480AFFF70AFD009905F5EC7000EE1D
:1059C000101AB8EE400A04F1CC020121FFF7FEFCE8
:1059D000019905F5087000EE101AB8EE400A04F1BE
:1059E000EC020121FFF7F2FCDAF830009AED090A27
:1059F0009AED0A1A9AED0B2ACAF8580004208AED8B
:105A00000E0A8AED0F2A8AED101A8AED000A8AED35
:105A1000011A8AED022AFBF78DFE0120FBF78AFEB0
:105A20000220FBF787FE0320FBF784FE002002B074
:105A3000BDEC068B01B0BDE8F04F40B27047FF20CF
:105A400040B2704790ED001AB4EE401AF1EE10FA31
:105A500002DA80ED000A7047B4EE601AF1EE10FA37
:105A6000B0EE600AC8BF80ED000A704790ED000AF2
:105A700091ED001A92ED002A30EE011A93ED003AF2
:105A800031EE021A31EE031AB7EE002AB4EE421AD2
:105A9000F1EE10FAD8BF704782EE011A20EE010A2B
:105AA00080ED000A91ED000A21EE000A81ED000A66
:105AB00092ED000A21EE000A82ED000A93ED000A41
:105AC00021EE000A83ED000A70470000000000008C
:105AD0002DE9F04F81B000F20C548046211D04F1F5
:105AE000080204F10C032046FFF7C0FF94ED000A02
:105AF00094ED011A94ED022A94ED033A30EE414AF6
:105B000030EE010A30EE421A30EE020A31EE031A8C
:105B100030EE430A34EE425A34EE022A84ED051A7E
:105B200084ED060A9FED1E0B9FED1F1B35EE435AB9
:105B300032EE032A84ED045A84ED072A04F120058D
:105B400008F57A7A00265BEC109B54EC117B00BFC1
:105B5000D8F8240090ED460AD0ED470AA5F11000D0
:105B6000FFF770FF55F8100C06F0E6FD4A465B465D
:105B700006F0E8FA3A46234605F0CEFF05F09AFF14
:105B800000EE100A28600AEB0600FEF74DFF2036F3
:105B9000802E05F10405DBD1002001B0BDE8F08FB7
:105BA000E17A14AE47E1CA3F9A9999999999D13F00
:105BB000D0B110B590ED080A04460420FBF772FD41
:105BC00094ED090A0120FBF76DFD94ED0A0A02200D
:105BD000FBF768FD94ED0B0A0320FBF763FD002043
:105BE000BDE8104040B27047FF2040B2704700004F
:105BF000B0B500F2E445F0EE401AD5ED000A95ED9F
:105C0000070A9FED0E1A044600F50870FFF720FB07
:105C100005F1200085ED080ABFEE000AF7EE000A44
:105C2000FFF710FF606A95ED081A90ED020A002058
:105C300030EE010A85ED0A0AB0BD00BF0000000089
:105C400000220146C0E9082282620020CA62704731
:105C5000F0B581B00446486804F2B447F8648A6835
:105C6000384640F8402F91ED032A91ED043A616ADD
:105C700097ED000A97ED011AD1ED430A33EE000AC1
:105C800032EE011A87ED0F0AB1EE600A07F138050E
:105C900007F13C0687ED0E1AFFF7D4FE606A97ED18
:105CA0000E1A90ED442A284631EE420A71EE020A9D
:105CB000FFF7C8FE606AD0ED450A3046B1EE600AD3
:105CC000FFF7C0FE002001B0F0BD0000B0B591EDBF
:105CD000010A9FED2C1A0446B4EE410AF1EE10FAC7
:105CE0004FF000051ADA91ED020A9FED271AB4EE83
:105CF000410AF1EE10FA11DD91ED041A9FED230A2D
:105D0000B4EE401AF1EE10FA08DA91ED031A00250C
:105D1000B4EE401AF1EE10FAB8BF0125FBF7C0FD52
:105D200006F035FD40F2FD11C2F2000125B39FEDF2
:105D3000180A01EE100A81EE000AD4E906021043A7
:105D4000BCEEC00A10EE100A04BF0022C4E906022D
:105D5000D4E90623801A4FF000029A41B0F57A7018
:105D600072F1000006D3087820B9012008700020E5
:105D7000C4E906000878B0BD0020C4E90600087830
:105D8000B0BD00BFCDCCCC3D6666663F666666BFE3
:105D900000007A44B0B500F5996595ED000A044617
:105DA00000F53270FEF740FE95ED010A04F53A70F9
:105DB000FEF73AFE95ED020A04F54270FEF734FE56
:105DC00095ED050A04F55A70FEF72EFE95ED040ACE
:105DD00004F55270FEF728FE95ED060A04F5627090
:105DE000FEF722FE95ED070A04F56A70FEF71CFE29
:105DF0000020B0BD80B50420FBF7B2FC0120FBF70A
:105E0000AFFC0220FBF7ACFC0320FBF7A9FC80BD34
:105E100080B586B00020CDE90400CDE90200012064
:105E2000019041F20040C4F2020001A9FCF7F0FA2F
:105E300006B080BD80B586B000200590CDE9030096
:105E40000120CDE9010041F20040C4F2020001A9A5
:105E5000FCF7DEFA06B080BD80B5806B01684A6849
:105E600022F003024A60416D41F0100141650121B9
:105E700080F85110FDF736F880BD000080B5806BCA
:105E8000FDF776FA80BD000080B5806BFDF74CFD14
:105E900080BD000080B5806BFDF76AFD80BD00000D
:105EA000B0B5846B0546FCF78DFB29680968C90508
:105EB00026D402462068A168436823F0200343608B
:105EC00031B96168B1F5827F02D16FF0030101E061
:105ED0006FF001014368194041602046642100F0E1
:105EE00079F800281CBF202060650020E087012091
:105EF00084F85100606D18B12046FCF7F3FFB0BD87
:105F00002046FDF723FAB0BDB0B582B0846B0546DC
:105F1000FCF758FB29680968C90528D4024620689F
:105F2000416821F020014160416821F00201416097
:105F30002046642100F096F818B1606D40F0200012
:105F40006065A06838B9002001902068C16801919F
:105F50008068019001980020E086012084F85100BB
:105F6000606D20B12046FCF7BDFF02B0B0BD2046F9
:105F7000FDF7CAFC02B0B0BDB0B5846B0546FCF7B6
:105F800021FB29680968C9051FD4024620684168B9
:105F900021F0200141602046642100F063F818B12F
:105FA000606D40F0200060652068416821F00301C9
:105FB00041600020E086E087012084F85100606D98
:105FC00018B12046FCF78EFFB0BD2046FDF7BEFCA1
:105FD000B0BD0000B0B582B0044640680B46B0F5D5
:105FE000827F20D1A168B1F5004F02D0B1F5806F5A
:105FF00004D121680D6825F040050D60B0F5827F61
:1060000011D1A068B0F5806F1DD10092204601210A
:106010000022002500F076F890B1606D032540F075
:10602000200060650CE0009220460121002200253E
:1060300000F068F820B1606D032540F02000606535
:10604000284602B0B0BD00922046802100220025E3
:1060500000F058F80028F3D0606D032540F02000D0
:106060006065EDE770B582B00D461646022101224B
:106070002B460446009600F045F838B1606D0325C4
:1060800040F020006065284602B070BD40F200007C
:10609000C2F20000006849F68171C1F25E61A0FBA6
:1060A0000101480D4FF47A71484301906068B0F5E2
:1060B000827F0FD12046802100222B4600960025AA
:1060C00000F020F80028DED0606D032540F02000AD
:1060D0006065D8E7019840B10198013801902068C7
:1060E00080680006F6D40025CDE70025CBE7000048
:1060F000006843F20001C4F20101401A18BF0120F8
:10610000400070472DE9F04782B00A9C984615463A
:106110000E468146FCF756FA201A00EB0804FCF7FD
:1061200051FA40F20001C2F200010968C1F3CB311B
:1061300061430191D9F8001089683140891BB1FA97
:1061400081F14909A94203D1002002B0BDE8F087DE
:10615000824608F101070CE0019801380190D9F856
:10616000000080683040801BB0FA80F04009A842EF
:10617000EAD0002FF3D0FCF725FAA0EB0A00A042EA
:1061800004D201980028E7D10024E8E7D9E900010A
:106190004268B1F5827F22F0E00242600BD1D9F86B
:1061A0000810B1F5004F02D0B1F5806F03D101683E
:1061B00021F040010160D9F82810B1F5005F07D146
:1061C000016821F400510160016841F4005101604F
:1061D000012089F85100002089F85000032002B006
:1061E000BDE8F0870000000080B500EE100AB8EEB0
:1061F000C00A10EE100A06F09FFA9FED110B53EC47
:10620000102B05F045FD41EC100B9FED0F1B04F02A
:106210008BFA53EC102B9FED0E0B51EC100B06F08C
:106220009DF99FED0D0B53EC102B05F08BFF9FEDAF
:106230000C0B53EC102B05F085FF05F0BFFE80BD65
:1062400000000000D0BCF8406C45D9CC955BC83F3D
:10625000000000000000F03F0000000040A5E54005
:106260000000000000408F4080B50C20892102F022
:1062700037FA00281CBF012080BD6420FBF7D4FA48
:1062800002F0D8F940B2B0F1FF3FF9DC02F04EF96C
:1062900002F0D0F94006FBD50D2002F0FDF941F2E5
:1062A000044100F0F002C2F20001102A08701CBF85
:1062B000022080BD7020032102F0DAF87020032153
:1062C00002F004F9072002F005FA002080BD00006A
:1062D0002DE9F04F81B02DED048B8846824602F007
:1062E000C5F941F20444C2F2000494ED041A00EE30
:1062F000100AB8EEC00AB8EEC11A80EE018A02F0A8
:106300009FF994ED031A41F21844C2F2000400EE22
:10631000100AB4F90000B8EEC00AB8EEC11AB4F918
:106320000250B4F90C90B4F90EB080EE019A05F069
:10633000A2FE9FED310B53EC102B05F003FF00EE96
:10634000105AB8EEC00A28EE000A064610EE100AEF
:106350000F4606F0F1F902460B463046394605F085
:10636000DBFB05F02BFECAF80000B4F9100094ED39
:10637000021A02EE100AB4F91400B8EEC22A03EEB3
:10638000100AB8EEC33A29EE033A33EE022A94ED2E
:10639000010AB8EEC11A29EE022AB4F9120032EE4F
:1063A000011A04EE100AB8EEC00A29EE011A03EE33
:1063B00010BAB8EEC44A31EE000A01EE109AB8EEF7
:1063C000C33A29EE044AB8EEC11A28EE092A34EE7F
:1063D000033A28EE011A22EE032A31EE000A32EEC9
:1063E000000ABDEEC00A002088ED000ABDEC048B57
:1063F00001B0BDE8F08F00BF000000000000E03FEA
:10640000074B19680868B0E8F04F80F30988BFF3BC
:106410006F8F4FF0000080F31188704700BF00BFFE
:10642000C009002080B500F055FF80BD80B501F0A7
:106430000FFA01F06BFA80BDB0B501380024B4EB5F
:10644000106F1CBF0120B0BD4EF21005CEF200054A
:1064500068604FF0FF300F2100F02AFF0720AC608A
:1064600028602046B0BD000080B5FCF7F7F903F0C6
:1064700035FA012818BF02F049FD80BD70B592B011
:1064800006AC20463021FAF706F8002543F6400016
:106490000595CDE90355CDE901550095C4F20200FB
:1064A0000168022641F080510160006800F08050D0
:1064B0000090009847F200000095C4F200000168C7
:1064C00041F480410160006800F480400090009831
:1064D000012006904FF4803007904FF480000D901B
:1064E00006200E90A820CDE90F060420119020462A
:1064F0000C96FCF753FB88B90F20CDE901064FF449
:10650000A05004904FF48050059001A805210395F8
:10651000FCF736FA002804BF12B070BDFBF78AFD05
:106520004EF68850CEF20000016841F4700101601F
:1065300070470000B0B540F6FF3E0568C4F2000E9B
:1065400040F2004C7045C4F2010C0FDCB0F1804FFA
:1065500019D040F20043C4F20003984213D040F631
:106560000003C4F2000398420DD011E040F600434E
:10657000C4F20003984206D0604504D00023C4F260
:106580000103984204D14B6825F0700243EA0205EA
:1065900041F6FF73C4F2000398420DDC70451FDC26
:1065A000B0F1804F41D040F20043C4F20003984262
:1065B0003BD040F6000321E043F6FF73C4F2010331
:1065C000984220DC42F20003C4F2000398422CD02F
:1065D0000023C4F20103984227D0604525D029E06A
:1065E00040F60043C4F2000398421ED041F6000377
:1065F000C4F20003984218D041F60043C4F20003ED
:10660000984212D016E044F20003C4F2010398420B
:106610000BD044F60003C4F20103984205D044F2C3
:106620000043C4F20103984204D1CB6825F44072C0
:1066300043EA02050A688C684B69C46240F48064CE
:106640008262644504BF09690163026825F0800124
:1066500042F0040219430260012242610160B0BDB0
:1066600080B501F01F014FF0010CD0F820E00CFACA
:1066700001F32EEA03030362036A02FA01F11943EC
:10668000016280BDB0B5026A036A40F2004523F0A2
:1066900001030362D0F804E0D0F818C08C6822F03F
:1066A000020240F48063C4F20105AB4242EA0402F4
:1066B00005D1CC6822F00C0224F0040422430C68BB
:1066C000AB4207D1D1E905532EF4407E45EA0E05D1
:1066D00045EA030E2CF073032343C0F804E0836102
:1066E000496841630262B0BD70B5026A036A40F254
:1066F000004423F010030362D0F804E0D0F818C07F
:106700008D6822F0200240F48063C4F20104A342A9
:1067100042EA051207D1CD686FF0400622F0C002B0
:1067200006EA05152A430D68A34207D1D1E905649D
:106730002EF4406343EA860343EA840E2CF4E643D6
:1067400043EA0523C0F804E083614968816302627B
:1067500070BD000070B5026A036A40F2004423F481
:1067600080730362D0F804E0D0F81CC08D6822F476
:10677000007240F48063C4F20104A34242EA05229D
:1067800007D1CD6840F2FF462D0222F44062B543A6
:106790002A430D68A34207D1D1E905642EF4405382
:1067A00043EA061343EA041E2CF073032B43C0F89C
:1067B00004E0C3614968C163026270BD70B5D0F87E
:1067C00020C0026A40F2004622F48052026242680F
:1067D000C3690C68D1F808E040F48065C4F2010692
:1067E000B54204D14D6922F4804242EA851223F475
:1067F000E64343EA04234260C3612CF4005649682F
:1068000046EA0E320164026270BD000010B500F06D
:1068100053FE46F601104CF65042C0F60000C0F69A
:106820000002002101F018F841F23044C2F20004E5
:10683000206046F6D9204CF67442C0F60000C0F63F
:106840000002002101F008F8606046F619404CF69D
:10685000BC42C0F60000C0F60002002100F0FCFFC0
:10686000A06046F6D1404CF60452C0F60000C0F6D7
:106870000002002100F0F0FFE06046F661304CF6C7
:106880009842C0F60000C0F60002002100F0E4FFCC
:10689000206105200C21002200F0A4FEA06105204B
:1068A0001021002200F09EFEE06103200C21002256
:1068B00000F098FE206203200C21002200F092FEDE
:1068C000606203200C21002200F08CFEA0620320F5
:1068D0000421002200F086FEE06203200421002251
:1068E00000F080FE206303201421002200F07AFED5
:1068F000606300F011FE00F0ABFF01F007F810BD7F
:1069000084B000F0C1FD05F0CDFB9FED6F0B53ECA3
:10691000102B05F0BDF905F081FB0646002000F0C4
:106920006BFD00F0A7FD40F20835C2F2000540F211
:1069300008010446C2F200012846FAF763FC284623
:10694000FAF73AFC40F2A43040F6BC01C2F2000073
:10695000C2F20001F9F780FE2846FAF72DFCB7EEE7
:10696000001A81EE000A40F668004CF64C52C2F262
:106970000000C0F600020021FEF728FD0520FAF70E
:10698000D9FE05F110009FED528A9FED529A41F217
:106990009C3B40F28C3A40F2842904EB06080290BA
:1069A00005F11C00C2F2000BC2F2000AC2F200099B
:1069B00003960190FAF774FDFAF7EAFBFAF7F4FB95
:1069C000FAF70AFCFAF716FC00F076FD2846FAF70B
:1069D000BBFC2846FAF702FD40F2A437C2F20007DA
:1069E000DDE9012140F6BC033846C2F20003F9F7A5
:1069F000F5FE40F29834C2F2000420463946F9F719
:106A0000BDFD00F089FDD5E90403AA6940F27821B3
:106A1000C2F20001C1E900038A60D7E90006D7E9A4
:106A20000223CBE90006CBE90223D4E90003A268E4
:106A3000CAE90003D5E9040705F11806C9E900070A
:106A400040F2BC37CAF808205CCEC2F20007C7E9A2
:106A5000003441F23044C2F20004A069C9F80820B1
:106A600000220023BE6000F00DFEE06959460022BE
:106A7000002300F007FE206A51460022002300F0A8
:106A800001FE606A49460022002300F0FBFDA06A77
:106A900039460022002300F0F5FDD5ED0A0A40F644
:106AA0006800C2F20000B0EE480AB0EE491AF0EEFB
:106AB000491AFEF7CDFB0520FAF7F4FD404600F039
:106AC000ABFC0398804475E70000000000408F4055
:106AD000000020420000000000F0D6FC05F0E2FAC1
:106AE0009FED1B0B53EC102B05F0D2F805F096FA36
:106AF0000446002000F080FC00F0BCFC05460820A5
:106B0000FAF72EFE0620FAF72BFE9FED130A072058
:106B1000FAF7C8FD0720FAF70DFE9FED108A25440D
:106B2000B7EE009AB6EE00AA00EE105AB8EE400A90
:106B300020EE080A04F028FC30EE090A20EE0A0ACA
:106B40000720FAF7AFFD284600F066FC2544EBE786
:106B5000000000000000594000000000A69B443BDC
:106B600000F092FC05F09EFA9FED290B53EC102BE0
:106B700005F08EF805F052FA8346002000F03CFC48
:106B800000F078FC40F2D828C2F2000805464046E2
:106B9000FBF726F840F24D39C2F200094846FBF7F0
:106BA0008BF905EB0B0741F2C43540F2683641F230
:106BB000304AC2F20005C2F20006C2F2000A13E037
:106BC000286805F108041ECCC6E90002DAF8340092
:106BD000C6E90213314600220023346100F052FD61
:106BE000384600F019FC5F440A20FBF773F90028CF
:106BF000E6D048464146FBF717F840462946FAF7E3
:106C0000C1FE4846FBF758F9DAE700BF00BF00BFF6
:106C10000000000000407F4000F036FC05F042FA22
:106C20009FED270B53EC102B05F032F805F0F6F929
:106C300080464FF4FA7000F0DFFB00F01BFC9FED84
:106C4000220A0446FDF7A0FC04EB080541F230449B
:106C500040F26C2641F28C3740F2843940F2883A97
:106C6000C2F20004C2F20006C2F20007C2F200093A
:106C7000C2F2000AA06931460022002300F06EFC37
:106C8000E06939460022002300F068FC96EC030A14
:106C9000D7EC041A48465146FDF720FCE06A494605
:106CA0000022002300F0EEFC206B5146002200235E
:106CB00000F0E8FC284600F0AFFB4544DAE700BFEF
:106CC0000000000000407F400000FA430000000088
:106CD00082B000F0D9FB05F0E5F99FED370B53ECDE
:106CE000102B04F0D5FF05F099F9054640F6B830B1
:106CF00000F082FB00F0BEFB0446FAF76BFF40F6A3
:106D00003868C2F2000841F278329FED2D0A014640
:106D1000C2F200024046FEF77BFD41F2304941F2EB
:106D2000783A01956719C2F2000908F2D44B08F2CB
:106D3000BC4408F5996608F59C6508F2E448C2F27F
:106D4000000A00BFD9F8200059460022002300F0B5
:106D500005FCD9F8240021460022002300F0FEFBA8
:106D6000D9F8280031460022002300F0F7FBD9F8BB
:106D70002C0029460022002300F0F0FBD9F8300057
:106D800041460022002300F0E9FBD9F834005146C7
:106D90000022002300F0E2FB40F63860C2F200005F
:106DA0005146FEF715FC384600F036FB01980744C3
:106DB000C8E700BF00BF00BF0000000000408F40D8
:106DC00000007A4480B5806B0021C185FDF7EAF8A8
:106DD00080BD000010B5846B2068406994F84110B4
:106DE000212907D110F0800004D00020E084204643
:106DF00000F09CF82068406994F84210222907D1DD
:106E000010F0400004D00020E085204600F05AF841
:106E1000606C40F0100060642046FDF7C3F810BDC0
:106E200080B50168806B0968C9052FD40021C18530
:106E3000016851E8031F026821F4807142E80313DE
:106E4000002BF5D1016851E8051F026821F001010E
:106E500042E80513002BF5D1016851E8051F0268CF
:106E600021F0400142E80513002BF5D1202180F8E4
:106E70004210016B012909D1016851E8031F026822
:106E800021F0100142E80313002BF5D100214163EA
:106E9000016B012903D1818DFDF782F880BDFDF7DB
:106EA000DFFA80BD80B5806B01214163016B012950
:106EB00004D1818D4908FDF773F880BDFDF7E4FA30
:106EC00080BD0000016851E8031F026821F4907141
:106ED00042E80313002BF5D1016851E8051F026851
:106EE00021F0010142E80513002BF5D1016B0129C6
:106EF0000AD100BF016851E8031F026821F01001A8
:106F000042E80313002BF5D1202180F84210002124
:106F10000163704780B50168CA6822F04002CA6008
:106F2000202180F84110FDF7C3FA80BD016851E8C7
:106F3000031F026821F0C00142E80313002BF5D1C2
:106F4000202180F84110704744F600010068C4F227
:106F5000000101F54C420323904208BF0123401A6F
:106F600018BF18467047000080B582B090F84210F4
:106F700022291ED18268B2F5805F02D10169002901
:106F80004AD0816AB2F5805F07D00AB9026922B19E
:106F90000268526802F07F0201E0026852680A70DB
:106FA0000121826A11448162C18D01390A04C185BF
:106FB00001D002B080BD0168CA6822F02002CA6018
:106FC000CA6822F48072CA604A6922F001024A61EA
:106FD000202180F8421000214163026B012A23D155
:106FE000016300BF016851E8031F026821F010012E
:106FF00042E80313002BF5D101680A68D20606D5D2
:10700000002201920A680192496801910199818DDB
:10701000FCF7C6FF02B080BD0168826A49686FF361
:107020005F2111800221BCE7FDF71AFA02B080BD92
:1070300010B504460068D4E902C22369016921F44D
:10704000405111430161626943EA0C01E369114354
:10705000C268194349F20C639A431143C160416904
:10706000A26921F4407141F20043114340F480626F
:10707000C4F201039A42416102D1FBF749FD01E0EC
:10708000FBF734FDE16963681922B1F5004FA0FBFD
:1070900002011CD15A00DB0FF9F706F948F21F5123
:1070A000C5F2EB11A0FB01235A096FF0630302FB49
:1070B0000300322303EBC000A0FB01014FF4F87082
:1070C00000EA111000EB0210C1F342111AE09A001D
:1070D0009B0FF9F7E9F848F21F51C5F2EB11A0FB3D
:1070E00001235A096FF0630302FB0300322303EB11
:1070F0000010A0FB0101F02000EA511000EB02108B
:10710000C1F3431122680843906010BDF0B581B00F
:10711000134600270446816283854764222084F851
:107120004200E06B46F6216546F6A5660A462168F0
:10713000C0F60005C0F60006C0E90F5646F6D55663
:10714000C0F600060431C0E91367FBF7F7F838B161
:1071500010206064202084F84200012001B0F0BDBE
:1071600000972068016800914068009000982069AD
:1071700050B100BF206850E8030F216840F48070D0
:1071800041E80302002AF5D1206850E8050F216884
:1071900040F0010041E80502002AF5D1206850E8DE
:1071A000050F216840F0400041E80502002AF5D1B2
:1071B000002001B0F0BD000090F84110212923D13A
:1071C0008168B1F5805F01D1016931B1016A02685E
:1071D0004B1C03620978516007E0016A036831F8CB
:1071E000022B6FF35F225A600162C18C01390A04DD
:1071F000C18418BF70470068C16821F08001C16078
:10720000C16841F04001C1607047000010B540F610
:107210002004C2F200042046FCF7D8FE2046FAF70C
:1072200077FB10BDFEE7000000F0FF40B0F1FF402B
:1072300018BF01207047000000F0FF40B0F1FF4090
:1072400018BF01207047000020F00040A0F1FF406F
:10725000B0FA80F040097047002848BF704700F03E
:107260001F01012202FA01F14EF280124009CEF212
:10727000000242F82010BFF34F8FBFF36F8F7047AB
:10728000002848BF704700F01F01012202FA01F1F7
:107290004EF200124009CEF2000242F82010704770
:1072A0004EF60C50CEF200000068C0F3022070478A
:1072B0004EF6145300F00F02CEF2000309011A44F7
:1072C00000F16043B0F1FF3FC8BF03F564421170A5
:1072D000704700004EF61F50CEF2000000210170F2
:1072E000704700004EF60C51CEF200010A684FF6CE
:1072F000FF031A4060F30A2242F0806040F0FD7004
:107300000860704740F6DB7110EE100AC3F6C971D1
:1073100061F31E0000EE100A70470000F0B581B066
:10732000F0B1044640F6C010C2F200000068A0426E
:107330001FD001F06DFA40F6C810C2F20000656976
:10734000076840F6D010C2F20000066801F084FA27
:10735000BD424FF0020018BFB5420DD101B0F0BDE3
:107360004FF0500080F31188BFF36F8FBFF34F8F42
:10737000FEE7002001B0F0BD47F61060C2F2000049
:1073800085420CD047F624610120C2F20001002D95
:1073900008BF04208D4208BF042001B0F0BDA06AE0
:1073A00010B1022001B0F0BD94F85810032001295B
:1073B00008BF022001B0F0BDFBF75EFAFFF75EF8F0
:1073C000FDF75CFCFDF7EEFBFDF728FDFDF7B2FDD8
:1073D000FDF73EFEFDF786FEFDF768FDFDF73EFD7D
:1073E000FDF700FFFDF7E0FE00F052F8FDF728FC86
:1073F00000F078F8FEE70000EFF3058100291CBFDC
:107400006FF005007047002804BF0020704780B56A
:1074100001F002FB002080BD10B582B0EFF30581C2
:1074200019B16FF0050002B010BD044602F06AFA0F
:10743000211A0129019005DB01A801F017FB0020AA
:1074400002B010BD6FF0030002B010BD80B502F0B5
:1074500045FA022808BF80BD08B9032080BD40F26C
:10746000F810C2F2000000680138B0FA80F040095C
:1074700080BD000080B5EFF3058010B102F048FA3E
:1074800080BD02F03FFA80BD4FF47A707047000073
:10749000EFF3058000281CBF6FF00500704740F235
:1074A000F810C2F200000168002911BF4FF0FF3050
:1074B000012101600020704780B5EFF305800028AE
:1074C0001CBF6FF0050080BD02F008FA28B1022849
:1074D00005D101F023FC002080BD012080BD4FF0CC
:1074E000FF3080BD10B5EFF3058000281CBF6FF0A2
:1074F000050010BD40F2F814C2F200042068012813
:107500001CBF4FF0FF3010BDFEF78CFF0220206043
:1075100001F0B2FB002010BD10B5EFF3058018B1EB
:107520006FF00504204610BD02F0D8F902280ED0F5
:1075300080B902F07BFB01284FF001040CD002F06F
:10754000CDF9002808BF4FF0FF34204610BD0024BD
:10755000204610BD4FF0FF34204610BD10B582B05C
:107560001C46B0FA80F3B1FA81F25B095209EFF3DD
:10757000058CBCF1000F42EA030219D0002C18BFA1
:107580000124224315D10022019201AA01F082FFB9
:1075900001281AD10198A8B14EF60450CEF200008D
:1075A0004FF080510160BFF34F8FBFF36F8F09E041
:1075B0001AB16FF0030002B010BD224601F0A8FE20
:1075C000012806D1002002B010BD6FF0020002B009
:1075D00010BD6FF00100002C08BF6FF0020002B078
:1075E00010BD0000B0B582B0144600294FF0000570
:1075F000EFF3058218BF002802D1284602B0B0BDC3
:10760000002AFAD19CB1A568D5B1E268502A16D3F8
:107610002269A2B1D4F814C001FB00F20023944502
:107620004FF0000228BF012210D24DB10EE001231D
:1076300000226AB9E3B1002201F080FC0EE01DB91E
:10764000E2680AB92269C2B100220023002AF1D0FF
:10765000A36822690025009501F094FC054655B108
:10766000002C14BF21680021284601F09FF9C4E7CF
:107670000025002DF4D10025BFE76269B2FA82F23D
:107680005309D5E7B0B582B01C46B0FA80F3B1FA21
:1076900081F5EFF305825B096D09002A43EA0502D3
:1076A00007D0002C18BF0124224306D06FF0030539
:1076B0002CE0CAB16FF0030528E00022019201AA74
:1076C000002301F0BDFD01281CD10198E8B14EF660
:1076D0000450CEF200004FF080510160BFF34F8F95
:1076E000BFF36F8F002511E022460023002501F033
:1076F000D5FC01280AD06FF00105002C08BF6FF0FF
:10770000020503E06FF0020500E00025284602B004
:10771000B0BD0000B0B584B048B3B1F1FF3F26DD85
:1077200004464FF0FF300390EFF3058018B30025B7
:107730000DF1080C2046012200230295CDF800C06F
:1077400002F030F803AB204600210022009502F041
:1077500029F80298D0B14EF60450CEF200004FF056
:1077600080510160BFF34F8FBFF36F8F0EE06FF05A
:10777000030003900AE020460122002301F094FF59
:1077800003AB20460021002201F08EFF039804B0D5
:10779000B0BD00002DE9F04F83B00C46EFF305813A
:1077A00029B16FF00507384603B0BDE8F08F0546F4
:1077B000002849D44FF0000B9246A00758BFAB46B3
:1077C00002F0A0F800906FF0010804F001005446A8
:1077D0000027BAF1000F08BF6FF00208019002E025
:1077E0004746002EDFD00020594602AA234602F069
:1077F00043F906460128F3D1029807EA050140EA59
:1078000001090198002809EA050007D100286FF056
:10781000020718BF4F4607D0C5E700BFA8426FF068
:10782000020708BF4F46BED0BAF1000FBBD002F02E
:1078300069F800994F46401A241A4FF0000038BFEB
:107840000446002ECFD1AEE76FF00307ABE7000090
:1078500080B502F03DF880BD70B584B08E46002141
:1078600000280391EFF3058146D0002944D1FAB1F5
:107870009369002B08BF1823382B16D81179C90734
:1078800013D15569946811684FEA950C002D08BF13
:107890004FF0800CFCB1D6685C2E1BD3D5B11569B6
:1078A000C5B10024012555B91BE0002004B070BD0E
:1078B0000124002118234FF0800C00258DB194681D
:1078C00012690294CDE900326246734601F0B0FEBF
:1078D000039011E00CB9D4689CB100250024002D60
:1078E000EDD14CB103AC00931FFA8CF273460194B6
:1078F00001F06AFE012802D1039804B070BD002097
:10790000E6E71469B4FA84F46409D6E710B5EFF336
:10791000058100291CBF6FF0050010BD044660B151
:107920002046FFF7FBFC042804BF6FF0020010BDE7
:10793000204601F0EFF8002010BD6FF0030010BDED
:10794000F0B581B00D4647F6386140F6C016C2F278
:107950000001C2F200060F6831680446081D00F0FD
:10796000E1FE601C0AD14DB13068011D47F6106080
:10797000C2F2000000F034FF01B0F0BD3068E4193D
:1079800044600AD340F6D010C2F2000000683168AB
:10799000043100F007FF01B0F0BD40F6C810C2F29C
:1079A000000000683168043100F0FCFE47F69C508E
:1079B000C2F2000001688C4238BF046001B0F0BD23
:1079C00070B5044600F024FF47F27060C2F2000078
:1079D000016840F6C01501310160C2F20005296856
:1079E00047F60466C2F2000641B1306860B9286803
:1079F000E16AC06A884298BF2C6005E02C6000688C
:107A0000012801D100F0C2F947F27C60C2F2000007
:107A1000016801310160616447F28061C2F20001D6
:107A2000E06A0A68904288BF086040F6D81100EB0F
:107A30008000C2F2000101EB8000211D00F0D0FEA9
:107A400000F00AFF306880B12868E16AC06A8842A5
:107A500028BF70BD4EF60450CEF200004FF08051AA
:107A60000160BFF34F8FBFF36F8F70BD70B582B0F1
:107A700000F0CEFE47F63C66C2F20006306850BB0E
:107A800047F63C54C2F20004204600F07BFE47F665
:107A90005055C2F20005284600F074FE40F6C410AE
:107AA000C2F20000046040F6D410C2F2000040F6BA
:107AB000CC0240F66C1305600025C2F20002C2F24F
:107AC00000030A201021009501F05CFA306010B12B
:107AD00003A100F06BFF00F0BFFE02B070BD00BF5D
:107AE000546D725100000000F0B581B047F274652A
:107AF000C2F200052868E0B147F6246647F27067D5
:107B0000C2F20006C2F2000700F082FEF068C4680C
:107B1000201D00F007FE38680138386028680138F9
:107B2000286000F099FE204600F058F828680028E8
:107B3000EAD101B0F0BD000080B5026C002A08BF98
:107B400080BDD0E902C31344C360634524BF03680A
:107B5000C360C36808461946F8F71EFC80BD0000E4
:107B600070B5866B036C0446E3B115461AB3E06842
:107B70001A46F8F711FCE168206C2268091A914254
:107B8000E16003D2A16840420844E060A81EB0FA58
:107B900080F040093146002E18BF01210840361AF6
:107BA000002516E02068002598B9A06801F0ACFF18
:107BB000A56005460DE060681A46F8F7EDFB216CFC
:107BC000D4E90102002508446060904224BF206887
:107BD0006060711C2846A16370BD000010B50446AA
:107BE00090F85900022808BF10BD012803D030B911
:107BF000206B00F049FE204600F046FE10BD4FF01D
:107C0000500080F31188BFF36F8FBFF34F8F00BF19
:107C1000FEE7000040F6C411C2F2000109680A68DC
:107C2000B2FA82F35B090360002A0EBF0020C86825
:107C30000068704741F2BC40C2F20000C21D22F051
:107C4000070210F0070CA0EB020318BF104647F61E
:107C50000862C2F200020021C2E9000146F2A81245
:107C6000BCF1000F18BF1A440244083A40F6CC1386
:107C700022F00702C2F200031A60C2E90011111AD1
:107C80001A68C0E9002147F69850C2F2000001606E
:107C900047F69050C2F20000016047F66450C2F20D
:107CA000000001210170704740F6D8144EF60455CB
:107CB000C2F20004CEF200054FF08056FFF714FF29
:107CC00020680228FAD32E60BFF34F8FBFF36F8F67
:107CD000F4E70000B0B5049D002914BF2A602D60B0
:107CE000C5E90F01284601211C4601F097F985F8E6
:107CF0004C40B0BD2DE9F0470A9C8246206B1646E9
:107D00000F46DDE908599100A5229846F8F7BBFB1C
:107D1000206B00EB8600A0F1040020F007067FB185
:107D200004F13400002100BF7A5C42547A5C1AB13D
:107D30000F2901F10101F7D3002084F8430002E08C
:107D4000002084F834000027201D372D28BF372558
:107D5000E562C4E9135700F021FD04F1180000F0BA
:107D60001DFDC5F13800A0613046514642462461F0
:107D70006462676584F8587000F03EFBB9F1000F4B
:107D8000206018BFC9F80040BDE8F087B0B540F6E4
:107D9000D8150024C2F20005281900F0F3FC1434B1
:107DA000B4F58C6FF8D147F66854C2F2000420464F
:107DB00000F0E8FC47F67C55C2F20005284600F0CA
:107DC000E1FC47F6B050C2F2000000F0DBFC47F6E1
:107DD0002460C2F2000000F0D5FC47F61060C2F249
:107DE000000000F0CFFC40F6C810C2F200000460B2
:107DF00040F6D010C2F200000560B0BD80B547F675
:107E00000862C2F2000200BF114612688242FBD330
:107E1000D1F804C001EB0C03834203D140686044F5
:107E200048600846D0F804C000EB0C03934201D030
:107E300013460BE040F6CC13C2F200031B689A42D3
:107E400004D0D2E9003E0EEB0C0242608142036096
:107E500018BF086080BD000080B58C46014641F81F
:107E600004CF9445006108D99A4201D29C4511D2B1
:107E700040F6C410C2F2000007E08069D21A8242C4
:107E800008D240F6D410C2F20000006800F08AFC6C
:107E9000002080BD012080BD10B5044600F0B8FC74
:107EA000A06BB0FA80F0440900F0D6FC204610BD6B
:107EB00010B5044600F0ACFCA06BE16B401AB0FAC0
:107EC00080F0440900F0C8FC204610BD0848006856
:107ED000006880F308884FF0000080F3148862B6D1
:107EE00061B6BFF34F8FBFF36F8F00DF00BF00BFDE
:107EF00008ED00E070B582B040F6C412C2F2000294
:107F000012680546D2680E46D468201D00F00AFCAF
:107F100094F82800410704D400F0FE0084F82800FB
:107F200010E0A0693246411920462B46FFF794FF26
:107F300040B10026204600212A460023009601F089
:107F400039FF20B1216A2046884702B070BD4FF04A
:107F5000500080F31188BFF36F8FBFF34F8F00BFC6
:107F6000FEE700002DE9F04186B047F63C67C2F21B
:107F70000007386802A900224FF0000801F0C8F994
:107F800000286AD001AC02AD0BE000F0FE0086F8DC
:107F9000280000BF38682946002201F0B9F90028FE
:107FA0005BD00298B0F1FF3F03DCDDE903200599C7
:107FB000904702980028EDD4049E706910B1301DDE
:107FC00000F0B0FB204600F0B3F802990929E1D88F
:107FD0000246DFE801F0080808052A390808052AE2
:107FE00096F82800D1E796F82800039BB16940F085
:107FF000010086F8280019443046FFF72DFF0028BD
:10800000C8D0316A3046884796F828004007C1D565
:108010000398B16900230A1830460021CDF800808A
:1080200001F0C8FE0028B5D123E096F8280040F002
:108030000101039886F82810B06188B18118304694
:108040001346FFF709FFA5E796F8280081073FF5DB
:108050009CAF304600F018FC9CE706B0BDE8F0810C
:108060004FF0500080F31188BFF36F8FBFF34F8F35
:10807000FEE74FF0500080F31188BFF36F8FBFF31E
:108080004F8F00BFFEE7000070B582B00E46044679
:1080900000F044FE01A800F04BF8019919B101F07D
:1080A000C5FD02B070BD05464EB9A54207D301F02B
:1080B000BDFD20462946FFF71DFF02B070BD4EB141
:1080C00040F6D410C2F2000000680068B0FA80F0F8
:1080D000420900E0002247F63C60C2F2000000685E
:1080E000611B00F077FC01F0A1FD0028D9D14EF60C
:1080F0000450CEF200004FF080510160BFF34F8F6B
:10810000BFF36F8F02B070BD40F6C810C2F200001E
:108110000168096821B10068C068C068406801E072
:108120004FF0FF3047F69C51C2F2000108607047E3
:1081300070B5044601F0E6FB40F6BC16C2F200063C
:1081400031680546884203D200F008F8012000E0BB
:10815000002020602846356070BD00002DE9F04108
:1081600082B040F6C417C2F200073868016891B3C4
:108170004FF0000809E000BF6060386829462461BC
:1081800000F010FB3868016829B3C068C46806684D
:10819000251D284600F0C6FA216A2046884794F833
:1081A00028004007EED5A0693044B042E4D820460C
:1081B000002132460023CDF8008001F0FBFD0028AD
:1081C000E0D14FF0500080F31188BFF36F8FBFF301
:1081D0004F8F00BFFEE740F6D411C2F200010A68DB
:1081E00008603A6002B0BDE8F081000081B0002074
:1081F000009040F23C10C2F2000000684FF05001C5
:1082000081F31188BFF36F8FBFF34F8F013001D01F
:10821000FEE700BF00980028FCD001B070470000C6
:1082200082B001AC2046FFF7F5FC0199FFF72CFF67
:10823000FFF798FEF6E70000F0B581B0044600F0C5
:10824000E7FA94F94560012E0FDB04F1240500BF25
:10825000286850B1284601F0A1FC002818BF00F0A2
:10826000C9FC70B2013E0128F2DCFF2684F84560AB
:1082700000F0F2FA00F0CCFA94F94470012F0EDB12
:1082800004F11005286850B1284601F087FC002849
:1082900018BF00F0AFFC78B2013F0128F2DC84F88F
:1082A000446000F0D9FA01B0F0BD00002DE9F043C0
:1082B00081B0044600F032FD40F6CC16C2F2000652
:1082C0003068002808BFFFF7B5FC47F66458C2F2D3
:1082D000000898F80000002818BF4FF00040204226
:1082E0000DD0002401F0A2FC60071ED04FF050001A
:1082F00080F31188BFF36F8FBFF34F8FFEE7C4B1D8
:1083000014F0070004F108011EBF081A00F108016B
:108310005FEA41700ED04FF0500080F31188BFF338
:108320006F8FBFF34F8F00BFFEE7204601B0BDE85F
:10833000F083002147F69059C2F20009D9F80000F5
:108340004A1E8242CDD247F60860C2F2000005689C
:108350002F4657F8042F8A4211D22B685BB100BF19
:108360001F4657F8042F28461D468A4207D22B681D
:10837000002BF5D103E047F60860C2F20000336835
:108380009D42AED004682B68521A112A036010D3A4
:108390006818430709D04FF0500080F31188BFF3ED
:1083A0006F8FBFF34F8F00BFFEE742603960FFF76A
:1083B00025FD47F698503968D9F80020C2F2000030
:1083C0000368511A9942C9F8001038BF016098F843
:1083D0000000396800284FF0000018BF41F000414C
:1083E000286047F6A450C2F20000026808343960E1
:1083F000511C016076E70000034648F2ED10C0F61C
:1084000000004FF0807C21F0010103E903106FF0C0
:10841000020043F8240CA3F1440043F8202C7047D9
:1084200022EE034A21EEA25A34EE454A22EE833A66
:1084300021EE825A35EE033A22EE022A22EEA25AA9
:1084400032EE052A34EE044A33EE033A32EE022AC3
:10845000B7EE005A35EE422A24EE000A23EE203A07
:1084600030EE030A22EE011A31EE000A70470000D6
:10847000B0B50C460429054607D3092000F00CF9D5
:1084800040F00401092000F02BF9072C08D860B255
:1084900006A151F8200041F20441C2F20001C86077
:1084A00044EA0501062000F01BF9B0BD00000800F9
:1084B00000001800000038000000780000E0030011
:1084C00000E0070000E00F0000E01F00B0B50C4620
:1084D0000429054607D3092000F0DEF840F0080122
:1084E000092000F0FDF8072C08D860B207A151F868
:1084F000200041F20441C2F20001086145EA040093
:1085000040F08001072000F0EBF8B0BD000008004B
:1085100000001800000038000000780000E00300B0
:1085200000E0070000E00F0000E01F00F0B581B0A0
:10853000102000F0B1F80446112000F0ADF8210140
:1085400041EA101041F21846210648BF00F570407C
:10855000C2F200063080112000F09EF8044612207E
:1085600000F09AF804F00F0140EA0120210748BF0B
:1085700000F570407080132000F08EF8044614203F
:1085800000F08AF80546152000F086F8290141EA36
:10859000043141EA10100027CFF6F077210648BFDA
:1085A00038437060152000F077F80446162000F07C
:1085B00073F80546172000F06FF8290241EA0441DC
:1085C0000844210748BF3843B060182000F064F821
:1085D0000446192000F060F840EA0420B0811A2017
:1085E00000F05AF804461B2000F056F840EA042038
:1085F000F0811C2000F050F804461D2000F04CF8DB
:1086000040EA042030821E2000F046F804461F2075
:1086100000F042F840EA04207082202000F03CF88C
:108620000446212000F038F840EA0420B08201B06E
:10863000F0BD000080B5082000F02EF880BD0000DD
:10864000B0B5002000F028F80446012000F024F81E
:108650000546022000F020F8290241EA04410844BE
:10866000210648BF00F17F40B0BD0000B0B5032037
:1086700000F012F80446042000F00EF8054605202C
:1086800000F00AF8290241EA04410844210648BFE3
:1086900000F17F40B0BD000010B50446FCF71CF9A6
:1086A000EE20FCF7EBF8FCF757F92046FCF7E6F86C
:1086B000FCF752F9FCF710F9EF20FCF7DFF8FCF7B4
:1086C0004BF90020FCF7A8F80446FCF727F92046F0
:1086D00010BD000080B50146082000F001F880BD03
:1086E000B0B50C460546FCF7F7F8EE20FCF7C6F8E7
:1086F000FCF732F918B1FCF711F90120B0BD28469A
:10870000FCF7BCF8FCF728F92046FCF7B7F8FCF7B3
:1087100023F90446002818BF0124FCF7FFF820467F
:10872000B0BD0000D0E9013201699A60D1F804C0FF
:1087300082688445536008BF4A600022026108686D
:10874000013808600868704747F68403C2F20003E6
:10875000036047F28460C2F200000860802010606D
:108760007047000047F6E043C2F20003036047F69B
:10877000E000C2F2000008604FF4807010607047A3
:10878000704700004FF0FF31024642F8081F0021F9
:108790004260C0E9032201607047000000210161CE
:1087A0007047000080B5D1F800C01CF1010207D06D
:1087B00000F108039E465B681A686245FAD901E039
:1087C000D0F810E0DEF8042008614A609160C1F83A
:1087D00008E0CEF8041001680131016080BD00009E
:1087E000D0F800C0436808619A684B608A609A6854
:1087F000996051600CF1010101607047DFF80C00D5
:10880000016841F470010160704700BF88ED00E02D
:108810004FF0500080F31188BFF36F8FBFF34F8F7D
:1088200040F23C10C2F2000001684A1C026001B133
:1088300070474EF60450CEF200000068000608BFF4
:1088400070474FF0500080F31188BFF36F8FBFF374
:108850004F8F00BFFEE7000040F23C10C2F2000064
:10886000016839B10139016018BF7047002080F3F9
:10887000118870474FF0500080F31188BFF36F8F5D
:10888000BFF34F8FFEE70000B0B5002808BFB0BDB2
:10889000044647F66450C2F20000007854F8041C05
:1088A000002818BF4FF0004008420CD0A4F1080582
:1088B0002A6892B14FF0500080F31188BFF36F8F98
:1088C000BFF34F8FFEE74FF0500080F31188BFF3E6
:1088D0006F8FBFF34F8F00BFFEE721EA000044F81F
:1088E000040C00F01BFA47F69051C2F2000154F854
:1088F000040C0A68104408602846FFF77FFA47F620
:10890000A850C2F2000001680131016001F08EF947
:10891000B0BD00004EF21000CEF200000021016058
:10892000816040F20001C2F20001096844F6D352AE
:10893000C1F26202A1FB02124FF0FF3101EB921172
:108940004160072101607047EFF30580102814D3C0
:108950004EF2F031CEF20001405C47F26461C2F2A7
:1089600000010978884208D24FF0500080F3118846
:10897000BFF36F8FBFF34F8FFEE74EF60C50CEF272
:10898000000047F268610068C2F20001096800F463
:10899000E060884298BF70474FF0500080F3118824
:1089A000BFF36F8FBFF34F8FFEE7000047F6C45C45
:1089B0000022C2F2000C00BF5CF8323023B1013259
:1089C000082A08BF7047F7E70CEBC2034CF83210D7
:1089D0005860704770B515460E460446FFF718FFFD
:1089E00094F84400FF2804BF002084F8440094F861
:1089F0004500FF2804BF002084F84500FFF72CFF46
:108A0000A06B28B904F1240031462A4600F014F97D
:108A10002046FFF711FC70BD10B5D8B1044647F2EF
:108A20007860C2F20000006848B14FF0500080F357
:108A30001188BFF36F8FBFF34F8F00BFFEE700F0C9
:108A40006DF920460021FEF77BFF01F0EFF80028CA
:108A500018BF10BD4EF60450CEF200004FF080510A
:108A60000160BFF34F8FBFF36F8F10BDB0B590B1F2
:108A70000D46D1B1044647F27860C2F200000068AA
:108A8000E8B14FF0500080F31188BFF36F8FBFF350
:108A90004F8F00BFFEE74FF0500080F31188BFF307
:108AA0006F8FBFF34F8F00BFFEE74FF0500080F392
:108AB0001188BFF36F8FBFF34F8F00BFFEE700F049
:108AC0002DF947F63860C2F2000000682268904233
:108AD00002EB050102D2914202D309E0914201D397
:108AE000814205D92160081A0021FEF729FF00E024
:108AF000216001F09BF8002818BFB0BD4EF604506D
:108B0000CEF200004FF080510160BFF34F8FBFF3F2
:108B10006F8FB0BD70B50446FFF77AFE40F6C01601
:108B2000002CC2F2000608BF3468251D2846FFF756
:108B3000F9FDA06A18B104F11800FFF7F3FD47F240
:108B40007C60C2F20000016801310160306884423B
:108B50000CD047F27060C2F2000001680139016078
:108B60002046FFF73BF8FFF7CFFA0DE047F6246009
:108B7000C2F200002946FFF733FE47F27460C2F2EA
:108B80000000016801310160FFF766FE47F60460EE
:108B9000C2F200000068E8B13068844218BF70BDBE
:108BA00047F27860C2F20000006840B14FF0500018
:108BB00080F31188BFF36F8FBFF34F8FFEE74EF640
:108BC0000450CEF200004FF080510160BFF34F8F90
:108BD000BFF36F8F70BD000047F6A051C2F20001D5
:108BE0000968016047F63861C2F200010968416016
:108BF0007047000047F64460C2F2000001210160A6
:108C00007047000010B568B10C4640F6C011C2F2C2
:108C1000000109681831FFF7C5FD20460121FEF764
:108C20008FFE10BD4FF0500080F31188BFF36F8F9F
:108C3000BFF34F8FFEE70000B0B590B10D4640F690
:108C4000C011C2F20001096814461831FFF7C8FDCF
:108C5000002C18BF4FF0FF3528462146FEF770FE66
:108C6000B0BD4FF0500080F31188BFF36F8FBFF39A
:108C70004F8F00BFFEE7000010B586B0002405A8A6
:108C800004A903AACDE90444FFF75EFDDDE9032052
:108C900005990023CDE9010147F6A940C0F600007F
:108CA0001CA1009400F0C4FC47F69451C2F20001EC
:108CB000086010B101F044F80446601C20D0012C7B
:108CC0001CD14FF0500080F31188BFF36F8FBFF3BA
:108CD0004F8F47F69C50C2F200004FF0FF31016009
:108CE00047F60460C2F200000121016047F63860D7
:108CF000C2F200000021016000F07EF806B010BD55
:108D00004FF0500080F31188BFF36F8FBFF34F8F88
:108D1000FEE700BF49444C450000000047F2786080
:108D2000C2F20000016801310160704710B547F2DE
:108D30007860C2F20000006830B147F64460C2F2C9
:108D400000000121016010BD47F64460C2F200003E
:108D5000002140F6C0140160C2F200042068006BDC
:108D60000168B1F1A53F0BD14168B1F1A53F07D131
:108D70008168B1F1A53F03D1C068B0F1A53F04D02F
:108D8000206821683431FFF7FBFC47F2806CC2F2A7
:108D9000000CDCF8001040F6D81201EB8103C2F29F
:108DA000000252F8230048B902EB8300A0F114033B
:108DB000B9B153F8140901390028F9D001EB810049
:108DC00002EB800252F8040F4368101D83421360C7
:108DD00001D1586810601068C0682060CCF800109D
:108DE00010BD4FF0500080F31188BFF36F8FBFF3B9
:108DF0004F8F00BFFEE7000080B582B04EF200400A
:108E0000CEF200004CF27021C4F20F11D0F800290C
:108E10004B1C9A4209D14FF0500080F31188BFF3E8
:108E20006F8FBFF34F8F00BFFEE7D0F800298A4253
:108E300009D14FF0500080F31188BFF36F8FBFF35B
:108E40004F8F00BFFEE7017847F264620191FF2176
:108E500001700178C2F200028DF803109DF8031032
:108E600001F05001117047F26861C2F2000107225F
:108E70000A609DF90320B2F1FF3F0CDC0A6800BFD5
:108E80009DF80330013A5B008DF803309DF9033003
:108E9000002BF5D40A600A68032A2DD14FF4E06351
:108EA00003EA02220A6001990170D0F8201941F406
:108EB0007001C0F82019D0F8201941F07041C0F8B5
:108EC0002019FFF727FD40F23C10C2F200000021FC
:108ED0000160FFF793FC4EF63470CEF2000001689B
:108EE00041F040410160FEF7F1FFFFF71FFFFFF780
:108EF0007DF9002002B080BD4FF0500080F3118852
:108F0000BFF36F8FBFF34F8FFEE7000080B54FF0C8
:108F1000500080F31188BFF36F8FBFF34F8F00F0C5
:108F200001FD30B14EF60450CEF200004FF08051FA
:108F30000160002080F3118880BD0000F0B581B091
:108F4000B0B105464843503014460E46FFF7AEF91F
:108F5000074650B1002007F1500287F84600284626
:108F6000314623460097FEF7B5FE384601B0F0BD06
:108F70004FF0500080F31188BFF36F8FBFF34F8F16
:108F8000FEE70000B0B582B068B11D46ABB1F1B9E3
:108F9000EAB14FF0500080F31188BFF36F8FBFF339
:108FA0004F8F00BFFEE74FF0500080F31188BFF3F2
:108FB0006F8FBFF34F8F00BFFEE74FF0500080F37D
:108FC0001188BFF36F8FBFF34F8F00BFFEE751B122
:108FD0004AB94FF0500080F31188BFF36F8FBFF391
:108FE0004F8F00BFFEE750230193019B502B0AD106
:108FF000069B019C012485F846400095FEF76AFE19
:10900000284602B0B0BD4FF0500080F31188BFF386
:109010006F8FBFF34F8F00BFFEE7000070B5F8B150
:1090200004460E46FFF7F4FB2068D4E90F12002532
:1090300002FB0103013901FB0201A563C4E901033D
:10904000FF20E16084F8440084F8450004F110003A
:109050007EB1FFF797FB04F12400FFF793FB18E0C4
:109060004FF0500080F31188BFF36F8FBFF34F8F25
:10907000FEE7016869B100F091FD50B14EF6045071
:10908000CEF200004FF080510160BFF34F8FBFF36D
:109090006F8FFFF7E1FB012070BD00002DE9F04F5D
:1090A00083B00292B8B11D460E460446E9B1022DC6
:1090B00003D1E06B012840F09A8000F00FFC00BB68
:1090C0000298F0B14FF0500080F31188BFF36F8F1A
:1090D000BFF34F8FFEE74FF0500080F31188BFF3CE
:1090E0006F8FBFF34F8F00BFFEE7206C0028DED0EC
:1090F0004FF0500080F31188BFF36F8FBFF34F8F95
:10910000FEE7FFF785FBA06B022D58D0E16B88428C
:1091100055D304F1100801206F464FF0000B0DF1FC
:1091200008094FF0805A00BF0299002900F07B80A7
:10913000C00702D03846FFF74FFDFFF78DFBFFF762
:10914000EDFDFFF765FB94F84400FF2808BF84F8A5
:1091500044B094F84500FF2808BF84F845B0FFF7F5
:109160007BFB3846494600F0EBF900285ED12046EB
:10917000FEF79EFEA0B102994046FFF743FD204650
:10918000FFF75AF800F052FD78B94EF60450CEF2CF
:109190000000C0F800A0BFF34F8FBFF36F8F04E053
:1091A0002046FFF749F800F041FDFFF731FBA06BC7
:1091B000022D04D0E16B88424FF00000B4D220466B
:1091C00031462A46FEF7CCFC54F8241FC9B120468C
:1091D00000F0E4FC08B34EF60450CEF200004FF06D
:1091E00080510160BFF34F8FBFF36F8F15E04FF0D9
:1091F000500080F31188BFF36F8FBFF34F8F00BF14
:10920000FEE750B14EF60450CEF200004FF0805110
:109210000160BFF34F8FBFF36F8FFFF71DFB01207E
:1092200003B0BDE8F08FFFF717FB04E02046FFF71F
:1092300003F800F0FBFC002003B0BDE8F08F000055
:109240002DE9F04381B0E8B11E46914605460F4630
:1092500009B3022E02D1E86B012837D1FFF774FB66
:10926000EFF311884FF0500080F31188BFF36F8F38
:10927000BFF34F8FA86B022E19D0E96B884216D32B
:1092800000203FE04FF0500080F31188BFF36F8F54
:10929000BFF34F8FFEE7286C0028DAD04FF0500064
:1092A00080F31188BFF36F8FBFF34F8FFEE795F800
:1092B0004540A86B284639463246FEF751FCFF2C44
:1092C0000DD0601C85F8450001201BE04FF05000D8
:1092D00080F31188BFF36F8FBFF34F8FFEE755F810
:1092E000240F70B1284600F059FC0146B9F1000F77
:1092F0004FF0010006D000291CBF0120C9F8000072
:1093000000E0012088F3118801B0BDE8F08300007F
:109310002DE9F04F85B0049298B10C46054600291E
:1093200000F0A58000F0DAFAA8B9049898B14FF0DF
:10933000500080F31188BFF36F8FBFF34F8F00BFD2
:10934000FEE74FF0500080F31188BFF36F8FBFF33B
:109350004F8F00BFFEE705F1240005F110090190D1
:1093600002AF0DF1100A4FF000080AE02846FEF7A0
:1093700063FF00F05BFC2846FEF78EFD002840F0FE
:109380008480FFF745FAD5F838B0BBF1000F1DD047
:1093900028462146FEF7D0FBABF10100A8632869FF
:1093A00070B1484600F0FAFB50B14EF60450CEF2D0
:1093B00000004FF080510160BFF34F8FBFF36F8FFC
:1093C000FFF74AFA00200126A0B95FE0049850B1E7
:1093D000B8F1000F02D13846FFF7FEFB4FF001084D
:1093E000012038B952E0FFF737FA002600200028A4
:1093F0004CD000BFFFF730FAFFF790FCFFF708FAF8
:1094000095F84400FF2804BF002085F8440095F833
:109410004500FF2804BF002085F84500FFF71CFA2F
:109420003846514600F08CF800289FD12846FEF7B8
:1094300033FDB0B104990198FFF7E4FB2846FEF72D
:10944000FBFE00F0F3FB00289BD14EF60450CEF259
:1094500000004FF080510160BFF34F8FBFF36F8F5B
:109460008FE72846FEF7E8FE00F0E0FB89E7286C6E
:1094700000283FF457AF4FF0500080F31188BFF33E
:109480006F8FBFF34F8F00BFFEE70026304605B059
:10949000BDE8F08F2DE9F04381B000B39146054659
:1094A0000E4631B3FFF750FAEFF311884FF050003A
:1094B00080F31188BFF36F8FBFF34F8FAC6B24B372
:1094C00095F8447028463146FEF736FB601EFF2FA4
:1094D000A8631CD0781C85F8440001202AE04FF0D6
:1094E000500080F31188BFF36F8FBFF34F8F00BF21
:1094F000FEE7286C0028D5D04FF0500080F311888B
:10950000BFF36F8FBFF34F8FFEE7002012E055F8D7
:10951000100F70B1284600F041FB0146B9F1000F71
:109520004FF0010006D000291CBF0120C9F800003F
:1095300000E0012088F3118801B0BDE8F08300004D
:10954000B0B5D0B10D4611B30446FFF761F947F647
:109550003860C2F2000001682868421C21D047F63A
:10956000A0536268C2F20003D3F800C091421AD33C
:1095700023689C4517D0012422E04FF0500080F36F
:109580001188BFF36F8FBFF34F8F00BFFEE74FF01F
:10959000500080F31188BFF36F8FBFF34F8F00BF70
:1095A000FEE700240CE0891A884206D9401A286098
:1095B0002046FFF711FB002402E000200124286070
:1095C000FFF74AF92046B0BD2DE9F04383B00746C6
:1095D0009000984615468946FEF768FE78B1064623
:1095E0005C20FEF763FE38B10446066354B94FF0C1
:1095F000FF3003B0BDE8F0833046FFF745F90024A3
:10960000002CF4D0DDE90A10002284F85920CDE9BD
:109610000010384649462A4643460294FEF76AFB44
:109620002046FEF7CDF9012003B0BDE8F08300002D
:1096300070B586B00B9CCCB10C9E06B35C2504952E
:10964000049D5C2D25D1049DDDF828C0022586F8F7
:10965000595005AD3463CDE900C50296FEF74AFBCB
:109660003046FEF7ADF9059806B070BD4FF05000DA
:1096700080F31188BFF36F8FBFF34F8FFEE74FF07A
:10968000500080F31188BFF36F8FBFF34F8F00BF7F
:10969000FEE74FF0500080F31188BFF36F8FBFF3E8
:1096A0004F8F00BFFEE70000F0B581B0D0B11D467E
:1096B000174604460E46FFF7ABF8002D1CBF606D41
:1096C000286094F858000221042F84F8581012D80A
:1096D0000125DFE807F023031C262000616D3143DC
:1096E00061651FE04FF0500080F31188BFF36F8F6A
:1096F000BFF34F8FFEE7616D013113D04FF0500083
:1097000080F31188BFF36F8FBFF34F8FFEE7616D5A
:109710000131616506E0022803D1002501283CD112
:1097200003E066650125012837D1261D3046FEF786
:10973000F9FF47F28061C2F20001E06A0A689042D4
:1097400088BF086040F6D81100EB8000C2F200012B
:1097500001EB80003146FFF743F8A06A48B14FF0B3
:10976000500080F31188BFF36F8FBFF34F8F00BF9E
:10977000FEE740F6C011C2F20001E06A0968C96A5A
:1097800088420AD94EF60450CEF200004FF08051C4
:109790000160BFF34F8FBFF36F8FFFF75DF828466F
:1097A00001B0F0BD2DE9F04120B31D461746044637
:1097B0000E46FFF7C9F8EFF311884FF0500080F321
:1097C0001188BFF36F8FBFF34F8F002D1CBF606DEB
:1097D000286094F858000221042F84F8581012D8F9
:1097E0000125DFE807F023031C262000616D3143CB
:1097F00061651FE04FF0500080F31188BFF36F8F59
:10980000BFF34F8FFEE7616D013113D04FF0500071
:1098100080F31188BFF36F8FBFF34F8FFEE7616D49
:109820000131616506E0022803D10025012849D1F4
:1098300003E066650125012844D1A06A48B14FF0D4
:10984000500080F31188BFF36F8FBFF34F8F00BFBD
:10985000FEE747F27860C2F20000006830B147F6D8
:10986000B05004F11801C2F2000015E0261D304688
:10987000FEF758FF47F28061C2F20001E06A0A6811
:10988000904288BF086040F6D81100EB8000C2F219
:10989000000101EB80003146FEF7A2FF40F6C01147
:1098A000C2F20001E06A0968C96A88420AD90698CA
:1098B00000281CBF0121016047F64460C2F200008D
:1098C0000121016088F311882846BDE8F08100007D
:1098D00040F6C010C2F200000068704747F604600E
:1098E000C2F200000068002804BF0120704747F260
:1098F0007860C2F200000068B0FA80F040094000D1
:109900007047000047F63860C2F2000000687047F8
:1099100080B5FFF719F847F63860C2F2000000681A
:1099200080BD00002DE9F04F81B047F27860C2F2AF
:109930000000006840B147F6AC50C2F20000016878
:1099400000240131016092E047F63860C2F2000065
:1099500001684E1C066021D340F6C810C2F2000018
:109960000168096849B14FF0500080F31188BFF3D6
:109970006F8FBFF34F8F00BFFEE740F6D012C2F2E9
:10998000000201681368036047F6A0501160C2F23C
:109990000000016801310160FEF7B6FB47F69C51FB
:1099A000C2F20001086840F6C01A40F6D818864294
:1099B000C2F2000AC2F2000801D2002445E040F6DB
:1099C000C817C2F2000738680024006898B347F24D
:1099D000806BC2F2000B19E0D9F82C00DBF8001004
:1099E000884288BFCBF8000000EB800008EB8000C5
:1099F0002946FEF7F5FED9F82C00DAF80010C96AFE
:109A00003A68884228BF01241068B8B13868C06835
:109A1000D0F80C904D4655F8040F864210D32846D6
:109A2000FEF780FED9F828000028D5D009F11800EB
:109A3000FEF778FED0E74FF0FF3005E04FF0FF3043
:109A400047F69C51C2F200010860DAF80000C06AD3
:109A500000EB800058F82000012847F64460C2F26D
:109A6000000088BF01240068002818BF0124204698
:109A700001B0BDE8F08F00002DE9F0411E4615460B
:109A800088460746FEF7C4FE40F6C014C2F2000442
:109A9000206890F85800022819D02068416D21EA0A
:109AA0000701416520684FF0010180F8581076B138
:109AB00030460121FDF744FF4EF60450CEF200007F
:109AC0004FF080510160BFF34F8FBFF36F8FFEF7F0
:109AD000C3FEFEF79DFE15B12068406D286020682A
:109AE000002590F858100020022905D12168012591
:109AF0004A6D22EA08024A65216881F85800FEF79B
:109B0000ABFE2846BDE8F081B0B580B1044640F612
:109B1000C010C2F200000068A0420AD04FF050000E
:109B200080F31188BFF36F8FBFF34F8FFEE70020E4
:109B3000B0BD206D38B3013820654FF0000018BF6C
:109B4000B0BDE16AE26C91421CD0251D2846FEF7AB
:109B5000E9FDE06CC0F13801A16147F28061E0628B
:109B6000C2F200010A68904288BF086040F6D8112E
:109B700000EB8000C2F2000101EB80002946FEF7F5
:109B80002FFE0120B0BD4FF0500080F31188BFF3CD
:109B90006F8FBFF34F8F00BFFEE70000B0B5C06806
:109BA000C5687DB105F118042046FEF7BBFD47F2FC
:109BB0007860C2F20000006868B147F6B050C2F2A7
:109BC00000001DE04FF0500080F31188BFF36F8F4D
:109BD000BFF34F8FFEE72C1D2046FEF7A3FD47F293
:109BE0008061C2F20001E86A0A68904288BF08609A
:109BF00040F6D81100EB8000C2F2000101EB8000BA
:109C00002146FEF7EDFD40F6C011C2F20001E86A00
:109C10000968C96A884291BF002047F64461C2F2D0
:109C20000001012088BF0860B0BD00002DE9F04FA1
:109C300081B047F27864C2F20004206868B1FEF790
:109C4000E7FD206801382060206880B10024FEF71D
:109C500003FE204601B0BDE8F08F4FF0500080F3C6
:109C60001188BFF36F8FBFF34F8F00BFFEE747F23E
:109C70007060C2F20000006800285DD047F6B05660
:109C8000C2F20006306847F64468C2F2000890B39A
:109C900047F2806740F6D81940F6C01BC2F20007B1
:109CA000C2F20009C2F2000B4FF0010AF068C56869
:109CB00005F11800FEF736FD2C1D2046FEF732FD9B
:109CC000E86A3968884288BF386000EB800009EB99
:109CD00080002146FEF784FDE86ADBF80010C96ABF
:109CE000884228BFC8F800A030680028DED1002DC7
:109CF00018BFFEF709FA47F6AC54C2F20004256813
:109D000055B10126FFF70EFE002818BFC8F8006005
:109D1000013DF7D100202060D8F8000070B14EF668
:109D20000450CEF200004FF080510160BFF34F8F1E
:109D30000124BFF36F8F8AE7002488E7002486E7B9
:109D400080B586B0FDF792FE47F63C60C2F2000097
:109D5000006808B30020CDE9040005A804A903AAFF
:109D6000FEF700FDDDE903200221DDF814C0CDE996
:109D7000001048F22120C0F600000CA10023CDF80D
:109D800008C0FFF755FC47F64061C2F200010860C9
:109D900010B1012006B080BD4FF0500080F3118853
:109DA000BFF36F8FBFF34F8FFEE700BF546D72207C
:109DB0005376630010B584B0A8B147F63C64C2F294
:109DC000000484462068C0B10529CDE90012CDF811
:109DD00008C015DCFFF782FD01462068022916D174
:109DE000069A694615E04FF0500080F31188BFF3E2
:109DF0006F8FBFF34F8F00BFFEE7002004B010BD90
:109E000069461A460023FFF71BFA04B010BD6946E5
:109E100000220023FFF742F904B010BD03B40198FB
:109E20004100009850EAC12018BF04204A0D18BF15
:109E300040F0010040F2FF72B2EB515F08BF40F00A
:109E40000200012808BF052002B070474100080247
:109E500018BF04200A0E18BF40F001004FF07F42E7
:109E600032EA010108BF40F00200012808BF0520C6
:109E70007047000010B54FF00E402DED028BB0EE94
:109E8000408A18EE104A00EB4400B0F1506F4AD8F7
:109E90004FF0FC40B0EB440F22D2B0EEC80AF7EE10
:109EA000000A30EEC00AF6EE000A60EE208A18EED4
:109EB000900A01F0D4FD01EE100A14F0004F1DBF0E
:109EC000DFED2D0A9FED2D0AB1EE411ADFED2C0AD0
:109ED00008BF9FED2C0AF8EE001A21EE218A05E05A
:109EE000DFED290A68EE088AB0EE600A9FED271AB6
:109EF000DFED271A30EE080A48EE811A9FED251A89
:109F000008EEA11ADFED241A48EE811A9FED231AFC
:109F100008EEA11A68EE281ABDEC028B01EE810A48
:109F200030EE200A10BD4FF0E440B0EB440F0CD9E6
:109F300018EE100AFFF78AFF042808BF01F092FC10
:109F4000B0EE480ABDEC028B10BD4FF07F40B0EB85
:109F5000440F07D2B0EE480ABDEC028BBDE81040BA
:109F600001F072BC0120F6F7C5FABDEC028BBDE82A
:109F7000104001F06FBC00000000C9BF22AAFDB96B
:109F80000000C93F22AAFD390000000024FE1C3D4C
:109F9000C78AD83C1E67383D1B93993DAFAA2A3E1D
:109FA00070B59B482DED020B2DED068B079D25F01E
:109FB0000044A04218DC9748844202DC0AD106988B
:109FC00040B19DED060BBDEC068B02B0BDE87040C4
:109FD00001F0F6BB002DCCBF9FED8F0B9FED900BDA
:109FE000BDEC068B02B070BD8F48A04215DD8F48D6
:109FF000A042D8BF4FF0FF3458DD9DED060B51EC69
:10A00000100BFFF70BFF042808BF01F00DFC9DEDBE
:10A01000060BBDEC068B02B070BD9DED060B51EC3E
:10A02000100B01F0D9FCCDE9060181489FED828B30
:10A03000A0423CDD8248A0421FDD00249FED82ABA0
:10A040009DED060B53EC1A2B51EC100B01F064FD47
:10A050009DED060B41EC190B53EC1A2B51EC100B38
:10A0600002F070F853EC182B02F078FA53EC192B2D
:10A0700001F00EFECDE9060149E09DED060B01243D
:10A0800053EC182B51EC100B01F046FD9DED060B27
:10A0900041EC190B53EC182B51EC100B02F05EFA4B
:10A0A00053EC192B01F0F4FDCDE906012FE06848CF
:10A0B000A0421FDD02249FED689B9DED060B53EC33
:10A0C000192B51EC100B02F03DF853EC182B01F05A
:10A0D00023FD9DED060B41EC180B53EC192B51ECB5
:10A0E000100B02F03BFA53EC182B01F0D1FDCDE937
:10A0F00006010CE09DED060B032453EC102B9FEDA5
:10A10000580B51EC100B01F0C3FDCDE906019DED9C
:10A11000060B53EC102B51EC100B02F013F841EC32
:10A12000180B53EC182B02F00DF841EC190B4E48AC
:10A130000621B0EE490AF0EE690A784401F0AAFA65
:10A1400053EC182B51EC100B01F0FCFF41EC180BF9
:10A150004648B0EE490AF0EE690A0521784401F05C
:10A1600099FA53EC192B51EC100B01F0EBFF41EC79
:10A17000100B51EC180B53EC102B002C0EDA01F0E5
:10A18000CBFC9DED061B53EC112B01F0DBFF9DED8D
:10A19000061B53EC112B02F009F935E001F0BCFC71
:10A1A0009DED061B53EC112B01F0CCFF41EC100B85
:10A1B0002F48784400EBC40090ED001B51EC100BCD
:10A1C00053EC112B02F0CAF99DED061B53EC112B39
:10A1D00002F0C4F941EC100B2648784400EBC400AF
:10A1E00090ED001B51EC100B53EC112B02F0DEF83C
:10A1F00041EC100B002DA2BFBDEC068B02B070BD70
:10A2000051EC100B01F04AFC41EC100B01E700008F
:10A21000000010440000F07F182D4454FB21F93F4A
:10A22000182D4454FB21F9BF0000DC3F0000203E04
:10A230000000F33F00000000000000000000F03FBD
:10A240000000E63F000000000000000000000040A9
:10A250000080034000000000000000000000F83F04
:10A26000000000000000F0BF2A2A0000E0290000E2
:10A270006A2900002229000070B56F4E2DED040BF5
:10A280002DED048B82B0DDF824C0DDE907235C42AC
:10A290002CF000411C4341EAD474069D22F000409A
:10A2A000B44205D86C422C4340EAD474B4420BD972
:10A2B0009DED081B9DED060B02B0BDEC048B04B0B8
:10A2C000BDE8704001F086BAACF14054A4F17F645F
:10A2D0001C430BD0022404EAAC7444EAD274054354
:10A2E0009FED578B9FED582B07D015E09DED060B8A
:10A2F00051EC100B01F068FB42E0002C11BF012C67
:10A300009DED060B02B0BDEC048B04BF04B070BD24
:10A31000022C38D0032C3BD00B439FED4D1B9FEDFF
:10A320004E0B0AD0B14218D1B04209D121F0804180
:10A3300020F08040099107900FE0002A15DA10E024
:10A34000474B7B44002C08BF93ED000B0DD0012C34
:10A3500010D0022C17D0032C1AD0B0421DD1002AE5
:10A3600003DAB0EE410AF0EE610A02B0BDEC048BF4
:10A3700004B070BD93ED000B51EC100B01F08EFB9F
:10A3800041EC100BF1E7B0EE480AF0EE680AECE79A
:10A39000B0EE420AF0EE620AE7E7401A00159FEDC0
:10A3A000329B3C28C8BF8DED000B17DCBCF1000FC1
:10A3B000BCBF10F13C0F8DED009B0FDB9DED080B3A
:10A3C00053EC102B9DED060B51EC100B01F060FCD3
:10A3D00001F002FB01F0F8FACDE90001B4B1012C63
:10A3E00010D0022C9FED220B53EC102B9DED000B97
:10A3F00051EC100B19D002F0B1F853EC182B02F00D
:10A40000ADF8BDE7019880F0004001909DED000B94
:10A4100053EC192B51EC100B01F094FD04BF0220FA
:10A42000F6F768F89DED000B9FE702F097F853EC04
:10A43000182B01F0BBFFA3E70000F07F0000000035
:10A44000182D4454FB210940182D4454FB2109C008
:10A45000182D4454FB21F9BF182D4454FB21F93F1A
:10A460005228000000000000000000000000000072
:10A47000075C143326A6A13C70B54FF068422DED61
:10A48000048BF0EE408A18EE900AB0EE608A18EE67
:10A49000101A02EB4003B3F1654F3CBF02EB4102DF
:10A4A000B2F1654F7DD200BFC0F3C753C1F3C752AD
:10A4B0009A1A1B2A09DD10F0004F14BF9FED830A82
:10A4C0009FED830ABDEC048B70BD12F11A0F36DAD2
:10A4D00011F0004F09D010F0004F0CBF9FED7D0A26
:10A4E0009FED7D0ABDEC048B70BD88EE889A19EE55
:10A4F000100AFFF7ABFC042808BF01F0B3F918EE0F
:10A50000900AFFF7A3FC054618EE100AFFF79EFC21
:10A51000044619EE100AFFF799FC042D18BF052D0B
:10A5200008D1042C18BF052C04D1002804BF022038
:10A53000F5F7E0FFB0EE490ABDEC048B70BD4200B8
:10A54000B2EB410F3AD910F0004F19BFDFED630AAB
:10A550009FED630ADFED630A9FED630AB0EE481AD0
:10A560000A46B1EE688A80F00041F0EE418A10465A
:10A570000A1A5200B2F1807F34D2484010F0004FE6
:10A58000DFED5A1A9FED5A2A1DBFBEEE001A70EE7B
:10A59000E10A30EE420AB6EE001A08BF70EEA10AD8
:10A5A00000E040E008BF30EE020AB0EE682A01EE9B
:10A5B000482A08EE818AC2EE081A15E011F0004F11
:10A5C00004BF9FED4C0AF0EE400AD1D010F0004FCE
:10A5D00019BFDFED490A9FED490ADFED490A9FEDFA
:10A5E000490AC5E7C8EE881A21EEA11A9FED462A4E
:10A5F000DFED462A41EE022A9FED452A01EE222A8E
:10A60000DFED442A41EE022A9FED432ABDEC048B84
:10A6100001EE222A21EE811A01EE020A30EE210A11
:10A6200030EE200A70BD4FF07F42B2EB400F28BFE2
:10A63000B2EB410F09D2F0EE480AB0EE680ABDEC69
:10A64000048BBDE8704001F002B940EA01035B00F1
:10A6500008BF41F0FF410BD0B2EB400F08BFB2EB97
:10A66000410F08D120F0804008EE900A21F080418F
:10A6700008EE101A18E7B2EB400F12BF5FEA410371
:10A6800040F0FF4001F000413FF40EAFB2EB410F4C
:10A6900012BF5FEA400200F0004041F0FF413FF48A
:10A6A00003AF4A0092EA40033FF5FEAE002AACBF7A
:10A6B0009FED1A0A9FED1A0A68EE808A28EE008A3A
:10A6C00018EE900A18EE101AEEE60000DB0FC9BF74
:10A6D000DB0FC93FDB0F4940DB0F49C00000C9BF9A
:10A6E00022AAFDB90000C93F22AAFD390060ED3E53
:10A6F000C30ACE3700000000000049C022AA7DBA7C
:10A700000000494022AA7D3A2DAD65BD8FB8D53DE8
:10A710000FB511BE61C84C3EA8AAAABE0000804F6A
:10A720000000802F000000002DE9F04D2DED040BFE
:10A730002DED0E8B94B0DDE92350259CDDF888A02B
:10A7400025F0004624F00048BAF1000F14BF0121A3
:10A75000002101EB4502FC4953184A1093422AD3C9
:10A76000002814BF0123002303EB44030B44F749E3
:10A770008B4220D358EA00019FEDF5AB76D0DFF88D
:10A78000D8B35D4503D1BAF1000F05D188E0BAF125
:10A79000000F08BF002100D0012101EB450111F598
:10A7A000001F08D8002814BF0121002101EB44013B
:10A7B00011F5001F0BD99DED241B9DED220B14B04C
:10A7C000BDEC0E8B04B0BDE8F04D01F003B80027DE
:10A7D000002DBCBFE149884521DAE1498845A8BF81
:10A7E00002271CDAC3451ADCDE4901EB2851142983
:10A7F00008DDC1F1340220FA02F101FA02F28242CC
:10A800000DD108E058B9C1F1140228FA02F101FA99
:10A8100002F2424503D101F00101C1F1020756EAFB
:10A820000A0124D1002C22DA002D18BF022F01D0FA
:10A83000012F0AD00220F5F75DFE14B0BDEC0E8B9F
:10A8400004B0BDE8F04D00F0A3BF0220F5F752FEC2
:10A8500000F09EFF51EC100B01F020F941EC100BC1
:10A8600014B0BDEC0E8B04B0BDE8F08D18E09FED88
:10A87000BE9B9FEDBF8B002871D1B848804522D187
:10A8800005F1804010F5801008BFBAF1000F07D025
:10A89000B3450ADC002CA8BF9DED240BE0DA0DE0E7
:10A8A000B0EE4A0AF0EE6A0ADAE7002C06DA9DED0D
:10A8B000240B51EC100B01F0F1F86FE0AE48784436
:10A8C00090ED000BCCE7D8454DD1002C48DA2EB1E5
:10A8D00086423AD1BAF1000F42D126E0BAF1000F18
:10A8E00013D00220F5F706FE00F08EFF8DED020B6F
:10A8F0009DED220B8DED000B10EE900A039961F394
:10A900001E0003909DED020BAAE78DED029B9DEDCD
:10A91000220B19EE901A10EE900A8DED000B61F3E8
:10A920001E0003909DED020B9AE78DED028B9DEDCD
:10A93000220B18EE901A10EE900A8DED000B61F3C9
:10A940001E0003909DED020B8AE709DA9DED220BB4
:10A9500051EC1A0B53EC102B01F09AF91EE020E099
:10A960009DED220B7CE786421BDAB4F1804F0DD0BF
:10A97000A4F10050B0F1FF5013D1002D11DB9DED7B
:10A98000220B51EC100B01F033F807E09DED220B88
:10A9900053EC102B51EC100B00F0CABC41EC100B27
:10A9A0005EE79DED220B51EC100B01F015F8BAF1AA
:10A9B000000FCDE90A0142D19FED710B46B3A6F11C
:10A9C000E040B0F17F600CD05E4538D1002D00DA58
:10A9D000A7B3022F0CBF01204FF0FF3001F04BFB5B
:10A9E000DCE7002D01DD002C0DDA002D01DD002C4F
:10A9F0001FDB002D16DA002C14DB012F08BF9FEDA2
:10AA0000620B3FF42DAFB0EE490AF0EE690A27E77A
:10AA1000022F18BF002D0CD0012F0AD1002DFFF6F8
:10AA20001FAF06E0002DB8BF002C08DA012F3FF45D
:10AA300017AFB0EE480AF0EE680A11E71BE00120FC
:10AA400000EBE57050EA070115D0791EB0EE4A8A96
:10AA5000F0EE6A8A084308BF9FED4D8B4E480025F3
:10AA6000804570DD4D494E48884514DDB0420DDB10
:10AA7000002C19DB2FE00120F5F73CFD14B0BDECF4
:10AA80000E8B04B0BDE8F04D00F0AEBEB34502DC65
:10AA9000002C09DC1FE0864202DA002C1BDA03E0FE
:10AAA0005E452BDD002C16DD0220F5F723FD00F0BE
:10AAB000ABFE8DED020B53EC192B51EC180B01F092
:10AAC00041FBCDE900010399019861F31E00039059
:10AAD0009DED020BC4E60220F5F70CFD00F0A4FE8C
:10AAE00010EE901A18EE900A8DED020B8DED008B92
:10AAF00061F31E0003909DED020BB1E69DED0A0B84
:10AB000053EC1A2B51EC100B01F028FD9FED260B96
:10AB1000CDE90A0153EC102B9DED0A0B51EC100B03
:10AB200001F010FB9FED221B53EC112B01F03EFCBA
:10AB30009DED0A1B53EC112B01F004FB9FED1E1B36
:10AB400053EC112B3CE08CE0FFFF1F00FFFF0F00D8
:10AB5000000000000000F03F0000F03F0000F07F28
:10AB60000000404301FCFFFF000000000000F07FF8
:10AB70000000000000000000D622000000000000DD
:10AB80000000000000000080000000000000F0FF56
:10AB9000000000000000F0BF0000E0410000F043B2
:10ABA000FFFFEF3F00000000000000000000D03F6A
:10ABB000555555555555D53F000000000000E03F64
:10ABC00001F0F4FB9DED0A0B41EC190B53EC102B3B
:10ABD00051EC100B01F0B6FA53EC192B01F0B2FA5C
:10ABE0009DED0A0B41EC1B0B53EC102B9FEDFE0B64
:10ABF00051EC100B01F0A6FA41EC190B9FEDFC0B88
:10AC000051EC1B0B53EC102B01F09CFA41EC1B0B8D
:10AC10009FEDF90B53EC102B9DED0A0B51EC100B33
:10AC200001F090FA53EC1B2B01F098FC41EC1B0B4C
:10AC300051EC190B53EC1B2B00F06EFF0490CDE987
:10AC400004519DED040B53EC192B51EC100B01F04A
:10AC500085FC53EC1B2B01F0A9FB41EC100B00F021
:10AC6000A9B90020B6F5801F0EDA9FEDE50B53EC75
:10AC7000102B9DED0A0B51EC100B01F063FACDE99E
:10AC80000A016FF034000E4600EB2650A0F2FF37A9
:10AC9000C6F31300DC4940F07F6646F04056884218
:10ACA000D8BF002408DDD9498142C8BF012403DC94
:10ACB0000024A6F580167F1CD548784400EBC40814
:10ACC0000B9698ED000B53EC102B9DED0A0B51ECFD
:10ACD000100B01F043FC98ED000B41EC1B0B53EC07
:10ACE000102B9DED0A0B51EC100B00F015FF41EC01
:10ACF000100B51EC1A0B53EC102B00F0C9FF41EC78
:10AD00001C0B51EC1B0B53EC1C2B01F01BFA41EC00
:10AD1000190BC0488DED0E9B78440E9590ED000BFD
:10AD20004FF0005040EA660000EB84408DED120BBE
:10AD300000F50020139098ED000B53EC102B9DEDC7
:10AD4000120B51EC100B01F009FC9DED0A1B53ECAA
:10AD5000112B01F02BFB41EC100B53EC102B9DED54
:10AD60000E0B51EC100B01F0EDF99DED120B41ECC7
:10AD70001D0B53EC102B9DED0E0B51EC100B01F045
:10AD8000E1F953EC1B2B01F011FB53EC1D2B01F0EF
:10AD9000E5FB53EC1C2B01F0D5F941EC1C0B53ECFB
:10ADA000192B51EC190B01F0CDF941EC1B0B9A4812
:10ADB0000621B0EE4B0AF0EE6B0A784400F06AFC14
:10ADC000B0EE401AF0EE601AB0EE41DAF0EE61DA61
:10ADD00053EC1B2B51EC1B0B01F0B4F953EC1D2B66
:10ADE00001F0B0F99DED0E0B41EC1B0B53EC192B50
:10ADF00051EC100B00F090FE53EC1C2B01F0A2F96B
:10AE000053EC1B2B00F088FE9DED0E0B41EC1B0B51
:10AE100053EC102B51EC100B01F094F941EC1D0B8D
:10AE200053EC1D2B9FED7EEB51EC1E0B00F074FEDE
:10AE300053EC1B2B00F070FE1290CDE912519DEDEA
:10AE4000120B53EC1E2B51EC100B01F087FB53EC53
:10AE50001D2B01F083FB53EC1B2B01F0A7FA9DED9A
:10AE6000120B41EC1D0B53EC102B9DED0E0B51EC16
:10AE7000100B01F067F941EC1B0B53EC192B51EC53
:10AE80001D0B01F05FF99DED120B41EC190B53EC1A
:10AE9000102B51EC1C0B01F055F953EC192B00F061
:10AEA0003BFE41EC190B51EC1B0B53EC192B00F042
:10AEB00033FE0490CDE904519DED040B53EC1B2BA4
:10AEC00051EC100B01F04AFB53EC192B01F06EFA18
:10AED0009DED040B41EC190B53EC102B9FED520B25
:10AEE00051EC100B01F02EF941EC1B0B9FED500BB8
:10AEF00051EC190B53EC102B01F024F99DED040BD0
:10AF000041EC190B53EC102B9FED4B0B51EC100B3C
:10AF100001F018F953EC192B00F0FEFD41EC100B79
:10AF20004748784400EBC40090ED001B51EC100B37
:10AF300053EC112B00F0F0FD41EC190B384601F0F9
:10AF40009AF8CDE90A0153EC192B51EC1B0B00F0D8
:10AF5000E3FD41EC100B3B48784400EBC40451EC9A
:10AF6000100B94ED001B53EC112B00F0D5FD9DED63
:10AF70000A1B53EC112B00F0CFFD0490CDE90451D6
:10AF80009DED0A0B53EC102B9DED040B51EC100BB7
:10AF900001F0E4FA94ED001B53EC112B01F0DEFA02
:10AFA00053EC1B2B01F0DAFA53EC192B01F0FEF9EC
:10AFB00041EC100B9DED241B53EC102B8DED001B71
:10AFC00000959DED240B51EC100B01F0BBF89DEDAD
:10AFD000000B41EC190B53EC102B9DED240B51ECA5
:10AFE000100B01F0BBFA2FE0000000604715F73F9F
:10AFF000FE822B654715F73F44DF5DF80BAE543EEC
:10B0000000000000000040438E9803007AB60B0059
:10B01000BA1D00007C1E0000EA1C000000000000B9
:10B020000000000000000840000000E009C7EE3FFB
:10B03000FD033ADC09C7EE3FF5015B14E02F3EBE8D
:10B04000721B00002C1B00009DED041B53EC112B08
:10B0500001F078F853EC192B00F05EFD9DED040B28
:10B0600041EC190B53EC102B9DED000B51EC100B28
:10B0700001F068F8CDE904019DED040B51EC190BCA
:10B0800053EC102B00F048FDCDE902010C46AA4913
:10B090008C422FDB611A084318D19DED040B53EC51
:10B0A000102B9DED020B51EC100B01F057FA41EC07
:10B0B0001B0B9FEDA30B51EC190B53EC102B00F065
:10B0C0002BFD53EC1B2B01F03BF92DD20220F5F7A1
:10B0D00011FA00F099FB10EE901A18EE900A8DED1F
:10B0E000020B8DED008B61F31E0003909DED020BB2
:10B0F000FFF7B6BB944A24F00041914214D3934920
:10B10000214408437FF4E7AC9DED040B53EC102B76
:10B110009DED020B51EC100B01F020FA53EC192BB2
:10B1200001F00EF97FF6D7AC24F000408849894A37
:10B13000002601EB205182422BDA481C4FF480118B
:10B1400021FA00F02044844AC0F30A517A44A1F263
:10B15000FF3192ED000B814A8DED0A0BCA4020EAC7
:10B160000202C0F3130040F48010C1F1140120FA70
:10B1700001F60B92002CB8BF76429DED0A0B53EC02
:10B18000102B9DED040B51EC100B01F0E7F9CDE90C
:10B1900004019DED040B51EC190B53EC102B00F046
:10B1A000BBFC9FED6F0B0A90CDE90A5153EC102BBD
:10B1B0009DED0A0B51EC100B00F0C4FF41EC1B0B92
:10B1C0009FED690B53EC102B9DED0A0B51EC100B0E
:10B1D00000F0B8FF9DED040B41EC1C0B53EC102B61
:10B1E0009DED0A0B51EC100B01F0B8F953EC192B43
:10B1F00001F0DCF89FED5E1B53EC112B00F0A2FF79
:10B2000053EC1C2B00F088FC41EC190B51EC1B0B90
:10B2100053EC192B00F080FCCDE902019DED020BEF
:10B2200053EC1B2B51EC100B01F098F953EC192B3C
:10B2300001F0BCF89DED020B41EC190B53EC102B07
:10B2400051EC100B00F07EFFCDE90A014A489DED5C
:10B250000A0B0521784400F01DFA9DED0A1B51EC04
:10B26000100B53EC112B00F06DFF9DED021B53EC06
:10B27000112B01F09BF8CDE904019DED020B53EC7D
:10B28000192B51EC100B00F05DFF53EC192B00F063
:10B2900043FC9FED3B0B41EC190B53EC102B9DED48
:10B2A000040B51EC100B01F059F99DED040B41EC2E
:10B2B0001B0B53EC102B9DED020B51EC100B00F00F
:10B2C00041FF53EC1B2B00F0E3FC53EC192B01F076
:10B2D00045F99DED021B53EC112B01F03FF953ECA6
:10B2E0001A2B01F063F8CDE9020101EB06500115BC
:10B2F0000029C8BF039015DC9DED020B324651ECCE
:10B30000100B01F071FBFEF789FD042808BF00F067
:10B310008BFA32469DED020B51EC100B01F064FBF1
:10B32000CDE902019DED020B51EC180B53EC102BF3
:10B3300000F008FFFFF732BB000090400000000063
:10B34000FE822B654715973C00CC904000346F3F40
:10B3500001FCFFFF0000E03F481A0000FFFF0F0064
:10B3600000000000432EE63F396CA80C615C20BE53
:10B37000EF39FAFE422EE63F801800000000000080
:10B38000000000000000004000B510EE101A2DED86
:10B39000028B81B0524A6846B2EB410F2ED94FF072
:10B3A000E640B0EB410F94BF00204FF0FF3000901B
:10B3B0000098B0EE408A00286ADB10F0010F4BD0F5
:10B3C00068EE080A9FED471A9FED470A00EE810AD2
:10B3D0009FED461A10F0020F00EE801AB7EE000A39
:10B3E00000EE810A02BF01B0BDEC028B00BD00BFC0
:10B3F00001B0B1EE400ABDEC028B00BD3C4B21F028
:10B400000042934241D911F0004FDFED3A0A20EE9D
:10B41000201ADFED390A19BF31EE601A71EE200AE9
:10B4200031EE201A71EE600ABDEEE01A11EE100A3C
:10B430009FED321A00F0030000EEC10A9FED301AB2
:10B44000009000EEC10A9FED2F1A00EEC10A9FED99
:10B450002E1A00EEC10AABE728EE080A9FED2B1A60
:10B46000DFED2B0A10F0020F40EE010A9FED291AC2
:10B4700000EE201A61EE000AB0EE480A08EE200A3B
:10B48000B6D101B0BDEC028B00BD00F0F3F98FE73F
:10B4900018EE100A4000B0F17F4F0DD218EE100ADE
:10B4A000FEF7D4FC042808BF00F0DCF9B0EE480A2F
:10B4B00001B0BDEC028B00BD09D10120F5F71AF8EF
:10B4C00001B0BDEC028B5DF804EB00F0C3B901B034
:10B4D000B0EE480ABDEC028B5DF804EB00F0B4B9A5
:10B4E000B61F927EB93AB2BACA9F2A3DDDFFFFBEAF
:10B4F000490E494683F9223F0000004B0000C93F36
:10B5000000A0FD390020A2331A61342C336D4CB9F0
:10B51000DA82083CA0AA2ABE00B510EE101A2DED62
:10B52000028B81B04D4A6846B2EB410F3CD94FF0D7
:10B53000E640B0EB410F94BF00204FF0FF30009089
:10B540000098B0EE408A00285FDB28EE080ADFEDA5
:10B55000440A9FED441A00EE201ADFED430A40EE44
:10B56000010A9FED421A00EE201ADFED410A10F0A9
:10B57000010F40EE010A9FED3F1A00EE201A61EE26
:10B58000000AB0EE480A08EE200A02BF01B0BDEC86
:10B59000028B00BDBFEE001A01B0C1EE000ABDEC87
:10B5A000028BB0EE600A00BD334B21F000429342A3
:10B5B00028D911F0004FDFED310A20EE201ADFED1F
:10B5C000300A19BF31EE601A71EE200A31EE201AEE
:10B5D00071EE600ABDEEE01A11EE100A9FED291A15
:10B5E00000F0030000EEC10A9FED271A009000EE64
:10B5F000C10A9FED261A00EEC10A9FED251A00EE42
:10B60000C10A9DE700F036F99AE718EE100A4000EB
:10B61000B0F17F4F0DD218EE100AFEF717FC042888
:10B6200008BF00F01FF9B0EE480A01B0BDEC028B74
:10B6300000BD09D10120F4F75DFF01B0BDEC028B24
:10B640005DF804EB00F006B901B0B0EE480ABDECBD
:10B65000028B5DF804EB00F0F7B80000B61F927E95
:10B66000BCE9223C0B6D063B8A76CE3CACB5593D1D
:10B6700035A1083E29AAAA3E490E494683F9223F30
:10B680000000004B0000C93F00A0FD390020A2339C
:10B690001A61342C70B504462DED028B4D1E00EB63
:10B6A000C500B0EE408AF0EE608A90ED000B35F0F8
:10B6B000060017D053EC182B51EC100B00F042FD94
:10B6C00041EC100B6D1E04EBC50090ED001B51EC1E
:10B6D000100B53EC112B00F01FFA41EC100B35F05E
:10B6E0000600E7D1022D36D0042D1CD0062D1CBF3C
:10B6F000BDEC028B70BD53EC182B51EC100B00F01D
:10B7000021FD94ED0A1B53EC112B00F005FA53ECCC
:10B71000182B00F017FD94ED081B53EC112B00F0D3
:10B72000FBF941EC100B53EC182B51EC100B00F013
:10B7300009FD94ED061B53EC112B00F0EDF953ECD1
:10B74000182B00F0FFFC94ED040B53EC102B00F0D1
:10B75000E3F941EC100B53EC182B51EC100B00F0FB
:10B76000F1FC94ED021B53EC112B00F0D5F953ECD6
:10B77000182B00F0E7FC94ED001B53EC112B00F0AC
:10B78000CBF9BDEC028B41EC100B70BD000000004A
:10B790009FED070B10B553EC102B9FED070B51ECF1
:10B7A000100B00F075FA41EC100B10BD000000000A
:10B7B0000000000000000000000000000000F03F5A
:10B7C00010B553EC102B51EC100B00F0A5F941EC27
:10B7D000100B10BD10B553EC112B51EC100B00F0F9
:10B7E0009BF941EC100B10BD9FED050B10B553EC10
:10B7F000102B51EC100B00F04BFA41EC100B10BD6C
:10B8000000000000000000009FED050B10B553EC98
:10B81000102B51EC100B00F095FC41EC100B10BDFF
:10B8200000000000000000709FED050B10B553EC08
:10B83000102B51EC100B00F085FC41EC100B10BDEF
:10B84000000000000000001030EE000A704730EEEB
:10B85000200A7047DFED020A80EEA00A7047000060
:10B86000000000009FED020A20EE000A7047000071
:10B87000000000102DE9F0014FF07F42B2EB410FC4
:10B880009FBF4FF0FF310160BDE8F00170474FF0FE
:10B89000004242EA0123C1F3C752783A551112F02F
:10B8A0001F0C434CCCF120067C44C1F3C752A2F1DB
:10B8B00078024FEA621204EB820254F8254008BF76
:10B8C000D2E9015612D0556804FA0CF425FA06F7AD
:10B8D0003C43976805FA0CF527FA06F8D26807FA90
:10B8E0000CFCF24045EA08054CEA0206A4FB034CB6
:10B8F000A5FB0352A6FB03631D449D4234BF0126F2
:10B9000000261319334416B1934202D903E093423F
:10B9100001D2012200E00022624402F1200C9206D2
:10B92000DC0C42EA443200EE102A5B03DFED210A10
:10B93000F8EEC01A00EE103A4FEA9C1C11F0004FCE
:10B94000B8EE400AC0F800C020EE201A00EE105AEF
:10B95000DFED190AB8EE400A20EE200A71EE810AE6
:10B9600070EE800A10EE902A02F500626FF30B026F
:10B9700000EE902A70EEE11A31EEC11ADFED101AD6
:10B9800030EE411A9FED0D0A20EE800A01EE210AE9
:10B990009FED0C1A00EE810A04BFBDE8F00170476C
:10B9A000CCF180510160BDE8F001B1EE400A704772
:10B9B000F4120000000000360000802C22AAFD29AD
:10B9C000DB0FC92F0000C92F10B541EC100BFEF79B
:10B9D000E7FA51EC100B10BD82B0CDE9000121F067
:10B9E000004001909DED000B02B051EC100B704730
:10B9F00000B52DED048B83B041EC190B00F0E2FC97
:10BA000041EC180B18EE100A18EE901A8DED008B11
:10BA1000002818BF0120084320F00040C0F17F60DB
:10BA200000F1E040C00F14D019EE101A19EE900A80
:10BA30008DED009B002918BF0121084320F0004034
:10BA4000C0F17F6000F1E040C00F04BF0120F4F7B7
:10BA500051FD51EC180B03B0BDEC048B00BD10B5CB
:10BA600000EE100A2DED028BB1EEC08A18EE100A1E
:10BA700020F00040C0F1FF40C00F0AD010EE100AC5
:10BA800020F00040C0F1FF40C00F04BF0120F4F7D8
:10BA900031FD18EE100ABDEC028B10BD81F00041A3
:10BAA000704780F00040704721F00041704720F05F
:10BAB0000040704721F0004201F00043A2F16052C3
:10BAC000B2F5801F28BFD2F17F6C0BD95FEA001C52
:10BAD00043EAC20242EB507018BF704728BF20F003
:10BAE00001007047B2F5801FBCBF184670474FEA8F
:10BAF000410C1CF5001F02D2084600F0CBBE70B509
:10BB000000F0CAFB00000089FFF7F6BF4FF00040CD
:10BB1000A0F580007047000010B591EA030F48BF00
:10BB200083F0004300F12285841A71EB030C05D2E7
:10BB3000121943EB0C03001B61EB0C014FEA11548B
:10BB4000A4EB135CDFF81CE11EEA430F18BF9EEA6A
:10BB5000445F00F0748021EA045123EA0E0343F4A9
:10BB60008013DCF1200E32D322FA0CFE10EB0E0013
:10BB700023FA0CFE41EB0E01CCF1200E03FA0EFE6F
:10BB800010EB0E00CCF1200E51F10001B1F5801F39
:10BB900032D201EB045112FA0EF2BDE8104058BF48
:10BBA0007047401C38BF5FEA420218BF7047002848
:10BBB00014BF20F0010041F100014FEA410313F5E9
:10BBC000001F38BF7047A1F1C04100F0B3BB012A8C
:10BBD00043EB0302ACF1200CDCF11F0E32BF4FF03F
:10BBE000000E23FA0CF310EB030041EB0451B4EB0D
:10BBF000115FD0D0A1EB045101F58011490801EB90
:10BC000004515FEA30000ED350F1000038BF12FA41
:10BC10000EFE08D1BDE81040C9E7401C38BF5FEAFE
:10BC20004202CAD1C3E7BDE810404FEA410313F511
:10BC3000001F38BF7047A1F1C04100F07BBB9EEAF6
:10BC4000445F08D011EA5E0FBDE8104004BF01F068
:10BC5000004100207047BDE8104070B500F01CFBAB
:10BC600064FBBE3E0000E0FF02494FF0000000F020
:10BC700089BE00BF0000F87F491058BFC1F14041A4
:10BC80005B1058BFC3F140438B42EFF30080704715
:10BC90002DE9C04130B4DFF8A4C23CEA111418BF4A
:10BCA0003CEA131400F0ED801CEA111481EA03054C
:10BCB00044EAD57418BF1CEA131500F0C880A4EB41
:10BCC000050404F17F7404F500344FF0004545EAA3
:10BCD000C12145EAC32341EA505143EA52534FEA96
:10BCE000C0204FEAC222994208BF904200F09D80D6
:10BCF0004FEA13650FF24416765D4FEA134506FBD3
:10BD000005F7C7F1807706FB07F74FEAD737A7FBA0
:10BD100003687642A7FB06CEC8F5803838BFA8F185
:10BD2000010807FB08E6A6FB028C4FF0000EE6FBBD
:10BD300003CEDCF1000CCEF1004E38BFAEF1010EA7
:10BD4000A6FB0C584FF00007E6FB0E87A1FB08C6C8
:10BD5000A0FB07CE16EB0E064FF0000545F10005DF
:10BD6000E1FB076515F1E04E7EBFA4F580345FEA84
:10BD700046066D4116F1800745F100054FEA172789
:10BD800047EA05674FEA15254FEA0666A6F1DE4643
:10BD9000B6F1805F20D9384605EBC47124F0010C60
:10BDA00001EB0C11BCF1FE6F02D8F0BCBDE80081C4
:10BDB00024425CBF01F5801E9EEAC47F02D4F0BC21
:10BDC000BDE80081244200F13980A1F1C041F0BCFE
:10BDD000BDE8004100F0AEBA4FEAD02040EA415041
:10BDE0004FEAD1214FEAD22242EA43524FEAD3230B
:10BDF000A7FB028607FB036605FB02661EEA0E0F21
:10BE000058BFA6EB0056B6EB00564FEA520E4EEA6C
:10BE1000C37E18EB0E0E56EB530EBCD518EB020882
:10BE20005E417F1C55F10005B5E74FF480154FF0DA
:10BE300000074FF000064FF00008ACE701F1C041E9
:10BE400001F000414FF00000F0BCBDE800810CEAB9
:10BE5000131511EA0C1F00D00CE013EA0C1F00F0C0
:10BE600026804FF0000081EA030101F00041F0BCA0
:10BE7000BDE80081F0BCBDE8004181EA030100F0AB
:10BE800059BAF0BCBDE8004170B500F005FA00BF3A
:10BE9000097EFC3E00F007B84FF0000081EA030184
:10BEA00001F00041704781EA030100F043BAF0BCA1
:10BEB000BDE8004122494FF000007047FFFDFBF94B
:10BEC000F7F5F4F2F0EEEDEBE9E8E6E4E3E1E0DECD
:10BED000DDDBDAD8D7D5D4D3D1D0CFCDCCCBCAC83F
:10BEE000C7C6C5C4C2C1C0BFBEBDBCBBBAB9B8B766
:10BEF000B6B5B4B3B2B1B0AFAEADACABAAA9A8A859
:10BF0000A7A6A5A4A3A3A2A1A09F9F9E9D9C9C9B26
:10BF10009A999998979796959594939392919190D1
:10BF20008F8F8E8E8D8C8C8B8B8A89898888878762
:10BF30008685858484838382828181800000FF07D7
:10BF40000000F87F51EA030C17D41CF5801F58BF7E
:10BF5000BCF5801F00F10680994218BF704708BFEA
:10BF60009042704707D711F5801F58BF13F5801F07
:10BF700019D499427047894270471CF5801F08D533
:10BF8000BCF5801FF7D58B4218BF704708BF8242AF
:10BF900070474FF4001C1CEB410F38BF1CEB430FE4
:10BFA00001D28B42704770B500F076F992244900B7
:10BFB0004FF000514FF08053FFF75EBE4FEA410350
:10BFC0004FEA5353A3F58063D3F11E03C8BFD3F1E7
:10BFD000210C0CDD4FF0004242EAC12242EA5052ED
:10BFE00032FA03FC8CEAE17CACEBE1707047102B79
:10BFF000C4BF0020704703F5787CBCF1FF3F04D03C
:10C000006FF0004282EA2100704770B500F044F9F9
:10C010004992248000207047F2E700004FEA115354
:10C02000A3F58063D3F11E03A8BFD3F1200C08DB76
:10C030004FF0004242EAC12252EA505232FA03F073
:10C04000704709420BD4102BC4BF0020704703F582
:10C05000787CBCF1FF3F05D04FF0FF3070474FF0C8
:10C060000000704770B500F017F900BF49922480B6
:10C0700000207047F0E710F0004248BF4042B0FA9D
:10C0800080F310FA03F10AD0C3F11D0303F58063B6
:10C0900002EB03524FEA415002EBD12170474FF0BF
:10C0A00000007047B0FA80F310FA03F10AD0C3F130
:10C0B0001D0303F580634FEA03524FEA415002EB40
:10C0C000D12170474FF000007047000051EA030C87
:10C0D00017D41CF5801F58BFBCF5801F00F10680E7
:10C0E000994218BF704708BF9042704707D711F5B3
:10C0F000801F58BF13F5801F19D499427047894299
:10C1000070471CF5801F08D5BCF5801FF7D58B4202
:10C1100018BF704708BF824270474FF4001C1CEBE9
:10C12000410F38BF1CEB430F01D28B42704770B5F3
:10C1300000F0B2F8922449004FF000514FF08053C4
:10C14000FFF79ABD70B5DFF848C11CEA111E1EBF8B
:10C150001CEA13159EEA0C0F95EA0C0F00F06F8095
:10C1600081EA03044EEAD47EAE4421EA4C1123EA6C
:10C170004C1341F4801143F48013AEF17F7EA1FB98
:10C18000024CA0FB0365361955EB0C05A1FB034CD3
:10C190004CF10003A0FB021C16EB0C06654153F1A9
:10C1A0000003094218BF46F0010613F4007F0BD1CB
:10C1B0004FEA03314FEA053041EA155140EA165083
:10C1C00034036FF003020AE04FEAC3214FEAC520AF
:10C1D00041EA555140EA5650F4026FF0020202EB78
:10C1E0002E4201EB025585EACE710AD05FEA440C7B
:10C1F00018BF24F0004450F1000041F1000120EA92
:10C20000D47040F2FE7C624500D270BDA84214BFDB
:10C210004FF080444FF04044002E08BF0024BEF190
:10C22000806FA8BFA1F1C041BDE8704080F282805C
:10C2300001F1C04101F000414FF0000070470CEAED
:10C2400013159EEA0C0F18BF95EA0C0F06D081EA71
:10C25000030E4FF000000EF0004170BD00F01CF81E
:10C260008900013E00F007B800F009B84FEA430C1E
:10C270005FEA5C5C08D081EA030100F05BB84FEA3A
:10C28000410C5FEA5C5CF6D102494FF00000704758
:10C290000000FF070000F87F0EF1020E2EF0030EE3
:10C2A0005EF8046B364205D4012A43EB030515F50D
:10C2B000001F12D8012841EB010C1CF5001F0CD8FF
:10C2C0000ED14FEAD17C0CEB4C0C0CF1020C15F5A5
:10C2D000001F08BF4CEBD37C04E04FF0080C01E0DA
:10C2E0004FEAD37C0CEB4C0526FA05F606F0070660
:10C2F000B6F1040C06D20EEB860CBDE870404CF093
:10C30000010C6047DFE80CF0090B02024FF000411E
:10C31000A1F500214FF0000070BD1946104601281C
:10C3200051EB010418BFD4F5001484BF002001F0C4
:10C33000004170BD0808A0F500114FEA31017047B7
:10C3400053EA010C17D41CF5801F58BFBCF5801FA1
:10C3500000F106808B4218BF704708BF82427047C9
:10C3600007D713F5801F58BF11F5801F19D48B42D2
:10C3700070479B4270471CF5801F08D5BCF5801F95
:10C38000F7D5994218BF704708BF904270474FF4E5
:10C39000001C1CEB430F38BF1CEB410F01D299422C
:10C3A00070470FB40CBC03BCFFF7C1BE10B591EAD7
:10C3B000030F81F000413FF5B7AB83F0004300F07D
:10C3C000D5B800002DE9F04101F5801CBCF5001F37
:10C3D000C0F2A9804FEA115C21EA0C5141F48011AE
:10C3E0000CF1FD0C5FEA5C0C0CF5C07C01D3400045
:10C3F0004941890241EA905187022EA48E0EA45D24
:10C400000A0C04FB04F602FB06F6C6F14046A4FB48
:10C410000662F60D46EA422606FB06F4A4FB01235B
:10C420005242C3F1404338BF5B1EA6FB02420024C8
:10C43000E6FB0324D20B42EA4446A6FB0623A1FBFB
:10C4400002E2A3FB07E4E3FB61426442C2F1404E17
:10C4500038BFAEF1010EA6FB04234FF00002E6FB4D
:10C460000E32A2FB03463400E2FB6264A1FB06E647
:10C47000A4FB07E8E4FB61687642C8F1405838BF86
:10C48000A8F10108A2FB06E4A3FB08E5E2FB68545F
:10C49000A1FB05E6A7FB04E8E1FB648618F1200593
:10C4A00056F10006A80940EA8660B109A8F11B0808
:10C4B00008F03F08B8F10A0F1CD901EB0C51BDE898
:10C4C000F08100BFFCF5EEE8E2DDD8D3CFCBC7C3E7
:10C4D000C0BDB9B6B4B1AEACA9A7A5A3A19F9D9BA1
:10C4E0009A9896959392908F8D8C8B898887868564
:10C4F00084838281A0FB006800FB01F208EB420804
:10C50000B8EB872807D5341858EB0104D5D5401C63
:10C5100051F10001D1E7341A78EB0104CDD4401E6B
:10C5200071F10001C9E75FEA4C0C5FEA9C5C0DD138
:10C5300005D301F000414FF00000BDE8F081BDE8F7
:10C54000F04170B5FFF7A8FE6DDBFFBEBDE8F0411E
:10C5500001494FF0000070470000F87F10B591EAE4
:10C56000030F48BF83F000433FF5DEAA841A71EB46
:10C57000030C07D28CF0004C121943EB0C03001B88
:10C5800061EB0C014FEA1154A4EB135CDFF8A4E15A
:10C590001EEA430F18BF9EEA445F00F0B48021EA10
:10C5A000045123EA6E035242C3EB6E0338BF5B1E95
:10C5B000DCF1200E25D322FA0CFE10EB0E0043FA1C
:10C5C0000CFE41EB0E01CCF1200E03FA0EFE10EB37
:10C5D0000E00CCF1200E51F1000129D401EB0451E1
:10C5E00012FA0EF2BDE8104058BF7047401C1CBF45
:10C5F000B2F1004F704700280CBF491C20F0010029
:10C60000704712EB020E43EB030218BF4FF0010E0E
:10C610004EEA4202ACF1200CDCF11E0E56D943FA70
:10C620000CFE10EB0E00CCF11E0E51F1FF31D5D5F2
:10C630000EF1010E12FA0EFE404141EB010101EB39
:10C64000445C5FEA5C5C10D901EB045110EBDE70D6
:10C6500038BFBEF1004FBDE8104018BF704700283A
:10C660000CBF491C20F00100704734D24FEAD42C93
:10C6700024F4006411F500111BD0B1FA81F20B3AD9
:10C68000A41AA41ED2F12003914030FA03F31943F7
:10C69000904001EBCC7101EB0451002CBDE810403F
:10C6A000A8BF704701F1C04101F000414FF0000008
:10C6B0007047B0FA80F310FA03F102D1BDE81040E0
:10C6C0007047E41A173C4805C90AE2E701EB045138
:10C6D000BDE81040704749104FEA300001EB0451AB
:10C6E000BDE8104002E04FF0000170474A0008BF6B
:10C6F0000042F8D0B2F5001F28BF704701F000419A
:10C700004FF0000070479EEA445F07D011EA5E0FC9
:10C71000BDE8104004BF002100207047BDE8104074
:10C7200070B5FFF7B9FD00BF40DFF63E104683F05D
:10C73000004170470000E0FF43004FEAD30C4FEA8E
:10C740003C0C43401FBF40070CF1605113F0FE4FFB
:10C7500070471CF0006F03D10CF0004100207047BF
:10C760000CF0004343EA507040EACC0010B500F0F2
:10C770003EF800BF000000924FEA0001FFF7DABD6B
:10C780004FF00041A1F500214FF0000070474FF03D
:10C790007E5209E011F0004204D54042C1F100018F
:10C7A00038BF491E42F07E5202F170620B0012BF88
:10C7B00020235FEA00017047B1FA81FC01FA0CF115
:10C7C000A3EB0C0320FA03FC41EA0C0102EBC35279
:10C7D000C3F1200310FA03FC5CEA416C42EB112028
:10C7E00018BF5FF0806C28BF20F0010070470EF189
:10C7F000020E2EF0030E5EF8044B244204D44FEADE
:10C800004102B2F17F4F11D84FEA4003B3F17F4F9D
:10C810000CD80ED14FEAD07C0CEB4C0C0CF1020C76
:10C82000B2F17F4F08BF4CEBD17C04E04FF0080C15
:10C8300001E04FEAD17C0CEB4C0324FA03F404F042
:10C840000704B4F1040C06D20EEB840CBDE81040D2
:10C850004CF0010C6047DFE80CF0070802024FF0D3
:10C860000040A0F5800010BD0846420018BFD2F17C
:10C87000807288BF00F0004010BDF1EE100A4FF644
:10C88000FF71C0F2C03120EA010040F04070E1EEDB
:10C89000100A7047FF2141EAD050C00570470000E0
:10C8A000C2154FEA002318BF43F0004300F1108087
:10C8B000D2F1BE0240F2288023FA02F1B2F1200C3C
:10C8C0002EBF23FA0CF0C2F1200C03FA0CF07047D3
:10C8D000B0F15F4F00F2188012F0FF0208BF23F0A2
:10C8E0000043C2F1BE0223FA02F1B2F1200C2EBFC6
:10C8F00023FA0CF0C2F1200C03FA0CF04042C1F113
:10C90000000138BF491E704710B5FFF770FF00BF28
:10C91000922449804FF00001002070476FEAE070D8
:10C9200080F0004170470000C2154FEA002318BF95
:10C9300043F000430ED4D2F1BE0215D323FA02F124
:10C94000B2F1200C2EBF23FA0CF0C2F1200C03FA36
:10C950000CF070474FEA400CBCF1FE4F04D24FF090
:10C9600000004FF00001704710B5FFF740FF00BF17
:10C97000922449804FF00001002070476FEAE07078
:10C98000014670470CF00F03092B08BF082000F088
:10C9900059800A2B0BD0082B18BF704708BF1CF01A
:10C9A000400F0AD04FF000004FF0000170471CF01C
:10C9B000400F18BF4FF0004070471CF0100F08D018
:10C9C00000F07F4220F0704342EAD3014FEA437007
:10C9D000704700F0604021F07F4242EA000201F01F
:10C9E0007F4040EA727070474FF0FF0C4CF4E06CEF
:10C9F0001CEA11531CBF9CEA030C9445C2BFDA42E7
:10CA000001EB02517047002B0DD0BCF1000F0FD08D
:10CA100001F00041002AA4BF41F0E04141F07F61F4
:10CA20004FF00000704701F000414FF000007047E8
:10CA300050EA01334FF09B0C18BF4CF0806C7FF430
:10CA400013A970471CF4801F11D01CF4E02F03D0F1
:10CA50006FEACC31490070474FF04050EFF300824D
:10CA600022F0704242EA000282F3008870474FF0E1
:10CA70000000704700000000000000000000F03FD0
:10CA8000000000000000F83F00000000000000006F
:10CA90000000004003B8E23F00000000000000007A
:10CAA00006D0CF43EBFD4C3E033333333333E33F08
:10CAB000FFAB6FDBB66DDB3F4D268F515555D53F34
:10CAC00001411DA96074D13F65DBC9934A86CD3F02
:10CAD000EF4E454A287ECA3F3E5555555555C53FF0
:10CAE00093BDBE166CC166BF2CDE25AF6A56113FE2
:10CAF000F16BD2C541BDBBBED0A4BE726937663EE4
:10CB00004FBB610567ACDD3F182D4454FB21E93F65
:10CB10009BF681D20B73EF3F182D4454FB21F93F54
:10CB2000E2652F227F2B7A3C075C143326A6813CDA
:10CB3000BDCBF07A8807703C075C143326A6913C85
:10CB4000C4EB98999999C9BF711623FEC671BCBFF1
:10CB50006D9A74AFF2B0B3BF9AFDDE522DDEADBF59
:10CB60002F6C6A2C44B4A2BF0D5555555555D53F71
:10CB7000FF8300922449C23F6E204CC5CD45B73F8C
:10CB8000513DD0A0660DB13FEB0D76244B7BA93F04
:10CB900011DA22E33AAD903F0000000000000000EF
:10CBA000000000006E83F9A22915444ED15727FCDE
:10CBB000C0DD34F5999562DB4190433CAB6351FE97
:10CBC000000000000000000001020304060708093D
:10CBD00000000000010203041000000000000240F9
:10CBE00001000000000402401000000000080240A4
:10CBF0002000000000080240080000000018024069
:10CC00004000000000180240480700200800000013
:10CC1000B806002004000000B8060020080000004C
:10CC2000B80600200C000000B8060020000000003C
:10CC30000007002000000000900700200000000016
:10CC4000900700200400000090070020080000006A
:10CC50007CCD000800000000000000000000000083
:10CC600000000000000400001800000000000000A8
:10CC70000000000086CD0008000000000000000059
:10CC80000000000000000000000400001800000088
:10CC9000000000000000000078CD00080000000047
:10CCA0000000000000000000000000000004000080
:10CCB0001800000000000000000000008CCD0008FB
:10CCC0000000000000000000000000000000000064
:10CCD0000004000018000000000000000000000038
:10CCE000A1CD0008000000000000000000000000CE
:10CCF0000000000000040000300000000000000000
:10CD00000000000097CD00080000000000000000B7
:10CD100000000000000000000008000018000000F3
:10CD200000000000000000006CCD000800000000C2
:10CD300000000000000000000000000000020000F1
:10CD40001800000000000000000000009A99993EC1
:10CD50000000803F0AD7233C000000000000803F15
:10CD60000000803F00000000000000006465666174
:10CD7000756C745461736B00636D640061747469E5
:10CD80005F6573746900626C696E6B0068656967E2
:10CD900068745F63616C00717561645F6374726C69
:10CDA000005461736B5F496E69740000D0CD000858
:10CDB0000000002040010000C401000860CE00080F
:10CDC000400100200883000020020008000000004D
:10CDD000111324F41012022B073D63ADC1BA503A6F
:10CDE00033BBD3F2C93A64126412FA27E8039A9962
:10CDF000993E23803F47D0408FC2F53C18089A994E
:10CE0000193E21B03218A11DCDCC4C3F0439141964
:10CE1000080A2C3D20180F803FB81E053EEC513803
:10CE20003E0AD7A33B044A3D2C0B4570412039C430
:10CE300029787119D083404049303A0C103C0AD708
:10CE400023E41CCDCCCC347AF0602DC1B8323E0442
:10CE50001918373D6666663F0132101AAA010000B4
:040000050800018965
:00000001FF
